:10000000403300202D1300000DD300001913000011
:10001000191300001913000019130000000000005C
:10002000000000000000000000000000F1130000CC
:1000300019130000000000009113000019130000C4
:10004000BD1500001D590000BD150000BD150000C4
:10005000BD150000BD150000BD150000BD15000058
:10006000BD150000BD150000BD150000BD15000048
:10007000BD150000BD150000BD150000BD15000038
:10008000BD150000BD150000BD150000BD15000028
:10009000BD150000BD150000BD150000BD15000018
:1000A000BD150000BD150000BD150000BD15000008
:1000B000BD150000BD150000BD150000BD150000F8
:1000C000BD150000BD150000BD150000BD150000E8
:0C00D000BD150000BD150000BD150000AE
:1000E0007BB972B90029BEBF00204FF0004106E085
:1000F00008BF00281CBF6FF000414FF0FF3000F038
:1001000057B8ADF1080C6DE904CE002909DB002BCE
:100110001ADB00F04FF8DDF804E0DDE9022304B05B
:100120007047404261EB4101002B1BDB00F042F8BD
:10013000DDF804E0DDE9022304B0404261EB410157
:10014000524263EB43037047524263EB430300F0B8
:1001500031F8DDF804E0DDE9022304B0404261EB50
:1001600041017047524263EB430300F023F8DDF88E
:1001700004E0DDE9022304B0524263EB430370471D
:1001800053B94AB9002908BF00281CBF4FF0FF31FE
:100190004FF0FF3000F00CB8ADF1080C6DE904CE63
:1001A00000F008F8DDF804E0DDE9022304B0704750
:1001B000704700BF2DE9F04786468C460846089EEA
:1001C000154674461946002B40F0C2808542B2FAAB
:1001D00082F245D94AB1C2F1200300FA02FC2EFA9C
:1001E00003F3954043EA0C0C94404FEA154EA8B235
:1001F000BCFBFEF8230C0EFB18CC08FB00F943EA0D
:100200000C43994528D9EB1808F1FF3704D29945DA
:1002100002D9A8F102072B44A3EB0903A4B2B3FB54
:10022000FEFC0EFB1C330CFB00F044EA0344A0422E
:1002300014D92C190CF1FF3304D2A04202D9ACF12D
:1002400002032C44241A43EA07401EB1D440002381
:1002500034607360BDE8F0874746DDE76346F1E749
:1002600092BB431B01214FEA154EAFB2B3FBFEFC1C
:10027000200C0EFB1C330CFB07F840EA03439845A7
:1002800062D9EB180CF1FF3004D2984502D9ACF1D9
:1002900002002B44A3EB0803A4B2B3FBFEFC0EFB4D
:1002A0001C330CFB07F744EA0344A7424ED92C1930
:1002B0000CF1FF3304D2A74202D9ACF102032C4463
:1002C000E41B43EA0040C0E7C2F1200320FA03F137
:1002D000954090402EFA03F303434FEA154EAFB218
:1002E000B1FBFEFC0EFB1C10190C0CFB07F841EADD
:1002F0000041884504FA02F422D969180CF1FF3054
:1003000004D2884502D9ACF102002944A1EB0801CE
:100310009BB2B1FBFEFC0EFB1C110CFB07F743EA82
:1003200001439F420ED9EB180CF1FF3104D29F42DA
:1003300002D9ACF102012B44DB1B41EA004192E7F8
:100340006046E3E76146F7E76046A3E76346B7E741
:10035000834206D916B9002108467BE7C6E900E0CA
:10036000F9E7B3FA83F78FB9834201D3724508D80E
:10037000BEEB020460EB030301209C461EB9002182
:1003800068E73846FAE7C6E9004CF8E7C7F1200C01
:10039000BB4022FA0CF41C432EFA0CF120FA0CF3A9
:1003A000B84001434FEA14490EFA07F5B3FBF9F8D8
:1003B0001FFA84FE09FB18300B0C08FB0EFA43EA07
:1003C00000439A4502FA07F240D9E31808F1FF30DA
:1003D00004D29A4502D9A8F102002344A3EB0A03F0
:1003E00089B2B3FBF9F809FB183308FB0EFE41EAAA
:1003F00003418E452CD9611808F1FF3304D28E4594
:1004000002D9A8F10203214443EA0040A0FB02986C
:10041000A1EB0E014145CE46434602D306D14D45E0
:1004200004D2B9EB020E68EB04030138002EA6D00B
:10043000B5EB0E0261EB030101FA0CFC22FA07F3A3
:100440004CEA0303F940C6E9003198E74046C5E7A6
:100450004346D9E7000000002DE9F041684C94F8CC
:1004600032308CB003F00103002800F08A80002BAA
:1004700040F0A980627E94F8253004EB820204EB00
:100480008303D5699F6A0DB32E4616F8020BC0F39D
:10049000801003F09DFF0368C5F802308388B380A5
:1004A0002B785B0606D50621304602F06DFC00284D
:1004B00000F095803E4616F8020BC0F3801003F062
:1004C00087FF0368C7F802308388B380237D01214A
:1004D000C3F302030BA88DF82C3002F0BFFD0246D7
:1004E00000287AD03946284604F0B2FF4549464BE9
:1004F000A0FB0101C0184FF0000541F107013EA328
:10050000D3E90023C4E902552570FFF739FE278E91
:10051000606003F033FF0694029562683B4B0492DF
:1005200000F109063A4802F247121A60A7FB0001DF
:100530000993912303FB0711364B0793364B059321
:100540004FF6FF734FF002080AAF03932AA3D3E9D3
:100550000023CDF828800897FFF712FE03210190B1
:10056000334642460095284603F04EFE394604F0D5
:1005700077F990BB94F8323043F0010384F83230BD
:1005800021E003B3204604F07DF9844229D10BAD6C
:10059000022203211F4B009500200B9203F0ACFEBA
:1005A000294604F05DF990B91C4804F089F9D0B9E6
:1005B000134804F073F9844219D194F832306FF380
:1005C000000384F8323000200CB0BDE8F0810C4804
:1005D00004F064F9844200D000DE0C20F4E712201D
:1005E000F2E700DED3E77830E2D000DEE0E700DEBD
:1005F000E3E700BFAFF300808D49FD1A070000005C
:10060000A015002000CA9A3B8C49FD1A94150020C1
:10061000002AE78449440000C5540000B0150020BA
:1006200070B5037D8AB0C3F302030D460446012171
:100630000DF1230016468DF8233002F00FFD3146F0
:100640000246284604F004FF1F49204AA0FB01315E
:10065000981841F107011AA3D3E90023FFF790FD91
:1006600063689842054621D21B1A00220192184A5B
:100670000293184BA21AA3FB023202211209002393
:100680000A4409AE099114490591CDE903330321C8
:10069000D2B206960093184603F016FE314604F0D7
:1006A000DFF838B9656000200AB070BDFBD9C21A06
:1006B0000023DBE70C200AB070BD00BFAFF3008061
:1006C0008D49FD1A0700000000CA9A3B8C49FD1AAB
:1006D000A01500204FECC44E49440000000000006B
:1006E000F0B583B0C468054606F09CF8002006F01B
:1006F000EBF80021084606F0D9F800222521082051
:1007000006F016F9304B019301A806F0FDF82F49C9
:1007100040F25B6006F0A6F92379C3F3020262F3AC
:10072000C5032371204605F0F7FE27682E6838467A
:1007300005F0BEFB06446A6806F10901012006F0D7
:10074000B1FA06F03DFB204604F0FEFF811C324664
:10075000C9B2384605F0AEFB40B9204605F084FB2F
:1007600010B9002003B0F0BD00DEFAE70546184AD4
:100770001849194840F211430CF0F9FB174B0721B7
:10078000A5FB030301FB05310DA3D3E90023FFF70C
:10079000F7FC1349024613480CF0E9FB002585F3EA
:1007A0001188BFF36F8F0323184602DF0E482146DE
:1007B00006F00CF806F000F96FF08B00D2E700BFEE
:1007C00000CA9A3B00000000D6BE898E55555500E0
:1007D00040FC00008CFC000090FC00008D49FD1ADC
:1007E000DCFC0000B0FC0000D5610000000000004F
:1007F000032973B50546144660D8002A40D0072A5D
:100800005CD15A681C683848D1171346C4FB0031C4
:10081000012B71F1000225DB00F56E1000F65D7012
:1008200018182FA3D3E9002341F10001FFF758FC6A
:1008300080B202281ED004281ED008281ED01028FE
:1008400033D1032329492A6951F8231011615268D1
:1008500014691B01302223212846A44602B0BDE8BA
:10086000704060472248181861F100011CA3D3E9C9
:100870000023DBE70023E5E70123E3E70223E1E7C9
:100880001A881C4B33F8021B8A420BD12E697368FD
:100890000DF107029B68202128469847002807DAB7
:1008A00002B070BD01340B2CECD16FF01500F7E7EE
:1008B0009DF80720130704D4082C05D16FF085009C
:1008C000EEE70A2C08BF0924736802F00F0242EA1F
:1008D0000412DB68D2B2202128469847E0E700BF27
:1008E0003AA395000000000040420F00D00700200E
:1008F000632EB5FF64FF000010B50B4C20460EF0D0
:100900006FF978B12269A168136843F0010313609D
:100910000B684FF00112002120469847B0FA80F092
:10092000400910BD0120FCE76CF7000037B5044614
:1009300009480569836801A95B68984720B92A6856
:10094000019B534003F00100B0FA80F35B090020E3
:10095000237003B030BD00BF6CF7000008B503483A
:100960000EF03EF980F00100C0B208BDCCF70000E7
:1009700073B504460E4DAE684221F3682846984789
:10098000002802DA022002B070BD0D2133696A46E8
:10099000284698470028F5DB0099064A019B93FBFF
:1009A000F2F30A2201FB023323600020EBE700BFD1
:1009B000CCF70000A086010008B503480EF010F93E
:1009C00080F00100C0B208BDCCF7000073B504464A
:1009D0000A4DAE684221F36828469847002802DA9B
:1009E000022002B070BD102133696A46284698473C
:1009F0000028F5DB009B23600020F2E7CCF7000025
:100A000008B503480EF0ECF880F00100C0B208BD54
:100A10008CF7000070B588B005466846FFF7A8FF60
:100A200010BB01A8FFF7D2FFF0B9009B104C0A21C0
:100A300093FBF1F201FB12330292039304AA019B90
:100A4000049302A9204607F08FFD68B9A6684221E9
:100A5000F3682046984738B91C21336906AA204616
:100A6000984708B9069B2B60002008B070BD00BFF6
:100A70008CF70000F0B54FF0FF3385B0CDE90133BE
:100A800002241C4F03938DF8034001A8FFF7C2FF17
:100A900002A8FFF79BFF03A8FFF76AFF0DF1030011
:100AA000FFF744FFDDE90212019B9DF8030000F00F
:100AB00023F83B68019A9A4219DC9DF80330012B18
:100AC00015D002341E2CA8BF1E244EF660256543A7
:100AD0004FF4004640F2E73000214FF47A720023D1
:100AE000E5FB0601FFF74CFB0EF02FFBCDE70224E0
:100AF000EBE700BF38FB000030B5174C451E6171B5
:100B0000227268424FEA22214FEA23626841A272B0
:100B1000124DE0701A14E2721A12E17122736373BB
:100B20000FCD89B003AC0FC42B68236000230C49A0
:100B30000093012203A801F0A5FF10B1032009B022
:100B400030BD00214FF480400EF0FFFA02F0A8F80B
:100B50000028F4D0F2E700BFF407002010FB0000EB
:100B60003CFB0000014B1B68184700BFA806002093
:100B7000014B1860704700BFA806002030B585B053
:100B800004460D461022002168460EF065FC022343
:100B90008DF802302A46044B0193214668460BF03B
:100BA000EFFD05B030BD00BF650B000080B5054608
:100BB0000E46174698460BF059FA03460EF0C8FC4D
:100BC000DFF81890044649F800304246304639466E
:100BD000A84754F8090000F0C5FB00BF080000005A
:100BE0002DE9F047058B04462807904611D40229C9
:100BF00005F0070540F0CC8020460CF0E0F978B114
:100C00000138218B042811D8DFE800F0C2106D856F
:100C1000950001290CBF45F0100545F020052583FE
:100C200088F31188BFF36F8FBDE8F08701F0070AE2
:100C3000AA4500F0A5800027B9463E46A368002BD0
:100C400000F0BC8041F00801218388F31188BFF3D4
:100C50006F8FA168002900F0BA800D68002900F0AC
:100C6000B680D1F80480334652462046C047002D56
:100C700076D02B6829461D46F0E701F007035A1F7E
:100C8000012A1BD8002221F00701062B276889B210
:100C9000C4E9002209D13B4603E0628B0132628342
:100CA0001B68002BF9D141F00201218320460CF092
:100CB00086F900287AD041F0200176E0042B0AD191
:100CC00021F0070189B2218320460CF078F910B198
:100CD00041F020012183218B01F0070AAA454FD062
:100CE0000027B946AAE7236921F0070141F0060170
:100CF000062DD3F8009021832DD1B9F1000F3FD0FC
:100D000041F00801218388F31188BFF36F8F3A49BE
:100D10002046C84729E021F00701236941F004017A
:100D200089B2042DD3F804902183E6D000273E46F3
:100D30004FF0040A82E721F00701236941F0050121
:100D400089B2052DD3F808902183D6D000273E46DE
:100D50004FF0050A72E700273E464FF0060A6DE79E
:100D60002B4687E7B9F1000FD1D1EFF3118820238B
:100D700083F31288BFF36F8F238B23F00803238341
:100D8000258BEA062ED525F01003238305F00705F1
:100D90006669218B002EBFF670AF00232768C4E977
:100DA000003321F0070141F001012183218B01F083
:100DB000070AAA454FF000097FF440AF002F9CD0EE
:100DC00041F00801218388F31188BFF36F8F002F52
:100DD000C8D03D6839463346524620460CF01BF9D0
:100DE0002F46F4E7AB067FF51BAF25F020032383E6
:100DF00005F0070500E700BF43D00000014B03608A
:100E00000020704744FB000008B50348034A002156
:100E1000121A0CF073FA08BDD80800208C1A0020B2
:100E20000748084A084908B5121A0CF069FA074839
:100E3000074A0849BDE80840121A0CF061BA00BF21
:100E4000C0040020D8080020CC060100B80400200F
:100E5000C0040020C406010038B505460C4699B10F
:100E6000D1E901230F4809680CF074F8D4E9042390
:100E7000E1680D480CF06EF8E1690C480CF06AF876
:100E8000A1690B480CF066F8012D05D1EFF305813F
:100E9000084810390CF05EF821462846BDE8384075
:100EA0000AF06CB97AFF0000AAFF0000DAFF000028
:100EB000EAFF00001900010030BFFFF7FDBF00BFCF
:100EC0002DE9F0410B4EDFF8308006EB0807CC1B14
:100ED00005463246094920460EF096FAA0194246C8
:100EE0000021083C0EF0B8FA6C6707F10800BDE875
:100EF000F08100BF000000000400000010FB0000B3
:100F0000054B5A699B689A421FBF044A536843F0D5
:100F100080535360704700BF181A002000ED00E0B6
:100F20002DE9F843324D80463248894617460CF089
:100F300011F8AB6ADE0622D52F480CF00BF811240D
:100F4000AB6A1D0703D52D480CF004F81224284D78
:100F5000AB6A980715D52A480BF0FCFF6E6BAB6A9D
:100F6000190642D5274831460BF0F4FFB9F1000FBE
:100F700003D0AB6A23F08003AB62132403E0102498
:100F8000DEE76FF015061A4DAB6ADA0703D51E4887
:100F90000BF0E0FF1424AB6A9B0603D51B480BF053
:100FA000D9FF1524124B9A6AD50602D49A6A900783
:100FB0000AD55B68190507D54146304600F0B8FAF6
:100FC00010B180F309880224094B9A6A920642BF45
:100FD0005A6A22F400525A629A6A42F0FF029A62F6
:100FE00000233B702046BDE8F8836FF01506C4E788
:100FF00000ED00E02D000100440001007800010038
:101000008C000100A5000100BC000100DC00010013
:1010100010B51D4C1D480BF09DFFA36A990130D5FA
:101020001B480BF097FF1E20A36ADA0103D519486D
:101030000BF090FF1F20144CA36A1B0303D5164826
:101040000BF088FF2120A36A590303D513480BF046
:1010500081FF22200C4CA36A9A0303D510480BF0A1
:1010600079FF2320A36ADB0303D50E480BF072FF40
:101070002420054A936A6FEA03436FEA134393629D
:1010800010BD1D20D0E700BF00ED00E00C01010005
:101090002501010039010100540101007301010023
:1010A00099010100B401010070B5244C06462448A2
:1010B0000D460BF04FFFA36AD90435D521480BF03C
:1010C00049FF1720A36A1A0503D51F480BF042FFFA
:1010D00018201A4CA36A9B050FD51C480BF03AFF49
:1010E000A16BA36A180407D519480BF033FF1EB192
:1010F000A36A23F40043A3621920104CA36A590584
:1011000003D514480BF026FF1A20A36ADA050DD583
:1011100011480BF01FFF1B20084A936A43F47F43DA
:10112000936200232B7070BD1620CBE7A36A9B044B
:10113000F2D50A480BF00EFF1C20EDE700ED00E0B1
:10114000E0010100F701010078000100090201003F
:10115000230201003902010055020100DC000100F8
:101160002DE9F0415B4B5F688AB00446C7F308067F
:10117000002585F31188BFF36F8F02F07F43B3F131
:101180007F4F06D102F00C03082B13D152480BF00D
:10119000E1FE00252C464FF00008F31E8DF8078075
:1011A000092B00F28680DFE803F00A7A7E768484D9
:1011B0008484848210074CBF0C460125EBE7474826
:1011C000444E0BF0C7FE8DF80780F36A9A0704D5EA
:1011D00043480BF0BFFE002330E0F36A002B01DA36
:1011E0004048F6E7F36A5B00F5D53F480BF0B2FEE6
:1011F0007369A26943F480737361BFF34F8FBFF3C8
:101200006F8F736932F8022C23F480737361BFF31C
:101210004F8FBFF36F8F4DF602739A4209D0B36AB6
:10122000DBB253B30DF1070201212046FFF778FE30
:1012300033E021682D480BF08DFE23689DF80720D0
:10124000C2B902AE04F1200720686168324603C2C9
:101250000834BC421646F7D1099AB5B3C2F3080167
:1012600021B96FEA52226FEA4222099202A9184676
:10127000FFF7F2FD0AB0BDE8F081B36A13F47F4FC7
:1012800005D00DF107010120FFF70EFF05E0B36A5D
:10129000B3F5803F9FD3FFF7BBFE0346CEE70DF1CA
:1012A00007020021C1E70DF107010020ECE710481B
:1012B0008FE7104B1049114817F4F87FA6F1100280
:1012C00018BF19460BF046FE85E722F4FF7222F0A4
:1012D0000102CAE700ED00E09C020100C802010023
:1012E000E0020100020301001103010031030100CB
:1012F0004E030100830201006E020100730301002E
:10130000044B5A6942F010025A615A6922F00802ED
:101310005A61704700ED00E0EFF30880EFF30981B8
:1013200001B57246FFF71CFF01BD00BF0B4880F3FB
:10133000088807F0B1FF202080F3118808484FF497
:101340000461401880F30988EFF3148002210843F8
:1013500080F31488BFF36F8F00F0B2F840330020A1
:1013600080250020084B9B6883420BD1EFF3058357
:1013700043B1064B5A6842F080525A605A6A22F4CE
:1013800000425A620AF078BE181A002000ED00E010
:1013900014498A684FF030001044EFF3098C80E85C
:1013A000F01F202080F31288BFF36F8F0E4F4FF095
:1013B00000664A698A603E60506F0C4C2060906FF6
:1013C0000023936780F3118804B5104600F014F9E8
:1013D000BDE8044002F1300090E8F01F8CF309886A
:1013E00070470000181A002004ED00E0100D0020E6
:1013F0001EF0040F0CBFEFF30880EFF30980816942
:1014000011F8021C0229FFD001B572460BF07AFFD9
:1014100001BD00BF40B2002807DB044A4109012397
:1014200000F01F00834042F82130704700E100E0E7
:1014300040B200280CDB4309064900F01F002033AE
:101440000122824041F82320BFF34F8FBFF36F8FFB
:10145000704700BF00E100E0054B420900F01F00AB
:1014600053F82220012303FA00F01040704700BF18
:1014700000E100E040B20028A8BF00F1604001F1A7
:101480000101B8BF064B4FEA4111ACBF00F5614006
:1014900000F00F00C9B2B4BF195480F800137047B0
:1014A00014ED00E0044B054A23F07F039360BFF383
:1014B0004F8FBFF36F8F70470000000000ED00E01A
:1014C00008B5FFF7EFFF0B4AD2F8883023F470031A
:1014D000C2F88830EFF3148323F0040383F31488F5
:1014E000BFF36F8FFFF790FCFFF79AFC00F05AF8FC
:1014F00009F00CFF00ED00E042F8203C009B42F8B0
:101500001C3C0A49019B42F8183C029B42F8143CDF
:1015100021F001014FF0807342F8043C42F8081CAE
:101520000023203A02658367704700BFAD0B0000BF
:10153000094A0346906870B113F1160F406E05D04A
:10154000A0F140029A4205D8834203D2814228BFCB
:101550000020704700207047181A002008B5154673
:101560000B4A0C4B9060426F1A600E4600F044F834
:101570002C4686F309880020034B9847204600211B
:1015800000220023014C204729D30000AD0B0000AE
:10159000181A0020100D0020014B10221A6170470C
:1015A00000ED00E0044800232021C2180133272B5E
:1015B00082F80013F9D1704700E100E008B5EFF3BD
:1015C0000583064A103B02EBC30152F83300496819
:1015D0008847BDE80840FFF793BC00BF4CF8000007
:1015E000024B034A0348012100F076B800000120B5
:1015F0000000002044FB0000426E054B403A1A6098
:10160000044A4021C3E901121846012100F06EB8D6
:10161000140D002000000B15084AC2F898000B6852
:1016200023F01F03034343F01003C2F89C308B6880
:1016300043F00103C2F8A030704700BF00ED00E0A6
:101640002DE9F043DFF8608085B00E461F46044662
:101650004FF00009B14523DA6068D8B13FB1411EAF
:1016600008421BD11F2819D92368194216D12368B3
:1016700001930BF07CFEA36803430393D8F89050CA
:10168000C5F30725D0B2013DA84207D801A9FFF74D
:10169000C3FF421C09F101090C34DBE76FF01502AE
:1016A000104605B0BDE8F08300ED00E0044B0522D4
:1016B000C3F89420BFF34F8FBFF36F8F704700BF05
:1016C00000ED00E0BFF35F8F024B0022C3F89420CF
:1016D000704700BF00ED00E010B5034C01232278F5
:1016E000FFF7AEFF207010BD581A002008B50B4A56
:1016F00000231278FFF7A4FF10F1160F07D0084A55
:101700000021D2F89030C3F30723984200DB08BDD4
:10171000C2F89800C2F8A0100130F2E7581A002071
:1017200000ED00E02DE9F043534B544CD3F89030DA
:101730002568C3F307239D4285B000F29A80FFF726
:10174000C1FF00200C2685421AD14D4C4D4F25700B
:101750006846FFF753FBDFF82081DFF82C9106463F
:101760000025AE4213D1237843490020D1F89020C0
:10177000C2F30722934276DBFFF798FF002042E096
:10178000616806FB0011FFF747FF0130DBE70098B7
:1017900000EB05114FEA051CCB683B40B3F5000F89
:1017A00048D00AD8B3F5001F30D0B3F5800F36D03B
:1017B000B3F5801F10D00135D3E7B3F1807F42D05D
:1017C000B3F1007FF7D150F80C3088684A680BF00D
:1017D000CEFD40F4802009E050F80C3088684A685B
:1017E0000BF0C5FD40F0885040F43020CDE90123D6
:1017F0000390D8F890302078C3F30723013B984238
:101800002AD96FF0150005B0BDE8F08350F80C3010
:1018100088684A680BF0ABFD40EA0900E6E750F83B
:101820000C3088684A680BF0A2FD40F0C06040F4BC
:101830000030DBE750F80C3088684A680BF097FD01
:1018400040F08270D2E750F80C3088684A680BF09C
:101850008EFD40F08870C9E701A9FFF7DDFE23780F
:1018600001332370A7E7C1F89830C1F8A000013315
:101870007CE74FF0FF30C6E700ED00E050FB0000D2
:10188000581A00200000F0FF0000081108B5024BB4
:101890001B689847002008BD200D0020034B044A18
:1018A0001860937843F0020393707047200D002076
:1018B000AC06002008B50649064821F00701C1F131
:1018C000005202F580320BF006FB002008BD00BF7D
:1018D000F73D0020240D002070B54169867A0B4D3C
:1018E000044659B1437ADB0706D42C2303FB065385
:1018F0005B6A1B689B689847002363612C20214624
:1019000006FB0050BDE870400DF091BA2808002099
:10191000024B2C2202FB0030704700BF2808002039
:10192000827A064B2C2101FB02339A6A1B7F1B3300
:10193000801A23F00303B0FBF3F07047280800205F
:1019400038B5074B827A2C2404FB02335B6AD3E957
:1019500001240C601568FFF7E3FF04FB005038BD5D
:10196000280800202DE9F04385B00546684603911C
:1019700090461C460DF071FCDDE90067EFF311891C
:10198000202383F31288BFF36F8F6B8B002B41D022
:101990002A8B9A4225D900220023284609F0F6FD19
:1019A0000446F0B189F31188BFF36F8F039B002BBE
:1019B00041D032463B4668460DF074FCA27A264B75
:1019C0002C2101FB023320465B6A1B6803A91D68BA
:1019D000DDE90023A847606170BB2046FFF77CFF6C
:1019E00024E0698B4B1E6B8389F31188BFF36F8FE3
:1019F0002B7F2A8BAC6A1B3323F00303521A02FBA2
:101A00000344154B154AEB1A9B105343A3722B7FCB
:101A1000E372CBE789F31188BFF36F8F2346424609
:101A2000284609F0B3FD04460028BFD10024204613
:101A300005B0BDE8F0836361012300252381039B8A
:101A40006382E27A6560294604F118000DF004FD16
:101A500063692582E360EAE728080020A38B2EBA99
:101A600070B50D4C2C2500B970BD037A4668002B6B
:101A7000FAD0013BDBB20372002BF5D1C3604360A7
:101A8000837A05FB03431B6A13B198473046EAE7A4
:101A9000FFF722FFFAE700BF28080020024B0122CF
:101AA000C3F840250020704700E0014020B1034BFF
:101AB000800143F001031847704700BF30FB00006E
:101AC00010B50E4C20460DF08BF898B12269A16834
:101AD000136823F4806313600B684FF420220A21FB
:101AE00020469847002804DB212000210DF02DFB23
:101AF000002010BD6FF01200FBE700BF6CF7000084
:101B000008B50BF0E4FC0AF0BDF9044B1B680BB1FF
:101B10000A209847BDE808400AF0C8B9300D0020F7
:101B200038B5044608480BF03DFC054648B1631E35
:101B3000DBB21F2B96BF054A0021D15C0C300BF0A5
:101B400083FC284638BD00BF80080020A90301009F
:101B50000E38012810B50AD809480BF023FC0446BA
:101B600018B104210C300BF06FFC204610BD09B1F8
:101B70000448F2E7BDE810400220FFF7D1BF00BFE4
:101B8000AC0800202808002010B5012104460C30C4
:101B90000BF07BFC2146034A0078BDE8104000238F
:101BA0000BF0C0BCE8FB000010B5012104460C306E
:101BB0000BF06BFC2146034A0078BDE8104000237F
:101BC0000BF0B0BCE8FB000010B5012104460C305E
:101BD0000BF05BFC2146034A0078BDE8104000236F
:101BE0000BF0A0BCD0FB00002DE9F047884616465C
:101BF0008246002872D0BFF35B8FDFF8E4900023A9
:101C000059E8004F49E80032002AF9D1BFF35B8F51
:101C1000002C63D02046FFF783FE324D0C2303FBDC
:101C2000005027464388534511D0BFF35B8F59E8D6
:101C3000003F49E80072002AF9D1BFF35B8F002B07
:101C40004CD01F463846BDE8F047FFF709BFA64213
:101C500008D020460BF0A1FB328AF16804F10C0099
:101C60000BF0E9FB2046FFF75BFE0C2606FB00505D
:101C70004368ABB1B8F1000F12D12046FFF750FE18
:101C800006FB005001214268D2E90003127A03F0FA
:101C90001F06B1405B09DAB100EB83000BF02FFCAB
:101CA0002046FFF73DFE0C2606FB00508368002B04
:101CB000C8D02046FFF734FE704305F80080204668
:101CC000FFF72EFE06FB0055A86809F091FCB9E766
:101CD000C94300EB83000BF03CFCE1E7BDE8F08773
:101CE000D0050020340D0020094BBFF35B8F1A682C
:101CF000BFF35B8F02F00B02BFF35B8F53E8001F53
:101D000043E800200028F9D1BFF35B8F704700BF84
:101D1000940500202DE9F8430C460AF0B3F8E26878
:101D2000218A1378042B6DD1022908D82046FFF7A9
:101D300097FE00240AF0BAF82046BDE8F8835378ED
:101D40003E2B08D10329F1D0D378012B01D00A2BE7
:101D500049D1032705E0052BFBD00E3B012B42D8D0
:101D6000012704F10C0630460BF09FFB01210546CC
:101D70003046B4F810900BF080FB022130460BF097
:101D800084FB03783E2B804607D1E3681B78012B48
:101D900001D00A2B06D1032614E0052BFBD00E3B05
:101DA000012B29D91A4A1B491B4841F2F3030BF0B6
:101DB000DEF8002383F31188BFF36F8F03231846E7
:101DC00002DF0226154A98F80000032321460BF093
:101DD000A9FBB20712D56369A4F8109013FA85F530
:101DE000E560BB07A5D521460D480BF0DFFA0D498C
:101DF0000D480DF0BFF89CE70126E3E72046FFF70A
:101E00002FFEEEE72046FFF72BFE6FF0150491E75B
:101E1000C9030100FD03010016040100B8FB000026
:101E2000D4050020CC060020D808002038B51C4876
:101E30000BF0D1FA044688B300F10C0528460BF0EC
:101E40002CFB04281DD1284602210BF01EFB037831
:101E50000E3B012B05460ED8124A1349134840F693
:101E600063430BF084F8002383F31188BFF36F8F73
:101E70000323184602DF0E4A2878032321460BF07D
:101E800051FB2046FFF7ECFD0A4BD3F814312BB180
:101E9000BDE83840084909480DF06CB838BD00BFAE
:101EA000D4050020C9030100330401001604010019
:101EB000D0FB0000C0040020CC060020D808002081
:101EC00010B5C1E900239DF808300B720C46FFF7EE
:101ED00027FD034B0C2202FB00335C6010BD00BFEA
:101EE000340D0020F8B502460B4610480BF05AFAA4
:101EF0000446C0B104210C300BF093FA2046FFF7E2
:101F00000FFD0B4D0C2707FB005000264680204696
:101F1000FFF706FD07FB005086602046FFF700FD37
:101F200007FB00556E602046F8BD00BF5408002036
:101F3000340D0020034B0146D3F8340182689268C7
:101F4000104700BFC0040020014804210BF0D7BA9D
:101F500094050020014809F003BD00BFBC06002025
:101F600070B505460C4659B94FF0FF304FF0FF31C0
:101F7000FFF7B8FF044618B96FF06805284670BD32
:101F80002046FFF7CDFC164B0C2202FB0033A618AF
:101F900030465D800BF089FA03280BD903213046C7
:101FA0000BF05AFA0580238A033B837001213046E7
:101FB0000BF05AFA40F635439D4208D12046FFF710
:101FC000B9FF054648B12046FFF74AFDD6E7054868
:101FD00021460CF021FFFFF7BDFF0025CEE700BF33
:101FE000340D0020DC05002038B502460B46244D98
:101FF000D5F81C1109B9002038BD05F1F80009F029
:1020000031FB0028F7D10022002305F58E7009F07E
:10201000BDFA044668B91B4A1B491C4840F6734385
:102020000AF0A5FF84F31188BFF36F8F03231846CE
:1020300002DFD5F8100120B1FFF712FD0023C5F82B
:10204000103120460BF0DDF9C5F810012046FFF7EE
:1020500071FF98B10E4809F0CBFA2046FFF760FCFB
:102060000C4B0C2202FB00301F2140882246FFF758
:10207000BBFD2046FFF7F4FCFFF76CFF0120BBE738
:10208000C0040020C903010061040100160401001E
:10209000B8050020340D00202DE9F04F064687B02A
:1020A00017460C4669B94FF0FF304FF0FF31FFF78C
:1020B00019FF044660B96FF06805284607B0BDE80F
:1020C000F08F887AFFF724FC454B834240F08280F2
:1020D0000122002168460CF0B8FE2046FFF720FCE4
:1020E000DFF800A10C2303FB00A0C0F808D02046B5
:1020F0000BF087F901463046FFF732FF054618B16D
:102100002046FFF7ADFCD8E70DF022FA364B1A58FF
:10211000364B9A4220D1DFF8D8B036480CF091FE09
:10212000002181464FF4A020FFF75EFF804688B96A
:10213000314A32484FF4F97359460AF018FF3048D3
:1021400031460AF014FF88F31188BFF36F8F032321
:10215000184602DF4C45E0D14FF4A0220023684628
:1021600009F080FA804698B14FF4FC73224A254961
:1021700022480AF0FCFE2448424631460AF0F7FEA7
:10218000002383F31188BFF36F8F0323184602DF08
:102190002046FFF7C5FB0C2358431AF80060AEB188
:1021A0002046093EFFF75CFC092E0CD8DFE806F05C
:1021B000150B0B08050B0B0B0B126FF00B057CE7D7
:1021C0006FF00C0579E76FF0040576E7002F97D0E4
:1021D0003C6072E76FF015056FE76FF06E056CE716
:1021E00054080020340D002008000000D00B00200F
:1021F00065040100DC050020C9030100160401008C
:102200006D0401008D04010096040100F7B5002261
:10221000114640F60340FFF73FFF0446002853D124
:10222000FFF762FD214601AA41F20300FFF734FFE8
:102230000446002848D1019A854DD168D1F80100A3
:10224000D1F8051005F1780303C31046FFF708FC29
:10225000214601AA41F20100FFF71EFF044698BB88
:102260000198C3685A7885F870205A88A5F87220BA
:102270001A7985F87120B3F80720A5F87420B3F80F
:102280000530A5F87630FFF7EBFB214601AA41F2B5
:102290000200FFF701FF0446B0B9019FFA6805F19B
:1022A0008006531C413218685968344603C4083309
:1022B00093422646F7D13846FFF7D2FB95F87C309B
:1022C000580604D46FF01204204603B0F0BD01AAF2
:1022D000002142F20300FFF7DFFE04460028F3D19D
:1022E000019A5C4BD168D1F80100D1F8051003C305
:1022F0001046FFF7B5FB1F23A5F8E83095F87C30B2
:10230000990619D44FF0FF304FF0FF31FFF7EAFD87
:102310000646002800F0998002210C300BF085F869
:102320000123447003702246314640F66D40FFF7AA
:10233000B3FE04460028C7D195F89C301A0712D581
:1023400001AA002142F21C00FFF7A6FE0446002865
:10235000BAD10198C368D3F80120D3F80530C5E994
:102360003823FFF77DFB4FF0FF304FF0FF31FFF7D1
:10237000B9FD0446002868D008210C300BF055F850
:1023800002270022077042708270C270027142718F
:102390008271C271214642F20100FFF77DFE0446C0
:1023A000002891D14FF0FF304FF0FF31FFF79AFD39
:1023B0000646002849D008210C300BF036F880235F
:1023C0004370202304708470047144718471C77059
:1023D000C3712246314640F60140FFF75DFE0446D8
:1023E00000287FF471AF014601AA4FF60140FFF7C4
:1023F00053FE044620BB0198FFF732FB214601AA99
:102400004FF60240FFF748FE0446C8B90198C3687A
:10241000B3F80130A5F8C130FFF722FB95F8C130C1
:102420005B070DD501AA21464FF60340FFF734FEA6
:1024300030B90198C3685B7885F8C030FFF710FBAE
:1024400003B0BDE8F04000F097BA6FF068043BE7D6
:10245000C00400209805002073B5264D0646D5F827
:1024600034010CF0BDFB00283CD06FF0020105F1F7
:10247000D4000BF06EF801210BF041F810EA0104D2
:1024800033D11D4B1E600A4605F1F8000CF0DDFC4F
:1024900005F58E700CF082FC18480CF07BFD184995
:1024A000164800946FF007034FF4966209F05EFA45
:1024B000144912480CF099FDD5F83401124983688B
:1024C0001B689847044628B93EB9FFF79FFE78B9C4
:1024D000FFF73AFD204602B070BD05F1C40009F0D7
:1024E0003FFAF7E76FF01204F4E76FF07704F1E7D3
:1024F0000446EFE7C0040020400D0020D80800206B
:10250000C01A0020DB040100151D000010B5FFF704
:102510007DFE044608B9FFF717FD044B1B681BB18D
:102520002046BDE81040184710BD00BF400D0020F8
:1025300038B5032104460C300AF0A7FFE36805789C
:10254000B0F80100197840F6354398420AD0224687
:10255000FFF74AFB35B1044809F04AF8BDE83840B6
:10256000FFF7F8BC38BD00BFB805002038B504211E
:1025700004460C300AF089FF4578017840882246ED
:10258000FFF732FB35B1044809F032F8BDE83840B6
:10259000FFF7E0BC38BD00BFB805002070B54FF0B4
:1025A000FF320D464FF0FF3300210646FFF7D0FA09
:1025B000044660B90A4A0B490B481A230AF0D7FCB3
:1025C00084F31188BFF36F8F0323184602DF0221C3
:1025D00004F10C000AF029FF06704570204670BD1A
:1025E000E40401006104010016040100F8B50A4D7D
:1025F000EF7906460024E3B29F4202D86FF0010053
:1026000007E0294630460AF0DFFF0735631C08B1B2
:102610002046F8BD1C46EEE7C004002070B5144EFD
:102620000622314604460CF01FFFE0B14FF0FF30A8
:102630004FF0FF31FFF756FC0546B0B106222146A8
:102640000C300AF0F8FE0022294642F20500FFF79E
:1026500023FD48B93346226843F86929A288B2802D
:10266000012283F86820002070BD6FF06800FBE74E
:102670002905002037B504460D4689B1184928467A
:102680000AF0A2FF60B9174A2968C4EBC404A31872
:102690001151AA889A80AA799A71002003B030BD9E
:1026A00068460AF006FF0028F8D16846FFF79EFF4B
:1026B0000028F5DA0B4A00989DF80610C4EBC40414
:1026C000A3181051BDF8040098809971002DE4D032
:1026D00012592A609A88AA809B79AB71DDE700BF06
:1026E00096030100C004002070B5044611B16FF0DC
:1026F000150070BD80B11C490AF066FF60B9204624
:10270000FFF774FF002829DA2378012BEFD1A37992
:1027100003F0C003C02BEAD1144DEB79012B20D07C
:10272000BFF35B8FD5F8D430BFF35B8FDB0707D4E3
:10273000002CDCD00C4920460AF046FF0028D6D1F8
:10274000EE792146731C3046EB71FFF793FF08B911
:102750003046CEE7EB79013BEB71CAE76FF07700CB
:10276000C7E76FF00B00C4E796030100C004002028
:102770002DE9F3410446D8B101AA002141F2090034
:10278000FFF78AFC054698B9019E1249D6F80C80DD
:1027900008F10107062238460CF066FE28B10E4902
:1027A000062238460CF060FE30B93046FFF758F983
:1027B000002002B0BDE8F081D8F80130C4F8013043
:1027C000BB88A4F8053030462570FFF749F9012091
:1027D000EFE700BFA30301009D03010007B56846B2
:1027E000FFF7C6FF044BD87118B169460020FFF708
:1027F00041FF03B05DF804FBC0040020F0B5294D93
:10280000EE7989B0002E46D195F8C230DB0722D58B
:102810006A4631464FF60940FFF73EFCD8B9DDF86D
:1028200000C0DCF80C406378012B1E4628BF01264F
:1028300073B1A31C02AA123418685968174603C75B
:102840000833A3423A46F7D1186838609B88BB80AA
:102850006046FFF705F9EE71002416260127EB7993
:10286000E0B2834202D8B3B1002012E008AB06FB0D
:102870000033694653F8182C33F8143CCDF8012086
:10288000ADF805308DF80070FFF7F4FE0134002834
:10289000E5D009B0F0BD0021084609B0BDE8F04020
:1028A000FFF722BFC00400202DE9F0410D46174676
:1028B0001C460646002856D0002B54D00A03037845
:1028C00008D56D074FD40AF08FFE002849D10123A7
:1028D00023700CE0A9072CD026480FB1AA0608D413
:1028E000C3EBC302825C012A12D002B9227000201D
:1028F00037E090F8D820510638D5C3EBC302825C8C
:10290000012A05D002B92270237843F00203DFE7E1
:102910004FF00108072111FB0381014430460AF002
:102920005BFEF0B984F80080002FE0D0AB06DED566
:10293000EAE76A0711D50F49C3EBC3028E5C012E8B
:1029400008D1072212FB036319440AF045FE40B97F
:102950002670EBE7002EE9D1FAE70AF045FE0123E5
:102960002370BDE8F0816FF01500FAE76FF0850085
:10297000F7E700BFC004002010B50A4CE3790BB1A3
:10298000002010BDFFF72AFF0028FAD1E379002BC1
:10299000F6D1FFF733FF0028F3D1601CBDE81040EB
:1029A000FFF73CBEC0040020F8B54568690506463F
:1029B00035D4046914B115F0030330D0194F3078C1
:1029C000FB7983422BD9C0EBC0001749072238445A
:1029D0000CF04AFDA8B115F0030306D197F870205A
:1029E000082A02D8B2689F2A19D915F0300F09D0E9
:1029F000ACB1EA060AD405F46035B5F5603018BF0D
:102A00000120F8BDEB0601D4002CF4D1D6E9022355
:102A10009A4204D81F2A02D9B3F5804FEBD900207F
:102A2000EFE700BFC004002096030100F7B5CDE931
:102A30000001694642F208009DF8207016461D46C6
:102A40000AF0FCFD044668B97FB9BFF35B8F0C4BFD
:102A500053E8001F41F0040143E80012002AF7D1B7
:102A6000BFF35B8F204603B0F0BD694642F2090018
:102A7000CDE900650AF0E2FD0028E6D00446F1E762
:102A8000E80400202DE9F04F7F4ED0F810B0BFF3DE
:102A90005B8F9A463368BFF35B8FBBF100040F4630
:102AA00018BF0124590787B00546914640F1CC80F4
:102AB000FFF77AFF60B96FF015043846002340F243
:102AC0000111994540F0C980204607B0BDE8F08F5C
:102AD00028460AF0A0FD80460028ECD0BFF35B8FAB
:102AE00056F8AC2CBFF35B8FC2F30023D20500F184
:102AF000AE80CDE90333CDF81330AB686868ADF82C
:102B00000830EB68ADF80A300AF089FD8DF8150041
:102B1000BFF35B8F56E8003F23F4807346E8003232
:102B2000002AF7D1BFF35B8F2A7806F8BC2C06F891
:102B3000652C696822460DF10D03A6F1BC00FFF774
:102B4000B3FE04460028B8D1A6F1B303BBF1000FD1
:102B500011D02A69116846F8B31C9188998092793E
:102B60009A716B689C074BD1990502D4BAF1000F9A
:102B70005AD002230BE0454A116846F8B31C9188ED
:102B8000927999809A716B689807EDD05B468DF8C1
:102B90000C304FF0FF304FF0FF31FFF7A3F9044640
:102BA000002857D00F2202A90C300AF044FC21461D
:102BB000002242F20600FFF76FFA044600287FF475
:102BC0007CAFBBF1000F33D0314801210AF0ABFDDF
:102BD000044600287FF471AF6A682E4812F00302A1
:102BE00018BF012209210AF083FD42460A210AF09A
:102BF0007FFD6A680C21C2F380020AF079FD5CE770
:102C000013F0100F0CBF012304238DF80C302B6937
:102C10001A68CDF80E209A88ADF812209B798DF8AD
:102C200014304FF00008B4E703238DF80C30F8E7B8
:102C3000109BCDF80080524649463846FFF7F6FE15
:102C400004460028C0D038E76FF00A0435E76FF07B
:102C5000770432E76FF068042FE702888A4204D1D4
:102C6000426812B11278D20702D40133083028E743
:102C700009490A480CF094F94FF4702200230748E0
:102C800008F0E2FE20E700BF940500209603010053
:102C9000D8040020E804002079D70000F0040020C8
:102CA00010B50A4C20460AF064FDBFF35B8F236920
:102CB000BFF35B8FC3F30020DB0505D52046002161
:102CC000BDE810400AF02FBD10BD00BFD8040020A1
:102CD00000F1070C2CF0030C10B4541E1860A4B2C1
:102CE000ACF80020023A93B201FB04F24FF0000C62
:102CF00040F802C074B103FB011403FB01F220444D
:102D0000121B4FF6FF7C013B9BB263458050A0EB4A
:102D10000100F8D110BC70470346006810B102688A
:102D20000AB91A60704700F1070C2CF0030CD11D92
:102D3000BCF800C021F003010CF1FF3CA1F800C079
:102D4000EFE700BF0B687BB1073323F003031A885A
:102D5000013292B20346D1F800C043F807CB23F00A
:102D600003031A80086070470122F3E7531E1144E1
:102D70009BB242B1DB430138CA1811F8013D00F89B
:102D8000013F9142F9D17047014402E010F8013B44
:102D90001BB98842FAD1002070470120704700BF5C
:102DA00010600860704700BFD2F800C0CCF8000087
:102DB000D2F800C0CCF8041010607047884203D0ED
:102DC0001AB1436813607047002070470B68834254
:102DD00009D02AB1586810601A680A60184670470E
:102DE000002BF9D1FAE70023F8E700BF2DE9F04105
:102DF000DFF830800C4E0C2706F130044546221DCA
:102E0000214628460C3CFFF7CBFFA642A5F108055A
:102E1000F5D1043F3B1DA8F12008A6F13006EBD107
:102E2000BDE8F081C00D00204C0E0020F8B506462C
:102E30001C460D4602B322786378D21A12F00302C0
:102E40003AD1274F71004FEA450C3144AC44890018
:102E500001EB0C1101330431DBB27A186068237086
:102E60002146FFF7A1FF1F4B0122294630465A5544
:102E700003F0E4FF0020F8BD03F0CAFF0028DAD019
:102E80002946304603F0B6FF0028D4D005EB4502B2
:102E900006EB4601124F6378120102EB81023A44BD
:102EA0007100907AD27A90424FEA450C0CD020788B
:102EB000C01A10F00302C8D0012A03D00133DBB2DC
:102EC0002370D0E71046F8BD2278D21A920702D0BC
:102ED0000233DBB22370D4E902039847CAE700BF8C
:102EE000C80D0020440D00202DE9F04FDFF864915B
:102EF00019F8003089B0002B5AD0DFF85CA13C22D1
:102F000004234FF0000B00EB400712FB00330324B7
:102F1000CDE904BB09F800B00AEB0717039302944C
:102F20008346B8460023B96A58F8240F079307AAC6
:102F3000FFF744FF044607AAB4B1079D2E786978CD
:102F4000761A06F00306012E35D02B78591A01F0B7
:102F500003010129DBB23DD1D7E90901FFF72EFFBB
:102F6000044607AA002CE8D197F82E3097F82F20B6
:102F70009A4203D087F82F300123049397F82C301E
:102F800097F82D209A4203D087F82D30012305931E
:102F9000029B5D1EEBB2FF2B0293A7F10C07C0D181
:102FA000049AD846DDF814B012B1BBF1000F45D039
:102FB00009B0BDE8F08F01396970079BD3E90203BE
:102FC0009847079D2A786978D3B2521A02F0030213
:102FD000012A21D0B86A019300224146FFF7F6FE8C
:102FE0006C60019B6A786B702B789B1A03F003036B
:102FF000012B08D0D7E9090107AAFFF7DFFE012E50
:10300000044698D10EE0039B6A70294620460AEBDD
:103010000302FFF7C9FEEDE7D7E9090107AAFFF7A9
:10302000CDFE0446029B8BB101235946584609F850
:103030000B3003F003FF09B0BDE8F08F5A4641465C
:10304000404609B0BDE8F04F03F0C8BE002C8BD05D
:10305000EAE700BF440D0020C80D00204B1EDBB284
:1030600071B1411E00EB030C002011F8013F23B1A8
:103070005A1E01301340C0B2FAD16145F5D17047F4
:103080000846704730B5037E0568FF2B14D003EB6C
:1030900043028B4205EB021227D04FF0000C01E0F7
:1030A00099420BD09E4613789468FF2B03EB4302A2
:1030B000A44405EB0212F3D1002030BD714517D0B6
:1030C0000FFA8EFE137890680EEB4E0E4FEA0E1E2E
:1030D000FF2B05F80E3006D003EB430305EB03137B
:1030E0009A6802449A60604430BD9E464FF0000CDE
:1030F00013780376E4E700BFA2EB010C1CF4000F89
:1031000010B4836844690AD12CF07F4C6344A34215
:103110000DD8E41A00234461836010BC7047891AFB
:1031200021F07F418B4208D95B1AA342F1D91B1BC6
:1031300000244461836010BC70470C44E41AE9E742
:103140002DE9F843284DBDF82C7004464FF02C0EA5
:103150000EFB045E084604EB840104EB4104DEF838
:10316000041001EBC00605EB8405F47811F83080FB
:10317000717804F1010C5FFA8CFCE04598BF4FF0C8
:10318000000C61452DD0716804EB44044FEA04192A
:1031900001EB04144FF0040801F809806360089BF8
:1031A000A360099BE3600A9B23610C9BA361119BB5
:1031B00063620D9BE3610E9B23620F9BA362109BD6
:1031C000E36202236270A782A37086F803C0DEE97F
:1031D000083698472B4641460022B047A078BDE804
:1031E000F8830120BDE8F883880E00202DE9F04F18
:1031F0000346407AD3E9004587B0002800F0FE80FE
:10320000421ED2B205EBC2029A468B460392059546
:103210002346039A516856780491BBF1FF0F66D09C
:103220000BEB4B044FEA0418CDF804B013F808B0C8
:1032300003EB041400254FF0FF0C84F800C0DAF80B
:1032400000709AF8182007EB08096245D9F80810B1
:1032500018BF02960ED1CBE0091A06D1B9F81E802C
:10326000BEF81EE0F04500F2B680B85DFF28944637
:103270006DD0024602EB420607EB061E3601DEF871
:1032800008008842E8D9029EC9F80810BCF1FF0F77
:1032900089F8002064D00FFA8CFC0CEB4C0C4FEA40
:1032A0000C1C019807F80C00FF2A06D002EB420222
:1032B00007EB0217BA68521ABA60A278013262703C
:1032C000002DAAD0AA6A4FF000012970A97022B17E
:1032D000E96A019300209047019B6268002A9CD113
:1032E000AA6A2262EA6A6262BBF1FF0F98D1039A6E
:1032F000049F9278994606EB4601701CB2424FEA51
:10330000011CC6B207EB011568D0039B17F80C101F
:103310001878B04208BF00260429ECD16A7802EB85
:10332000420809EB0814012094F801E0A1788E45C9
:103330004FEA081818D04FF0000307F80C30AA6ABB
:10334000A8700AB1E96A9047039B9A78D3E70246CE
:10335000BCF1FF0F029EC9F8081089F800209AD12D
:1033600001988AF818009FE70192AA8ADAF81410E7
:103370004FF6FE7082424B4607D04FF6FF70121A8E
:10338000B2FA82F2520984F82C206A6AA262EA68D0
:1033900062602A690293002363622262AA8A4FF65E
:1033A000FD70824288BF1A46A283AA69A261EA69B7
:1033B000E2602A6A2261AA68A26063616A682046A4
:1033C000FFF79AFEE2784FF0000342F00102E38338
:1033D000E270029B2FE7029E014655E7039905988C
:1033E0004A7081424B46A1F1080207D0039210E7D0
:1033F00007F80820019A8AF818205EE707B0BDE8B0
:10340000F08F00BF2DE9F04F447E01238FB083760B
:10341000002C40F0B880037EFF2B814600F0B28084
:1034200003F0B6F9D9F81420D9F81C3099F81880AF
:10343000D9F800A0801A20F07F45AB4294BF00234A
:103440000123B8F1FF0F0493A3467AD0059408EB4B
:1034500048080AEB08144FEA0818A368AB426FD873
:10346000A0781AF80880ED1A9B4463781B1ADBB227
:10347000012B62D1A26AA3690393002A00F0F280B3
:103480001668002E00F08280002B40F09280049B92
:10349000002B00F00C8104230393137A590700F0EA
:1034A000FB80137A6FF302031372E78BE2786FF3FA
:1034B00000027B1CE27094F82C209BB2E383002A6C
:1034C00073D0A28B9A4270D2A26A002A00F048817F
:1034D000137A03F00703012B67D0012600205168FF
:1034E0005060A36A1A7A60F302021A72A078E76841
:1034F0000138A0700FB36369D9F8142094F803C0A1
:10350000ABEB0303134423F07F40626A23690CF0A2
:10351000010C002E40F0B780B4F81EE0CDE900C3E6
:103520007346B847039BE683002B049B18BF012317
:103530000493E37866F30003E370B8F1FF0F86D1DC
:10354000059C99F80B3099F80A209A4208D101326B
:10355000D2B2022A1ABF14462346002389F80B4030
:1035600009EB83030022C3F80CB0D9F8244089F892
:103570001A204B46012204210320A4460FB0BDE8C7
:10358000F04F604784760FB0BDE8F08F039B002BAF
:1035900066D0049B002B84D1D9F81C305B4580D8C1
:1035A000B8F1FF0F11D1049E98E7A378013BA370F7
:1035B000C3E7049B002B7FF470AFD9F81C309B4508
:1035C000FFF46BAFB8F1FF0F47D0039BE78B079376
:1035D0009C46A38B6668DDF81CE0BB429CBFFB1ACF
:1035E00099B208EB480388BF39460AEB031301FB85
:1035F0000661069199688E452DD3CDE90C70CDF802
:103600002CC0DDF81CC0CDF81C90DDF80C90CDF876
:103610002880CDE9085B8E46A346B0461446986ADA
:103620009A6910B1006800284FD1002A4DD11B784B
:10363000FF2B07D003EB43030AEB031399688E4477
:10364000E645ECD92246DDE90A8C5C46DDE9085BFB
:103650000D98DDF81C90CDF80CC0002A00F0978082
:1036600000263BE7039BA3B1049B002B7FF41DAF17
:10367000D9F81C309B45FFF418AFB8F1FF0FA4D167
:1036800004990E4633E7CDE900C34FF6FF73B84700
:1036900053E7039E00212AE7A08BE18B88423FF687
:1036A00000AF012161F302031372E78BFEE6D9F844
:1036B0001C305B453FF6EFAEB8F1FF0F53D04FF033
:1036C000040CE78BCDF81CC083E7DD8B9F8B5E6815
:1036D000BD422AD2002E41D1002CA8D03046266807
:1036E0002EB1B9F1000F02D1724496423FD2BD42D1
:1036F0009DD3DA789BF8031002F0010601F0010572
:10370000AE4204D84A40D50791D400288FD0224633
:10371000DDE90A8C5C460C9FDDF81C90DDE9085B56
:10372000002A32D1CDF80CC0C0E69EB1E81B80B2B1
:10373000B8F1000F0AD000FB0660401A06998142DA
:103740002CBF00200120002CC9D1D0E74046002C1E
:10375000C5D1CCE7002CC1D12046CAE72846E7E70F
:10376000A078012696E70423049E0393B6E622463A
:10377000DDE90A8C5C46DDE9085BDDF81C90CDF8DC
:103780000CC0002E3FF48DAE87E61668F7E71646AC
:103790001146ACE6837E002B40F042832DE9F04FCA
:1037A000467E8FB08246002E7CD1837AC27A012178
:1037B00041769A424169089100F05F830133DBB2A0
:1037C000022B12BF1A463246334600EB8202837246
:1037D000D268089B0692134423F07F434361012380
:1037E0000C939AF818300B9302F0D2FF9AF8092044
:1037F000DAF800300193531EDAF804500590DBB27A
:10380000002A00F04B8405EBC308FF2304930D96B8
:10381000CDF80CA0D8F804B04FF0000A2F4698F865
:10382000030098F802900FFA89F404EB440409F1BC
:10383000010348454FEA0416DBB20BEB041400F019
:103840000E8198F800209A4208BF002388F80230C1
:103850001BF806206178042A3AD9019801EB41034C
:1038600000EB0315082A4FEA03130293A8786B783C
:1038700022D81B1A13F0FF032CD1062A1CD1039B5C
:10388000DB7E8B424FD00BF806A0A36A84F802A01F
:10389000002BC4D00020E16A984798F8030098F8FC
:1038A0000290C0E7446A0421034601220420A44692
:1038B0000FB0BDE8F04F60470BF806A04FF00103D2
:1038C000A370A36A002BAAD0E16A01209847A6E75B
:1038D0009946A8E7052A1DD162684AB9A2683AB993
:1038E000E2682AB922691AB9626932F07F42E3D0EC
:1038F000012B1AD0039B04215C6A3D460122084635
:10390000A047454588F80290A8F1080300F0AD8073
:1039100098467FE7012B00F05F81062AEAD1039BDE
:10392000DB7E8B42AFD1616878E1DDF80C904846D0
:10393000FFF7A8FBA860D9F81410059B069A5B1A3C
:1039400023F07F431344984240F28081C01A6B6891
:10395000002B52D0A38A002B4FD0013B9AB2A282F7
:10396000D5F804C0EB8B604523D90CF1010907970A
:1039700009911AE06A6ADFF858E2964996448E4542
:1039800084BF02F1E87202F5D4324F46296A94BF2F
:10399000674602F5A572013BC01B521A9BB26045F7
:1039A0006A62EB8340F2D481A28A9A42E2D3079FF3
:1039B00009999A4220D9CDE909710CF10102D5F893
:1039C00020E007926A6ADFF80892824972449144C3
:1039D0008945674606D8A2F1E872A2F5D432079F5E
:1039E000A2F5A57201339BB26A62EB83A28A9A4266
:1039F0003844E7D8DDE90971AA8363680344AB6002
:103A0000A2686B69A86A13446B6128B103681BB193
:103A1000D4E901329B1A4360059A2846FFF76CFBF4
:103A2000E268AB691344AB61226993428CBF9B1A75
:103A30000023AB61A37D1BB1EA7863F30002EA7057
:103A4000E37D13B1013B85F82C30DDE90121049BB6
:103A500053546B786278049201336B7013E73D46E0
:103A60004545A8F108037FF453AF0D9EDDF80CA087
:103A70000C9B9AF81850002B00F07381059B089A54
:103A8000DAF800409B1AFF2D23F07F4700F03983BE
:103A9000DDF8188005964FF00009AB4607950BEB53
:103AA0004B0504EB051301939B6843454FEA05154D
:103AB00000F2CF820198019E81784278C08B521A21
:103AC000DAF81C108B4234BFC91A0021A8EB030896
:103AD000A7EB0307994424BF4FF0FF338AF81B304C
:103AE000CAF81C10B16AD2B2002900F026810B6816
:103AF000B669002B00F00D81002E40F00D81022AE6
:103B000000F0A282019900238B60635D8AF818306F
:103B10000B464968002940F0BE809B6A2BB11B7A96
:103B200003F00703012B00F0978042B1012A00D077
:103B300028B1019A136A13B1516A01209847019B79
:103B4000019A9B7853709AF818B0BBF1FF0FA6D179
:103B5000059E079D0B9B5B4503D1EB1A18BF012304
:103B60000C9350460499FFF741FBDAF80080019668
:103B700000275046027EFF2A00F0938215464FF040
:103B8000FF0900E01D462BB203EB430308EB0316CD
:103B90001B01B46A21463CB194F808C00CF0070C34
:103BA000BCF1010F00F06F8118F80330FF2BA9461C
:103BB000E8D18246019E1046002F40F0ED800B9B1D
:103BC000934240F0E9800C9B002B00F0D580E7E0A9
:103BD0005A2B17FF592B177F062A3FF450AEDDF8FA
:103BE0000C904846FFF74EFAAB78A8606B7099F8D6
:103BF0001B2063789A427FF446AE1BF80630062BF2
:103C00003FF491AE039AFF23D3761BF80630062BC0
:103C10003FF489AE082B3FF486AE0599039B5A69A1
:103C20008B1A1D0209D4069A23F07F43134403998B
:103C3000CA699A4288BFCB6125E6069B521A22F0D8
:103C40007F4293428CBF9B1A0023F0E76A691344BA
:103C50001B1A6B6100207AE6019A9378C2F80880FB
:103C60005370089B0198DAF8141003EB090222F054
:103C70007F42FFF741FA049B63554378019ACDF8E0
:103C800010B00133DBB253709AF818B0BBF1FF0FDC
:103C90007FF405AF5CE7019B9B6A23B11B7A03F0BD
:103CA0000703012BD8D0019BB3F81EC0BCF1000F55
:103CB00052D1B3F81CC06046019BCDE90245D3E95F
:103CC0000863002201F1010E04E00C460138224491
:103CD000441C10D0854C864D33441C19AC42F4D89A
:103CE0007446A3F1E8730138A3F5D4332244441C8D
:103CF000A3F5A573EED10198436290F82C00DDE99D
:103D00000245002800F08D80019B9A60A3F81EC038
:103D1000A7E7002E3FF4F6AE022A7FF4F3AE0028A8
:103D20007FF4F0AE0B7A03F00703012B3FF4EAAE09
:103D3000CAF81C608AF81BB0E4E6019B9E69002E5D
:103D40003FF4E0AE022A7FF4DDAE0028F0D0D9E6E1
:103D5000079F0999A28A2CE6019A93785370002054
:103D6000AAE750460499FFF741FA9AF818000B9B0E
:103D700083420ED19D420CD100238AF819309AF863
:103D80001A30002B49D0DAF824405346012203218F
:103D90008CE5FF2800F08E810B9BFF2B00F06D81DE
:103DA000DAF8003000EB400003EB0013D3F8088092
:103DB000B8F1000F64D002F0EBFC0A270446DAF8F1
:103DC0001430E21A22F07F42904507F1FF3702F1EA
:103DD00003011AD941452CBF5B18434423F07F45AA
:103DE0002846DAF82830984702F0D2FC031B2D1B36
:103DF00023F07F43033325F07F45AB4206D90FB153
:103E00000446DCE700DE0446D9E7012600238AF8F1
:103E100019309AF81A303343B5D10FB0BDE8F08F9E
:103E2000704797427FF670AF0290481C0390DFF80E
:103E3000C0E0029806940295039D05E00C462244DA
:103E40000130974280B210D9284C33441C19744574
:103E5000F4D82C46A3F1E8732244A3F5D4330130FF
:103E60009742A3F5A57380B2EED80199069C029DF6
:103E70004B6260441FFA80FC46E70C960696B0E45D
:103E80008AF819807FE7B268002A40F03281D6F8BC
:103E900018B0BBF1000F06D10A68002A00F0248197
:103EA0000C464FF0040BC26961680291043207921C
:103EB0002268914280F0D680A2EB010E18F8032010
:103EC0000892FF2A00F0CE80DE45C0F0CB800022B1
:103ED000AEEB0B01CDE90590CDE9031599460798A6
:103EE000089BDA46944617463BE000BF5A2B17FF63
:103EF000592B177F3D1F6544754528BF75460BEB51
:103F0000000296450CD355450AD3B269002A4AD01F
:103F1000227A120747D4B5EB0B0201D0824249D274
:103F20008A6A22B1127A02F00702012A31D08A6924
:103F30007AB3496869B30432BC4402EB0C00B2693D
:103F4000002A7FD0217A0907AEEB0B0200F1A38093
:103F500018F803300027FF2B2CD00BEB0C0AD645AA
:103F600028D303EB430308EB03111B018D682F4497
:103F7000042FBFD8B56985B1257A15F00805BED0E4
:103F800088690399BC4404306044814228BF0246DA
:103F9000DEE718F803300022DDE78A69BC4404320A
:103FA00062441046D4E70028BAD0A5EB0B05854241
:103FB000B6D302460299049D06984B4611446160AF
:103FC00018F80370DDF81490FF2F00F09C804FF07C
:103FD000FF0C9A4600E00F4639B201EB410108EBB5
:103FE000011E0901DEF80830934280F08E8018F837
:103FF0000110FF29BC46A2EB0302ECD15346FF2F70
:10400000B26015D0B9F1FF0F18F8031066D00FFA9F
:1040100089F202EB4202120108F802103FB207EBEC
:1040200047073A0118F8021008F8031008F8025080
:10403000F38B013BF383237A022262F302032372A0
:10404000012797E5024683E700287FF45BAD04264D
:1040500068E6019C059E079D42469B1AA3609AF85C
:1040600018B077E5029A626018F80330FF2B08BF9A
:10407000002248D00023B360DAE702F089FB04464F
:1040800002F062FB20B99AF81800CAF8144087E6DB
:104090009AF8180084E61146002276E7FF2304937D
:1040A000E6E4824637B90B9BFF2B03D10C9B002B18
:1040B0003FF462AE02F058FB044600287FF45CAE89
:1040C000CAF81C0002F064FB8AF81940CAF8140010
:1040D0009AF81A30002B3FF4A0AE54E601769DE723
:1040E000B16A00297FF4D8AE00DE4FF0040BB46A49
:1040F000D9E600DED6F818B0BBF1000FF0D0B46AF4
:10410000D1E6AB4626E5B26092E751469A460B46A9
:10411000AAEB0201CEF80810674670E7F8B5069ED4
:104120009DF81C50089CB8B9144F3A605A1E397259
:104130007B727E60D2B273B106EBC202546011464C
:1041400012F808398E4203EB4300A5EB030304EB9E
:104150000014DDB2F2D10DB10120F8BD099B3B6224
:104160000A9B7B62FF240B9BBB623C7602F010FB38
:104170007D817861FC76FD612846F8BD880E0020BF
:1041800040B9064B1A7EFF2A01D1187270476FF0B2
:104190000F0070476FF01500704700BF880E0020B9
:1041A00010B40A4B2C2202FB0032546A5CB100EBC3
:1041B000800200EB420003EB8003A446012210BC06
:1041C00003210220604710BC704700BF880E00200A
:1041D00010B58AB00C9C00940D9C01940E9C029426
:1041E000BDF83C400394109C0494119C0594129CCF
:1041F0000694139C0794149C089400240994FEF7D9
:104200009FFF0AB010BD00BF10B4BDF81040049469
:1042100010BCFEF795BF00BF2DE9F84F294DBDF842
:1042200034609DF83880044608462C2101FB045177
:1042300004EB840704EB470405EB84054C6804EBAE
:10424000C00E14F830909EF803409EF8017004F1FF
:10425000010C5FFA8CFCE14598BF4FF0000C6745FC
:104260009DF844902AD0DEF8047004EB44044FEA31
:10427000041A07EB04144FF0050B07F80AB063604B
:104280000A9BA3600B9BE3600C9B23610F9BA362C3
:10429000109BE36202236270A68284F8168084F881
:1042A0001790A3708EF803C0D1E9083698472B46C3
:1042B00000220421B047A078BDE8F88F0120BDE8B6
:1042C000F88F00BF880E002010B588B00A9C0094BB
:1042D0000B9C01940C9C0294BDF8344003949DF80F
:1042E000384004940F9C0594109C06940024079475
:1042F000FFF792FF08B010BD2DE9F0411E4D0646B4
:1043000008462C2101FB065E06EB860406EB4404FE
:10431000DEF8046005EB840706EBC00516F8306094
:10432000EC78697804F1010C5FFA8CFC664598BF63
:104330004FF0000C61451BD0696804EB4404260172
:1043400001EB04144FF0070801F80680A362069BF6
:10435000E36202236270A37085F803C0DEE90835CA
:1043600098473B4600220421A847A078BDE8F08189
:104370000120BDE8F08100BF880E002002F008BADD
:10438000401A20F07F40704700200021704700BF96
:10439000002303700B70704738B5054600200C46AB
:1043A00001F0E0F970B93DB9074B44B120681860DD
:1043B000A2889A80002038BD044B002CF6D11C60E6
:1043C0009C80F7E70C2038BDBC0E0020B40E002006
:1043D0000128034605D8044A0448002B08BF1046AC
:1043E00070470020704700BFBC0E0020B40E0020B4
:1043F00001280AD8064A074B002818BF1346186838
:1044000008609A888A8018467047002318467047CB
:10441000B40E0020BC0E002010B5044601F0E0FCF4
:1044200038B901F0AFFF48B92046BDE8104007F0A9
:10443000DFB800DE01F0A6FF0028F5D000DE204640
:10444000BDE8104007F0D4B80860014807F0D0B8C4
:104450004012002007F0CCB82DE9F041284E294F3A
:1044600082B04FF00008D6E9000101AAFEF7A6FCD1
:10447000044670B1019D002D3AD02B79022B0BD050
:1044800000DED6E9000101AAFEF798FC04460028E8
:10449000F0D102B0BDE8F081002270683146FEF72D
:1044A00095FCAA6832B11378002B26D01378013B13
:1044B000DBB213702B7B03B100DE85F80C807B7DB3
:1044C000397D0133DBB2052B08BF0023994212D09E
:1044D0002C60797D47F821507B75002AC3D0137872
:1044E000002BC0D19368002BBDD0D0689847BAE7A5
:1044F00000DE019DC1E700DEEFE700DED6E700BF8A
:10450000F00E0020201100202DE9F0471C4F3D88BF
:10451000FE2D2CD815F0FF0527D0DFF868A0DFF8B6
:1045200068809AF81540DFF864909AF814300134E6
:10453000E4B2052C08BF00249C42404615D0FEF78B
:10454000EBFB0646484686B1FEF7E6FB88B10660FF
:104550009AF815304AF823003B888AF81540013D47
:10456000013B15F0FF053B80DFD1BDE8F087FF255B
:10457000D3E730460449BDE8F047FEF7E3BB00BF90
:10458000F80E002090100020FC0E0020380F0020B4
:104590002DE9F84F304B314FDFF8C490DFF8B8B059
:1045A0000422981814214FF00008A7F81480FEF791
:1045B0008FFB2B4B042208219818FEF789FB97F8F4
:1045C00014A07C7D04260134E4B2052C08BF00242D
:1045D000A245484613D0FEF79FFB0546584675B1E5
:1045E000FEF79AFB002832D0C5F8048005607B7D79
:1045F00047F82300013E16F0FF067C75E3D1194B06
:104600000522181D4421FEF763FB174B0722181DD6
:104610000821FEF75DFB1448FEF77EFB98B1134AB4
:10462000111FFEF7BDFB1048FEF776FB68B1104A7C
:10463000111FFEF7B5FB0F4B04221A80FFF764FF32
:104640000020BDE8F88F00DEE9E700DEEFE704496F
:104650002846FEF777FBD2E7CC100020201100207F
:10466000A8100020380F0020FC0E0020F40E0020BF
:10467000EC0E0020F80E002030B51F4B1F4C1860C8
:1046800087B002F053F8237873B31D4A1D4D1E4CBA
:104690001E49CDE904251E4A0220CDE90224042347
:1046A0000C24CDE900141B4A087408760B700B72B9
:1046B00000200321FFF732FDD8B90122002116485E
:1046C0000AF0C3FB01F02AFB08B107B030BDFFF7C9
:1046D0005FFF0028F9D101F03DFE0028F5D107B0B9
:1046E000BDE8304000F0CABFFEF780FB0123237015
:1046F000CBE700DEE1E700BF3C120020591A0020A2
:10470000896E0000296F0000696E00009814002077
:1047100058120020B81400204012002010B586B0B6
:1047200000F0BCFF38BB194A194B0024A2F8004125
:104730009C820122214668460AF087FB154B2246DF
:1047400021460320C3F808D0FEF770FBA8B94FF04C
:10475000FF324FF0FF33684606F084FF00F0DEFFC3
:1047600068B9FFF715FF78B90021012006B0BDE850
:104770001040FFF711BE00DED5E700DEE7E700DE00
:10478000FFF706FF0028EFD000DEEDE7381100202C
:10479000901000200C07002008B5FFF7BFFF01F0C4
:1047A000F3FA00B108BDBDE80840FFF7E9BC00BF5F
:1047B00010B50022074B026082B0044601AAD3E97B
:1047C0000001FEF7FBFA08B1019B2360002002B054
:1047D00010BD00BFE80E002000B50B4983B00023D8
:1047E0004868019301AAFEF7F1FA58B10749FEF7AC
:1047F000A9FA019B1B790BB12D2B00D000DE03B071
:104800005DF804FB00DEF1E7E80E0020FC0E00205E
:10481000F8B50468064654B10F4D104F2046246881
:10482000037953B12D2B09D000DE002CF6D10023E3
:104830003360BDE8F840FFF767BE00DE2B88032B2E
:1048400007D8013339462B80FEF77CFA002CE5D1DE
:10485000EDE700DE2B88F4E7F80E0020380F00208B
:10486000022810B50C4602D00B68022B07D0044872
:104870004FF0FF324FF0FF3306F0F4FE206810BD1A
:104880004012002004490A680AB1104670470246E7
:1048900008601046704700BFE40E0020044A136809
:1048A00023B1984206BF00211160002318467047CB
:1048B000E40E0020014B1868704700BFE40E002092
:1048C00030B505682B7887B0EBB104460122002192
:1048D00068460AF0BAFA0D4BC5F80CD0AB602B78DD
:1048E0008BB10B4B0022114603209C60FEF79EFA11
:1048F00038B94FF400420023684606F0B3FE07B013
:1049000030BD00DEF5E76FF07700F8E755440000B2
:10491000FC0600200B490A7D4B7D9A420AD8A3EB86
:10492000020C5FFA8CFC604509D89A4207D051F816
:104930002200704705339B1ADBB29842F7D900205A
:10494000704700BF901000202DE9F0431A4D9DF8EC
:104950001C8095F801C10CF1010E5FFA8EFEBEF1CC
:10496000080F994695F8003108BF4FF0000E7345C7
:104970001DD0144605EB4C1CE36807460E46106834
:104980005168926864460FC49CF81C30CCF81860DB
:1049900008F0010823F0030343EA0803CCE9049775
:1049A0008CF81C3085F801E16046BDE8F0834FF0DB
:1049B000000C6046BDE8F08338110020054890F8EF
:1049C000003190F801219A4214BF00EB43100020FF
:1049D000704700BF3811002001460B480A7890F854
:1049E0000131072A84BF90F800210A70934208D051
:1049F000531CDBB2082B08BF002300EB42100B70E6
:104A000070470020704700BF381100202DE9F04F9B
:104A10003D4E96F8001196F8013187B08B42039015
:104A200047D04FF0000906EB41110A24CDF8109051
:104A3000CA46CB46CDF80890CDF814900D7FD1F83A
:104A40000080CF68C5F3400205F00105002C4FD06F
:104A5000013CE4B282B396F8011196F80031994214
:104A600027D00133DBB2082B08BF0023994286F818
:104A700000311ED006EB43115B01C868002ADDD16E
:104A800035BBBBF1000F37D0BAF1000F029A08BF57
:104A90004246029208BFBA460A7F9507CED4D20793
:104AA0001DD48345F3582BD08245C7D1029A9A4230
:104AB000C4D107B0BDE8F08F144B0398996011463C
:104AC0000192FEF7B3F9019A0028C4D000DEC2E7D4
:104AD000049A7AB1B9F1000F08BFB946DCE7BAF120
:104AE000000FABD1049B8342E3D04845A6D1E0E759
:104AF00000DEADE70497CFE7BB46CDF81480CBE7E7
:104B0000059A9A42D0D1D4E738110020DC06002063
:104B100070B5114A117D537D8B421BD04B1CDBB20B
:104B200052F82140052B08BF0023137594B10223CE
:104B3000054600262068094A237121462660A560A3
:104B4000FEF732F90122064B11463046FEF76EF9A8
:104B5000204670BD0024FBE720110020F40E002049
:104B6000EC06002010B582B0049B9C7A6FF34104E0
:104B70009C720024CDE9004401F01EFA02B010BD81
:104B800010B50346007F1A699969012482B020405C
:104B9000CDE90004586901F00FFA08B902B010BD60
:104BA0007730FBD000DEF9E70B8A002B33D030B52D
:104BB000054683B001F10C000C4608F06EFC01289C
:104BC00026D1002301A92046019300F0E1F9014616
:104BD000C0B1C36828691A78042A05D0036828463A
:104BE000984720B103B030BD5B78052BF6D1019D0D
:104BF00045B1284600F0F2FB0346019907486B7166
:104C00000AF00AF92046FCF72BFF002003B030BD64
:104C10006FF01500E6E76FF0150070474C150020A7
:104C200010B50469FFF7B8FD40B90548FCF79AFBD9
:104C30000448FCF797FB0020206010BD00DEF4E77D
:104C400078090020F80900202DE9F0432E4FD0F814
:104C5000108083B006464FF000094FF0FF324FF04E
:104C6000FF33384606F092FC0028F6D090F9053064
:104C700001905A1E032A2FD8022B35D04FF0FF3255
:104C80004FF0FF330220FCF74BFF04460198002C45
:104C900034D0214600F09CFB019B01A8C3F8009092
:104CA000FFF7B6FD204608F0ACFB05462146002084
:104CB00008F0ABFB2B8A012B04462946304607D966
:104CC000D8F80030984707F02DF9002CEAD1C4E756
:104CD0002846FCF7C5FEF6E700DE019B01A8C3F8F5
:104CE0000090FFF795FDB8E7002200230121002086
:104CF000FCF72EFF04460198002CCAD1046001A8DD
:104D0000FFF786FDA9E700BF4C15002070B5114ED6
:104D1000114D82B00DF1020101A8FFF749FD0028F5
:104D2000F8D1019B6BB1FFF757FD019C204600F0C5
:104D300055FB0199607128460AF06EF8019B002B23
:104D4000E8D14FF0FF324FF0FF33304606F08AFCD7
:104D5000E0E700BF641500204C150020F0B50546C3
:104D6000076989B00E461F480AF018F84FF0FF3265
:104D700000211D480AF069F81B48FFF77DFC044636
:104D800060BB3E6000F02CFB002600276FF009039B
:104D9000CDE90334CDE90667CDE90144134B14494D
:104DA00000954FF4E072134806F0A0FE1249114836
:104DB0000AF01BF96FF00702CDE90324CDE906677D
:104DC000CDE901440D4B0E4900954FF460720D483A
:104DD00006F08CFE0C490B480AF007F9204609B092
:104DE000F0BD00BF4C150020641500200D4D0000E3
:104DF000C01F002078090020FCFB0000494C000087
:104E0000C0210020F80900200CFC000010B507F0BC
:104E100039F8054C204609F0CDFF204609F0BEFFC9
:104E2000BDE8104007F042B84C150020F0B501383D
:104E300087B01446092806D8DFE800F009273D05A9
:104E4000054F056180936FF0150007B0F0BD4E4B24
:104E50000D21188808F094FB0D2120600C3008F01B
:104E6000E4FA4FF0021400234FF480610322037030
:104E7000C0F80140A0F80510C2710372437283723A
:104E8000C3720373002007B0F0BD3F4B4121188867
:104E900008F076FB412120600C3008F0C6FA0021B2
:104EA00004463E2200F8031B0AF0D6FA40F2A7336C
:104EB000A4F80130E6E7344B0921188808F060FBBC
:104EC000092120600C3008F0B0FA0346002203F8F4
:104ED000012BC0F801205A60D4E7C9680020FFF711
:104EE0005BFA294B0121188808F04AFB012105468D
:104EF0000C3008F09AFA002303702560C2E7234EB5
:104F0000214F0FCE01AD0FC5336838882B701221A9
:104F100008F036FB122120600C3008F086FA0446B7
:104F2000002301AE04F8013B84460FCE2D78CCF867
:104F300001006160A260E3602574A3E7124B1821B1
:104F4000188808F01DFB182120600C3008F06DFA5D
:104F500000230446012100F8023B01F06DFB607064
:104F600090E7094B2121188808F00AFB21212060D5
:104F70000C3008F05AFA0146002301F8113B0130C9
:104F800001F0AAFB7EE700BF4C1A00202CFC0000B9
:104F9000F0B5038A8BB00026022B059636D904465D
:104FA00003210C3008F071FA228A83789A422DD3BB
:104FB0000188DE4FC1F38523082B88B23980C1F305
:104FC000090538D011D8032B24D0042B18D1691E21
:104FD000082915D8DFE811F0CC000101EF0014001A
:104FE0001400140014001400E0003F2B08D105AA9F
:104FF00021462846FFF71AFF163040F0E78138882F
:1050000001210BB0BDE8F04008F0CCBA00242046E6
:105010000BB0F0BD032D00F0CA81632D01D0012D2E
:10502000EED1012108F0ACFA012104460C3008F061
:10503000FCF90670EBE7691E4A29E1D801A353F891
:1050400021F000BFBF5200009F52000057520000E5
:1050500001500000A5530000895300007153000067
:1050600065530000595300003953000001500000FF
:1050700001500000015000000150000001500000EC
:1050800001500000015000000150000001500000DC
:10509000015000000150000001500000F3520000D8
:1050A000D5520000015000000150000001500000E6
:1050B0003952000001500000015000000150000072
:1050C000015000000150000001500000015000009C
:1050D000015000000150000001500000015000008C
:1050E000015000000150000001500000015000007C
:1050F000015000000150000001500000015000006C
:10510000015000000150000001500000015000005B
:10511000015000000150000001500000015000004B
:10512000015000000150000001500000015000003B
:10513000015000000150000001500000015000002B
:10514000015000000150000001500000015000001B
:10515000015000000150000001500000015000000B
:1051600001500000015000000150000019520000E1
:10517000092108F005FA092104460C3008F055F918
:105180004FF4506100236A4A01800D218370C3707F
:105190000171C0F805203AE7072108F0F1F907216D
:1051A00004460C3008F041F90146002001F8010BDB
:1051B000FFF71EF92BE7092108F0E2F9092104465F
:1051C0000C3008F032F90346002203F8012B60216D
:1051D000C0F801205A60417119E7412108F0D0F967
:1051E000412104460C3008F020F9002105464022F8
:1051F00000F8011B0AF030F9C022AA714FF40A72BC
:1052000004234C49A5F80F208022EB72EB75C5F8FA
:105210001A1085F82720FAE6032108F0B1F90321D6
:1052200004460C3008F001F90146002301F8023B66
:105230000130FFF7ADF8EAE6092108F0A1F90921EC
:1052400004460C3008F0F1F800234FF4407202607D
:1052500043600372DBE6092108F092F90921044654
:105260000C3008F0E2F80346002503F8015BC0F8B3
:1052700001505D600646FFF787F82B4661F3070390
:10528000C1F3072262F30F23090C61F31743090AE4
:1052900061F31F63C6F80100C6F80530B7E60421C4
:1052A00008F06EF9042104460C3008F0BEF8002323
:1052B0001B210322037041708370C270A7E6012195
:1052C00008F05EF9012104460C3008F0AEF8002326
:1052D00003709CE6092108F053F9092104460C30BB
:1052E00008F0A3F8002300F8013B082100F05CFD62
:1052F0008DE6E068002306AA00F1100101F066FEC9
:105300003888112108F03CF9112104460C3008F0CE
:105310008CF80646002306F8013B06AD07460FCD84
:10532000C7F801007160B260F36070E64C1A0020AB
:10533000F105FFFFF703C008E3681878FBF78CF866
:1053400005460121388808F01BF9012104460C307C
:1053500008F06BF805705AE6E16811F8010B00F0EF
:10536000D3FAEDE7E16811F8010B00F05FFAE7E727
:10537000022108F005F9022104460C3008F055F826
:1053800000230370437042E6E468A57BA379627949
:10539000217920880295657B01950734009400F0FF
:1053A000FFF8CDE7E1680120FEF7F6FFC8E7FFF759
:1053B000B5F93888012108F0E3F8012104460C30E2
:1053C00008F033F80670FFF721FD20E6059C1EE685
:1053D0000379032B00D000DE704700BF0020704728
:1053E000FFF714BD094A0A4B12781A7000B97047CA
:1053F00000B583B00191FFF75DFA0199814202D1B6
:1054000003B05DF804FB00DEFAE700BF5B1A002082
:105410005A1A00200D4B597E1A7D03EB810102F0D0
:105420003802C96942F007021A75062000224FF4BB
:10543000006CA3F830C00A70487093F8251003EB95
:10544000810304229B6A1A7058707047A0150020CF
:1054500010B4047804F00F0402F1FF3C022C1FFA90
:105460008CFC1FD0012C0AD04B781033DB0084B1A8
:10547000062C0ED040F253204FF4F37203E040F2BA
:10548000E33040F2162212FB0CF3184480B210BC39
:10549000704742781032D20002F21B31581802F5E0
:1054A000B372F0E7417810BC0CEB8C03C3EB031034
:1054B000400001F1100300F23B10DB0003FB02028D
:1054C00090B2704710B54FF6FF718AB08B429DF8CD
:1054D00030C00D9C19D021780131C9B2217000294A
:1054E00049D02749C1E900028A7A0B816CF3000296
:1054F000244B8A7204F110000022C86099600120D8
:105500001146FDF793FC002837D11F4A1F4B117835
:105510001B788B4201D00AB010BD0133042109A8C9
:10552000137000F04BFC099B1949A1FB0321A3EB6D
:10553000010C01EB5C0140F24710090A154A00FB1F
:1055400011331549A21AA1FB0212120913490020B6
:105550000232CDE905140133CDE90300CDE90100A4
:105560000090D2B201210993FEF7AEFE10F0FD0FBC
:10557000D1D000DECFE700DEB3E700DEC5E700BF35
:10558000841500201C0700205B1A00205A1A0020F6
:1055900021F1D490A01500204FECC44EE55300003B
:1055A00070B58C463349344C864603C982B00090AE
:1055B00094F832008DF8041010F001009DF81C5092
:1055C0009DF8201043D105F0070545EA81150CF13F
:1055D0000801BCF1010F0DEB010C667E1CF8081CE4
:1055E00094F814C004EB86060CF0380C45EA0C0560
:1055F000F669257508BF4FF0000EA4F830E0357845
:1056000001F00F0125F03F05294301F00F05012DA1
:10561000317002F0010C1DD06CF38611737860F3C9
:10562000C71131700BB90623737094F825302461CB
:1056300004EB83049201A36A02F04002597842F01D
:1056400004021A7009B906225A7002B070BD0C200B
:1056500002B070BD6CF3861163F3C7113346069D2B
:1056600003F8081B2D68B560069D0C21AD889D8050
:105670007170DAE724FB0000A015002010B5064C7D
:10568000204600F097FE04F10C0000F093FEFFF7B7
:10569000C1FE002010BD00BFB815002030B51C4C65
:1056A00094F83230DB0785B020D52046FFF7EAF8C2
:1056B000844225D103AD02220321164B0095002020
:1056C0000392FEF719FE2946FFF7CAF888B9124877
:1056D000FFF7F6F8B0B90E48FFF7E0F8844215D1AD
:1056E00094F832306FF3000384F83230002005B0B4
:1056F00030BD0748FFF7D2F88442F7D000DEF5E767
:1057000000DED7E77830E6D000DEE4E700DEE7E74A
:10571000A015002049440000B015002038B5094C00
:1057200004F10C05204600F055FE284600F052FE1C
:10573000204600F03FFE284600F03CFEFFF76AFEE0
:10574000002038BDB8150020044A0068044B801AB8
:10575000A3FB0030C0F30F10704700BFA01500205E
:105760004FECC44E28B9044B93F8320000F001000E
:1057700070470020704700BFA01500201F294ED899
:105780002DE9F041437E00EB830382B0DF693B7873
:1057900003F00F03012B044643D00E4618300DF1E1
:1057A0000701904600F060FE3A78037802F00F029D
:1057B00023F03F03134303703B780278C3F3801355
:1057C000394663F38612027011F8023BD2B2DB094C
:1057D00063F3C712054600F8022B062209F022FEE9
:1057E0003246414605F10800063609F00DFE6E709E
:1057F00094F83230DB0706D49DF80730637600203A
:1058000002B0BDE8F08194F8253004EB830329460B
:105810009A6A2046FAF704FF0028EDD0F0E712203C
:1058200070470C2002B0BDE8F08100BF03460A4675
:1058300001481946FFF7A2BFA01500201F295ED816
:105840002DE9F04190F8253000EB830382B09E6A89
:105850000F460446904600F12405002E40D028460D
:105860000DF1070100F000FE037823F03F033146FD
:1058700043F00403037011F8022BDBB2C2F3801271
:1058800003F03F0343EA82130370BB1D43700546D8
:105890000622023009F0C6FD3A46414605F10800ED
:1058A00009F0B2FD94F83230DA0707D49DF80730DA
:1058B00084F82530002002B0BDE8F081627E04EB60
:1058C00082024123D1690A7802F00F02D340DB073C
:1058D000ECD52A462046FAF7A3FE0028E6D0EAE7F0
:1058E000284600F067FDC0B258B994F8253004EBA3
:1058F00083039E6A0423337006237370AFE712207C
:1059000070470720D7E700BF03460A4601481946FB
:10591000FFF794BFA015002000F046BA684620F0BB
:1059200007018D4601B500F041FFFBF7E9FABDE83C
:1059300001408546704700BF08B50A4BD3F84021A7
:105940003AB90120FDF7D0FABDE808400220FDF782
:10595000CBBA0020C3F84001D3F84031FEF720FC59
:10596000EFE700BF00B000400020FDF7BDBA00BF68
:1059700090B90E4B0E4A197810788842CBB20DD1EF
:105980000C480D4990F800C0013313700B78634543
:1059900007D003780B70704700DEEAE700DE13786B
:1059A000EEE700DE03780B70704700BF5C1A002042
:1059B0005D1A0020611A0020601A00200B4A0C4B6F
:1059C000117893F800C08C450DD012781A70094AEE
:1059D000094B18B911781878884202D012781A70D9
:1059E000704700DEFAE700DEEFE700BF5F1A002035
:1059F0005E1A00205C1A00205D1A002000F0FCBF37
:105A000008B50B480B4B027819788A420CD00A4B28
:105A1000017000220399996001201146FDF706FAF2
:105A200000B908BD00DE08BD00DE1978EFE700BF51
:105A30005C1A00205D1A00202C0700202DE9F0419F
:105A4000304A314D12782B789A428AB00E4605D1F1
:105A50002E4B2F4A1B7812789A424BD03768DFF8CA
:105A6000B48007F12D0424F07F44D8F800102046BC
:105A7000FEF786FC10F4000002D10AB0BDE8F08108
:105A8000254A264B11781A7891421CD03046244B77
:105A9000C168C8F800400022CDE90732214BCDE9AA
:105AA0000322CDE90531CDE901222D2300932C7885
:105AB0000134E4B23B46114610462C70FEF788FBD9
:105AC0000AB0BDE8F081114A114912780978914273
:105AD000DCD01A780132D2B21A700022124B009236
:105AE00011461046FEF708FC10F0FD0FCED000DE88
:105AF00000DECBE70768DFF81C8007F12D0424F0F7
:105B00007F44C4E7601A0020611A00205C1A00205C
:105B10005D1A0020DC1500205E1A00205F1A0020AC
:105B200071590000015A0000BD5900007A4A93687B
:105B3000002B00F096802DE9F04F136889B0814664
:105B4000002B46D04FF0FF338DF80A300DF10A00DC
:105B5000FEF742FF044600283BD0037F9907F5D1AA
:105B6000857A15F00205F1D1C3684B4555D006681A
:105B7000A8462F460DF10A00FEF72EFF8346F0B12E
:105B8000027F9207F6D1827A9307F3D4C268B8F104
:105B9000000F21D04A4558D0DBF800A031465046CE
:105BA000FEF7EEFB00F4000000280DF10A001CBF18
:105BB0005F465646FEF710FF83460028E0D1002FCF
:105BC00008BF274639463846FFF738FF30F0020352
:105BD00039D109B0BDE8F08F4A458046DCD1237F3A
:105BE000E16843F0020323772046A3699847FF2327
:105BF0008DF80A300DF10A00FEF7EEFE044600288B
:105C0000E7D0037F9F07F5D1837A9E07F2D4C3685C
:105C10004B4502D000DED4F80C903F4A4846D2E90A
:105C2000001303AA98470646002843D010F1100F2E
:105C300059D0394A002093681168984716F10B0F24
:105C400010D08C36C5D000DEC3E7227FE16842F079
:105C5000020222772046A2699047D8457FF472AFAE
:105C6000C5E770472C4A0023D2F80890D2E90048D3
:105C700002261360FF278DF80B700DF10B00FEF765
:105C8000ABFE90B1037F9A07F7D40DB9DB07F4D4CC
:105C9000C368A342F1D1037F826943F00203037713
:105CA000214690478DF80B70E7E70125AE420AD0F8
:105CB0002E46E0E7237FA269E16843F002032377E1
:105CC0002046904785E70022CDE904220692039BF7
:105CD00000964946404604AA0794FEF735FE002880
:105CE0007FF477AFAFE7A37A43F00203A3720DF11D
:105CF0000A00FEF771FE014600283FF46AAF037FF9
:105D00009D07F4D1837A9C07F1D4FFF797FE30F01A
:105D100002033FF45EAF96E7E015002010B5174888
:105D200008F05EFF30B3164B00249C6000F0F6F9DB
:105D300000281EDB214601202246FBF79BFB224662
:105D40000B200121FBF796FB214622461820FBF78A
:105D500091FB0C4B1022C3F804230120FBF75AFBE4
:105D60000B20FBF757FB1820FBF754FB00F038FD26
:105D7000204610BD6FF0120010BD00BF6CF6000091
:105D8000E01500200010004008B500F0D7F9002809
:105D900009DB0120FBF74CFB0B20FBF749FB18202C
:105DA000FBF746FB002008BD034603488AB21946AC
:105DB00083681B68184700BF6CF6000030B4074DBD
:105DC000AB685C6834B18AB2A44601460023284619
:105DD00030BC60476FF0850030BC70476CF6000047
:105DE0000020704730B5044683B078B31D4B1A6865
:105DF000824225D0FF250DF107008DF80750FEF7F0
:105E0000EBFD38B91AE0A1420AD00DF10700FEF708
:105E1000E3FD98B1037F9B07F7D4C168002CF2D152
:105E2000037F826943F00203037790470DF1070077
:105E30008DF80750FEF7D0FD0028EBD103B030BD40
:105E40009B686BB1014600209847D3E7054A9368E9
:105E5000002BCFD011680029CCD000209847C9E78B
:105E600000DEC7E7E01500200020704710B50446AB
:105E7000FEF7A4FD8CB90D4B9A68AAB11C680022EC
:105E80009A601A6004B124680020FEF7BFFD204626
:105E9000FEF73EFE28B1002010BD0028F3D100DE41
:105EA000F1E700DE002010BD00DEE7E7E01500208E
:105EB0002D20704710B51446FEF760FA2146FEF714
:105EC0005FFA034610F4000004D10333092B88BFA6
:105ED000184610BD002010BD262810B504461DD060
:105EE000272813D0252809D00A281FD9272822D9E6
:105EF00000DE2046BDE8104000F0F2BC022000F0B9
:105F0000E9FC2046BDE8104000F0EABC502000F05B
:105F1000E1FC2046BDE8104000F0E2BC1A2000F091
:105F2000D9FC2046BDE8104000F0DABC0230400049
:105F300000F0D0FCE5E70330400000F0CBFCE0E7E8
:105F400008B500F059FDBDE8084000F08FBE00BF65
:105F500008B500F051FD00F089FE00F06DFEBDE8CF
:105F6000084000F04BBE00BF08B50146114800F0E4
:105F70002DFC00F06DFD60B100F008FF00F094FC16
:105F800000F004F900280EDBBDE808400020FFF710
:105F90006DBF00F011FD00F0F9FE00F085FC00F08F
:105FA000F5F80028F0DA00DE0020BDE80840FFF731
:105FB0005DBF00BFFD5900002DE9F04F89B01F46BD
:105FC0009DF848B0FF238046894692468DF81F30E1
:105FD0000DF11F00FEF700FD002866D0037F9D072E
:105FE000F6D1837A9C07F3D405683E689DF81F308C
:105FF0000593044629463046FEF7C2F9BBF1000F6F
:106000004CD0BC4208BF002426460DF11F00FEF70D
:10601000E3FCD0B1027F9107F7D1827A9207F4D4E2
:1060200002680490294610460392FEF7A9F9039AE4
:10603000049B00F4000000280DF11F001CBF154652
:106040001E46FEF7C9FC0028E4D1059B8DF81F30E1
:10605000314B9A687ABB76BB24B1BBF1000F48D1B3
:10606000BC4244D1FA681A60C3E901893846D04776
:1060700004460DF11F00FEF7AFFC014650B1037F4F
:106080009A07F6D1837A9B07F3D4FFF7D7FC30F059
:1060900002033FD1204609B0BDE8F08F0002B0D521
:1060A000FF23354605935C46AEE71B4B9A680446D2
:1060B000002AD7D026464946CDF800B05346404680
:1060C0003A46FEF741FC014678B1BBF1000F09D119
:1060D000BB7A980706D4C6B13046FFF7AFFC30F064
:1060E000020310D16FF07604D4E700DEEDE700DEA6
:1060F000B8E7CDF800B053463A4649464046FEF769
:1061000023FC0028EED100DEECE7002C14BF26466D
:106110000E46E1E700DEBDE7E015002010B50120E6
:1061200001F0A4FB0449002301244B608C60CB6088
:10613000BDE8104006F0A5BFF015002010B5012005
:1061400001F094FB0449044607F016F82046BDE828
:10615000104006F0EDBF00BFF015002008B50A4B57
:10616000BFF35B8F53E8002F511C43E80010002859
:10617000F8D1BFF35B8F002A01DD002008BD01F0DC
:106180007DFB002008BD00BFEC15002008B50E4BBC
:10619000BFF35B8F1A68BFF35B8F002A11DDBFF37B
:1061A0005B8F53E8002F511E43E800100028F8D100
:1061B000BFF35B8F012A01DD002008BD01F074FBF5
:1061C000FAE76FF0770008BDEC1500206FF08B0048
:1061D000704700BF10B50446FFF7BAFE00F022FD7D
:1061E0002046BDE81040FFF7BFBE00BF38B50446EB
:1061F00000F02CFCFFF7A4FE962000F047FD0023E2
:1062000018461A46194600F08BFC0120FEF782FB67
:10621000F0B11C3000F0B6FB00F004FC00BB2146DE
:10622000104800F0D3FA00F0D3FD002104460846E0
:1062300000F0B6FB00210546084600F0AFFB2C44F9
:10624000CB34201A00F0AEFDBDE8384000F0B8BDF8
:1062500000DE1C3000F096FB00F0E4FB0028DED0EE
:1062600000DEDCE79962000010B548B10C46FFF78C
:106270008DFF00280BDB2046BDE81040FFF7F6BD80
:10628000044800F0A3FABDE8104000F095BB00DE22
:10629000F1E700BFD561000070B5044600F0CCFB0B
:1062A000C0B248B9FFF754FE2146294800F08EFAE3
:1062B000BDE8704000F080BB00F0E0FB054600F058
:1062C000C5FCEDB2064600F0CBFC00F0A1FCFFF7E8
:1062D0003FFE002DE8D00120FEF71CFB0146002800
:1062E00032D0237A0A7F04EB8303D868037803F063
:1062F0000F05012DC3F38013D6D002F00F05032D37
:10630000D2D14D7F0C2DCFD125796D0602D5F6B2B5
:10631000002EC9D0B3EBD21FC6D1062224310230E1
:1063200009F0A2F80028BFD10948214600F04EFA32
:1063300000F056FC237D04EB8303986900F028FBF2
:1063400000F070FB10B970BD00DECAE700DE70BD62
:10635000C9650000084B042210B598182821FCF7E5
:10636000B7FC064B00249C8102222146044808F019
:106370006CFD204610BD00BF281600201816002016
:1063800000160020084B042210B598182821FCF7AD
:106390009FFC064B00249C8102222146044808F001
:1063A00054FD204610BD00BF2816002018160020FE
:1063B0000016002010B504460548FCF7ADFC20B1DE
:1063C000034600205870636010BD6FF00B0010BDD5
:1063D00028160020034600201870587098607047F7
:1063E00038B51E4D2B7B6A7B9A4202D055F823406C
:1063F00034B91B48FCF790FC044680B1204638BDF8
:10640000184805F055F92B7B6A7B9A42F6D0013388
:10641000DBB2032B08BF00232B73204638BD114885
:106420004FF42032002305F01DF9A0B90D4805F006
:106430003FF92A7B6B7B93420BD0531CDBB255F8A0
:106440002220032B08BF00232B7312B114462046D1
:1064500038BD00DED2E700DEE8E700BF18160020F6
:10646000281600200016002010B5027843789A42C2
:1064700014D0D4B244700278944204D05A1C4370B1
:10648000D3B2022B0ED01A4600EB82040B70606868
:1064900000B110BDFFF7A4FF606010BD0133DBB297
:1064A000022BF0D100221346EEE700BFF8B50278C8
:1064B00043789342044625D0D5B2154A00EB8507B0
:1064C000507B92F80CC0431CDBB2032B08BF0023A7
:1064D0009C450E46796806D042F8201053730D484B
:1064E00005F086F800216B1CDBB2022B0ABF0022EC
:1064F0001A46134679602370012104EB820431703F
:106500006068F8BD1A4604EB82046068F8BD00BFFD
:10651000181600200016002030B50379C3F3C2031B
:106520000446002B93FAA3F0B0FA80F008BF4FF0B6
:10653000FF3083B000F101003AD021795A1E134098
:1065400063F3C50124302171FFF7C6FC00230DF170
:10655000070104F108008DF80730FFF7A7FF054693
:1065600020B3284600F014FA2B7803F00F03022B17
:1065700013D00DF1070104F11400FFF797FFE0B10C
:1065800021460F4800F022F9962000F07FFB002002
:1065900003B0BDE8304000F07BBA0A48214600F065
:1065A00015F903B0BDE8304000F01ABB00DED8E7B3
:1065B00000DE2379C3F3C203BFE700DEE0E700BFDC
:1065C000ED610000C965000010B5044600F03EFA18
:1065D000FFF7BEFC237913F0380F06D100F022FB41
:1065E0002046BDE81040FFF7BFBC2046FFF794FFF0
:1065F00000F0DCF9BDE8104000F0E2BB10B582B05D
:106600000446FFF7ABFD002809DB084A08490948A2
:1066100000940023FEF7A6FA18B902B010BD00DE00
:10662000F3E77730F9D000DEF7E700BFE1060000BE
:1066300069620000CD6100004FF080530246D3F83C
:10664000A410013107D04FF08051D1F8A00010F014
:10665000010009D17047D3F8A8304FF6FF719BB203
:106660008B42F0D100207047D1F8A4301360D1F8EC
:10667000A8301371C3F3072363F03F035371D1F8BC
:10668000903001331CD0D1F89430013318D0D1F8B8
:106690009830013314D0D1F89C30013310D0D1F8A8
:1066A0009030C2F80630D1F89430C2F80A30D1F8F0
:1066B0009830C2F80E30D1F89C30C2F8123008E0A1
:1066C0000023C2F80630C2F80A30C2F80E30C2F811
:1066D00012300120704700BF00234FF0805203604A
:1066E00043608360C360D2F88030013318D0D2F8A1
:1066F0008430013314D0D2F88830013310D0D2F86E
:106700008C3001330CD0D2F880300B60D2F884305A
:106710004B60D2F888308B60D2F88C30CB607047F9
:1067200000230B604B608B60CB607047054B4FF4D0
:1067300080320021C3F80815C3F84423C3F80423AA
:10674000704700BF00B00040054B1878421C1A701B
:1067500018B9044B01221A6070470120704700BF2E
:10676000621A002000B00040074B187848B1013889
:10677000C0B2187018B9054B01225A607047012049
:10678000704700DE1878F2E7621A002000B000407F
:10679000014BD3F80405704700B00040024B00F5F0
:1067A000A87043F82010704700B00040044BD3F8A5
:1067B000103123B1034A044B10681B681847704717
:1067C00000100040CC160020D0160020024A034BD7
:1067D00011601860704700BFCC160020D016002052
:1067E0004FF080434FF0FF320021C3F8002EC3F872
:1067F000042EC3F8081EC3F80C2EC3F8101EC3F8ED
:10680000142EC3F8182EC3F81C2EC3F8202EC3F87C
:10681000242EC3F8282EC3F82C2EC3F8302EC3F82C
:10682000342E70474FF080521B49D2F8303100208F
:10683000C1F81805591C1FD0062B09D0174B4FF46F
:1068400090514FF41052C3F80018C3F80428704751
:10685000D2F83431033B042BF0D8114AD25CB2B1E8
:106860000D4AD2F8743723F0807323F0010343F00C
:106870008073C2F87437E1E74FF0704393F8E02F6C
:10688000062ADBD1D3F8E83FC3F30313E2E7054A56
:10689000D35C002BD2D0E3E70010004000F00140B1
:1068A000F0FC0000E8FC0000704700BF054B022828
:1068B0000CBF0421032140F20122C3F81015C3F8D4
:1068C0005026704700100040014BC3F80C0570477C
:1068D00000100040014BC3F808057047001000404D
:1068E000084B00F07F00C3F85405D3F8182522F0B8
:1068F0000072C3F81825D3F8182542F00072C3F8C7
:106900001825704700100040084A00210123C2F8F2
:106910002C15C2F83035C378C2F824358178038845
:1069200043EA01431B02C2F81C35704700100040C7
:10693000C2F38203A3F1020302F00302B3FA83F36A
:10694000013A5B091B06022A98BF43F4801300F04A
:106950000F000A4A184340F48070C2F81405D2F8B8
:106960001805074B0340C2F81835D2F818351943FB
:1069700041F44031C2F81815704700BF00100040C4
:106980000000F8FE014BC3F80405704700100040FA
:10699000014BC3F804057047001000400120704708
:1069A00002280CBF06200A20704700BF014B0122BD
:1069B0001A607047001000400B4B0C480C4910B493
:1069C0004FF41064C3F8084501224FF480245A6044
:1069D000DA60C0F84843074CC3F808450020C1F806
:1069E00000020A6110BC704700F0014000B0004096
:1069F00000100040C001700C094B0022C3F80021B8
:106A0000D3F80011C3F80421D3F80411C3F80C2102
:106A1000D3F80C11C3F81021D3F81031704700BF20
:106A200000100040034BD3F80001003818BF0120CC
:106A3000704700BF00100040034BD3F80C01003832
:106A400018BF0120704700BF0010004001207047B0
:106A5000034BD3F85005B0FA80F04009704700BFEF
:106A600000100040044B40F20312C3F83425C3F871
:106A70003805C3F83C15704700100040034BD3F8AD
:106A80000004003818BF0120704700BF001000400C
:106A9000F0B41D4B1D4D1E4E1E4C1F4F0322C3F85C
:106AA00000222A78C6F8687502F10C03DBB2D00028
:106AB000DB00910003F1804300F1804003F5F833DF
:106AC00000F5F83001F18041C6F86C0501F5104180
:106AD00004EB82041148C3F81045C3F81405D1F83B
:106AE00040352D2B8ABFD1F8403501232D3BC1F80D
:106AF00040350132064B4FF4106102F00102C3F839
:106B000004152A70F0BC704700100040631A002082
:106B100000F00140409100400C1100400410004082
:106B20002DE9F041284E294C294FDFF8A8E0DFF885
:106B3000A8800323C6F800322178CEF8688501F1D9
:106B40000C03DBB2DB00CD0003F1804303F5F83327
:106B500005F1804507EB810705F5F835CEF86C5552
:106B60004FEA810CC3F8107549F63465C3F8146513
:106B70004AF24E23022A18BF1D460CF1804C42F205
:106B8000B84241F24A53022818BF13460CF5104C84
:106B9000124A2B44A2FB0323DCF84025B2EB931FDF
:106BA00085BF9809DCF8403501231B1ACCF8403525
:106BB0000131084B4FF4106201F00101C3F80425C4
:106BC0002170BDE8F08100BF00100040631A002072
:106BD0004091004000F001400C110040D34D621084
:106BE0000449054B03204FF41062C1F80002C3F8BA
:106BF000082570470010004000F00140034B0022C0
:106C0000C3F81C21D3F81C31704700BF00100040AE
:106C1000034BD3F81C01003818BF0120704700BF98
:106C200000100040034AD2F8403623F0FF03C2F8B8
:106C30004036704700100040034B0022C3F8142177
:106C4000D3F81431704700BF00100040034BD3F855
:106C50001401003818BF0120704700BF0010004029
:106C6000014BD3F810047047001000400449054B55
:106C7000054A4FF48020C1F84803C3F8082570473F
:106C800000B0004000F00140C001700C034B044A0A
:106C90001B7803F5A87342F823007047631A00209D
:106CA00000900040F0B4A2F574232F4DA3F51073AB
:106CB000AB42044606D902F1E87202F5D43201393A
:106CC00002F5A572294B2A482A4D2B4E0127DF6079
:106CD0000027C3F80475A0FB02020427C3F810754F
:106CE000900C0227C3F80875244AC3F84005C5F87C
:106CF00048154FF48021C5F844134021C2F840657F
:106D0000C2F84435C2F804154CB34FF48013C2F8EE
:106D100004351B4A012100240423D160C2F8044534
:106D2000C2F81035154BC2F8084511601549C3F873
:106D300050150C32C3F8542502F5AF32124CC3F88B
:106D4000584502F5FC7201F50041C3F85C25383165
:106D50000832C3F86015C3F86425F0BC70474FF4DF
:106D60000013C2F80435D4E7BFBDF07F00800040B7
:106D700083DE1B4300B0004048B1004000F00140FA
:106D8000009000400C110040409100400349044A2B
:106D900001234B600B61536013617047008000401A
:106DA000009000400449054BC1F844054FF088624B
:106DB000C3F80425704700BF0080004000F0014088
:106DC000024B4FF00062C3F80425704700F0014009
:106DD000014BD3F848057047008000400139012974
:106DE00005D80B200AB1FAF715BBFAF721BB00DE74
:106DF000704700BF29B10139012905D80B20FAF7E6
:106E00002BBB1820FAF728BB00DE0020704700BF1C
:106E100088420FD0012807D002280DD1A1F101002E
:106E2000B0FA80F040097047A1F10200B0FA80F09A
:106E3000400970470120704700207047012904D0A5
:106E4000022902D039B100DE7047064B4FF40062D0
:106E5000C3F800217047034B4FF08072C3F8002144
:106E6000704700BF00E100E0032803D8054B185C21
:106E700028B1704700DE034B185C0028F9D100DE12
:106E8000704700BFF8FC0000013810B41C4604280D
:106E900006D8DFE800F008111A23030004292FD0D8
:106EA00000DE10BC70470429FAD1194B9C6010BC5D
:106EB00002210020FBF7BABF0329F1D1154B0121B4
:106EC0009C6010BC0846FBF7B1BF0429E8D1124B07
:106ED0009C6010BC02210120FBF7A8BF032908D049
:106EE0000429DDD10D4B02219C6010BC0846FBF744
:106EF0009DBF0B4B9C6010BC01210220FBF796BF8D
:106F0000084B9C6010BC02210320FBF78FBF00BF21
:106F10008C0700207C0700206C0700204C07002015
:106F20005C0700203C07002001460020FFF736BC2C
:106F3000124B30B40121044600205960C3F80445C7
:106F4000C3F80001C3F80401196005E0D3F8042177
:106F500032B9D3F804251AB1D3F80021002AF5D0AC
:106F60005960D3F80421002AE7D1D3F80455002D45
:106F7000E3D0C3F8042530BC704700BF00E00040F8
:106F800070B5114C0126D4F8045566600E20FAF74E
:106F90004FFAD4F8040140B10021C4F80411D5E936
:106FA0000E323046BDE870401847D4F8003143B186
:106FB000C4F80001D5E90E3205F12001BDE87040AA
:106FC000184700DE70BD00BF00E0004070B58CB017
:106FD0000E4615460146102268461C46FBF7C6FEC3
:106FE00010220DEB02003146FBF7C0FE6846FFF7AA
:106FF0009FFF25B1102208A92846FBF7B7FE2CB148
:1070000008AD0FCD20606160A260E3600CB070BD80
:10701000142870B503460C4612D80B4A12F810100B
:10702000D4E9000502EB4302A0FB010652780023DD
:1070300001FB0561F9F754F8C4E90001002070BDB7
:107040006FF01500FBE700BF1A05010030B5002303
:1070500085B0CDE901330B7903F01F00C3F30402BF
:1070600007288DF80D2003D96FF0150005B030BD4D
:1070700013F0200418BF8B794A798DF80B2008BFD4
:1070800023468DF80C300B780C2BEDD801A252F86A
:1070900023F000BFCF700000C9700000F370000043
:1070A00069700000F770000069700000FB7000005C
:1070B0006970000069700000FF700000037100003B
:1070C000697000000771000001238DF806304B78CD
:1070D000032B1AD0042BC7D14B8844F20A029342E7
:1070E00038D843F6FE72934213D8002BBCD102234A
:1070F00040E00223E9E70323E7E70423E5E705236C
:10710000E3E70623E1E70723DFE701238DF80730F4
:10711000E2E7A3F57F533F3B0B2BA5D801A252F822
:1071200023F000BFAD7100006970000069700000BD
:1071300069700000797100006970000073710000CF
:1071400069700000697000006970000069700000DB
:10715000EF70000044F21402934225D044F228025A
:10716000934223D044F20F0293427FF47DAF032376
:1071700000E001238DF808301B4A012505FA00F0D4
:1071800092F86030C0B214B38C798CB9034382F8A2
:1071900060300B7992F8611003F01F0305FA03F3D6
:1071A0000B4382F8613009E00423E3E70523E1E7BC
:1071B00023EA00038DF8095082F8603001A803F03B
:1071C0006DF80A4B98427FF44FAF00204EE703431F
:1071D00082F860300B7992F8611003F01F0305FA12
:1071E00003F321EA0303DCE7F80500200000AD0B00
:1071F00010B50C4C94F84A3023B1BDE810400A4851
:1072000003F0EAB903F038F9084B984208D06FF060
:107210000403636304F11C00BDE8104006F0AEBA3D
:1072200010BD00BFF8050020317200000000AD0B5A
:10723000F8B50378002B40F09F80574CE36B94F82F
:1072400060701F4225460BD1544B0022C3F8002525
:10725000A36B002B3FD15248BDE8F84006F08EBA30
:10726000018994F8A800A26E94F86160A0B9012188
:10727000DBB20B420BD00F4208D016EA010CB2F978
:10728000000023D000EBD070401010800232490083
:1072900089B2B942EDD9D7E7334015D002EB4101AD
:1072A0009142D1D0B2F9003003EBD3735B1022F8D6
:1072B000023BF5E732F91360002EB8BF22F8130045
:1072C00001338B42F6DBBFE71846FAE70028B8BF68
:1072D000A2F800C0DAE7236DB4F85C2033B131497D
:1072E00031489847012822D0022838D0B4F85C30C1
:1072F000B4F858209A4232D90133A4F85C3094F89B
:10730000A830C3B9A36E94F8622003EB4203A366CE
:1073100094F86210A06E03F069F8244B98420AD0EA
:107320006FF004031E48636306F028FA03E094F844
:10733000A830002BECD0E36C1BB9BDE8F840FFF798
:1073400057BFBFF35B8F55E8003F5A1E45E8002149
:107350000029F8D1BFF35B8F012BEEDCF8BDE36CA5
:10736000002B3FF478AF94F8A830002B7FF473AF74
:107370000F4807F0C4FF6EE7022B0AD103F07CF838
:107380000A4B9842EAD004486FF0040343631C3070
:1073900062E7052BE2D15EE7F805002000700040AF
:1073A00014060020300600200CF700000000AD0B92
:1073B00068060020094BBFF35B8F53E8002F511C78
:1073C00043E800100028F8D1BFF35B8F0AB9FFF73C
:1073D0000FBF6FF00F025A63704700BFF80500201F
:1073E00008B50D490D48002207F07DFF002002F08E
:1073F0000BFF0B4B98420CD1002201210720FAF71A
:1074000039F80848C36813B9043006F0B7F900200A
:1074100008BD6FF00400FBE7B573000068060020AC
:107420000000AD0BF80500202DE9FF410E464FF09E
:10743000FF3376484FF0FF3204F014F977687B1E73
:10744000FE2B08D96FF01504704806F097F9204616
:1074500004B0BDE8F08100252C4627FA05F3DA07D1
:1074600006D502F02BFFE840C307EBD50134E4B2A8
:107470000135082DF1D1002CE4D0337C083B062BDC
:10748000E0D801A252F823F0C37400004574000054
:10749000C774000045740000A57400004574000026
:1074A000CB7400000221012C727C10D0002AC9D1BB
:1074B000574B002083F8A800564B384602F004FFD3
:1074C0002CE00021EFE70121EDE70321EBE7082A9B
:1074D000B8D8DFE802F00505050505050505050036
:1074E0003368002BE4D05D68002DE1D118680138C5
:1074F0007F28DDD88DF808208DF809501B68444A94
:107500001B01013BADF80A30012382F8A8308DF849
:107510000C3002AA3F4B384602F00EFF3E4B984219
:1075200090D13268630012B1928902FB0333F26892
:107530009A4268D3364D85F8624095F8A830B06815
:10754000A8662F46002B4DD033689C890134A1B228
:1075500002F04CFF304B984280467FF473AFB44644
:10756000BCE80F002D4C0FC4DCF8003023604FF056
:10757000000CC5F834C03368002B41D00FCB261D5A
:1075800086E80F00EB6CAE63A5F85CC0C3B3BFF335
:107590005B8F57E8003F47E800C2002AF9D1BFF3EC
:1075A0005B8F95F8A810F9B9E86C1D4E1D4A4FF491
:1075B0000047E0FB076100233046F8F7E1FD0022B9
:1075C000CDE90001002304F1280005F045F8164834
:1075D0004FF0FF324FF0FF3304F044F800B168631E
:1075E0006C6B31E72146B3E702F046FF4045EED031
:1075F0006FF00403A4F12C006B6306F0BFF8E6E71C
:10760000FFF7F6FDE3E76FF00B041DE7FC05002034
:10761000F8050020317200000000AD0B300600209C
:107620003F420F0040420F0014060020084B70B587
:10763000C31A0D4607499B10044659430648402289
:1076400006F0A7F82B4601462046BDE870401847D3
:1076500018170020B76DDBB62CF6000073B50C4C84
:107660000C4A4023041B00930D460B460A49A41004
:1076700061430646094806F0B8F8011E05DA3046AF
:107680002B4602B0BDE87040184702B070BD00BF85
:107690001817002055D80000B76DDBB62CF6000097
:1076A00010B5EFF31184202383F31288BFF36F8F9B
:1076B000074A136823F00201DB07116002D401209E
:1076C00007F055F984F31188BFF36F8F10BD00BF29
:1076D00068170020002270B5012104461046F9F712
:1076E000C9FE0F4801F090FF0E4B984215D101F0F2
:1076F0009BFF26690C49304605F0B0FC00280BDBE7
:10770000012535642469084904F11C0005F0A6FC34
:10771000002801DBE564002070BD6FF00400FBE78A
:10772000517800000000AD0BFCFC00007FB500228A
:107730000123CDE9022304ABCDE90433094ACDF896
:1077400000D06B46CDF804D006F07DF8002805DBAC
:107750004FF480420023684603F084FF07B05DF8D1
:1077600004FB00BF6DD8000010B5074C23782BB97F
:107770004FF4A57007F018FA01232370BDE81040FC
:10778000002001F063BF00BF641A002030B4104B2A
:107790000C2202FB003301460020D3E90E5298630D
:1077A000EFF31180202484F31288BFF36F8F1C6CD9
:1077B00004F0C00444F002041C6480F31188BFF399
:1077C0006F8F1DB12B46034830BC184730BC704743
:1077D000181700202CF6000010B4EFF311822023BC
:1077E00083F31288BFF36F8F1748016841F00204DA
:1077F0000460C80707D482F31188BFF36F8F01209C
:1078000010BC01F023BF4FF08041D1F80C04D1F837
:107810000C14C907EFD5EFF3118083F31288BFF37F
:107820006F8F0A490B6C03F0C00343F002030B6433
:1078300080F31188BFF36F8F82F31188BFF36F8FCE
:10784000002010BCFFF7A2BF681700201817002007
:1078500010B1012804D07047034B1B6C5B0701D1AA
:10786000FFF794BF704700BF18170020024AC3B249
:107870001C2003FB0020704718170020094BBFF3A2
:107880005B8F53E8002F42F0010143E8001000280D
:10789000F7D1BFF35B8F930702D4012001F0D6BE6E
:1078A000704700BF6817002010B5EFF31184202344
:1078B00083F31288BFF36F8F074A136823F0010127
:1078C0009B07116002D4012007F051F884F311885E
:1078D000BFF36F8F10BD00BF681700202DE9F04186
:1078E0003849BFF35B8F0746012251E8003F41E86A
:1078F00000200028F9D1BFF35B8F33B932493348F8
:107900004B60CB608A6005F0BCFB7B1E012B2BD843
:10791000012F07D14FF08043D3F81C3403F0030349
:10792000012B21D007F05BFB0546F8B9284B1B78EB
:10793000E3B14FF080430222C3F808230646DFF884
:1079400094804FF08044D4F81824D4F81834D2032B
:1079500015D503F00303012B01D0012F0FD155B32F
:1079600086F31188BFF36F8FBDE8F081EFF31186C6
:10797000202383F31288BFF36F8F0125DFE7ADB1BA
:10798000304605F0E5FCD4F81835002BDBD1D4F8EF
:107990000421002AD7D0C4F80431D4F804310123DB
:1079A000C4F81835C8F88031A360CCE70021212045
:1079B00007F0CBFBE7E74FF080430222C3F8042334
:1079C000D2E700BF1417002004170020341700204E
:1079D000871A002000E100E008B5074807F000F929
:1079E00038B10648F9F75AFF0448F9F7C1F8002002
:1079F00008BD6FF01200FBE78CF60000017A000072
:107A00000A2838B5074D044604D1AB680D215B68E0
:107A100028469847AB6803485B68E1B29847204620
:107A200038BD00BF8CF60000EFF31182202383F3F2
:107A30001288BFF36F8F0A4BD3F8001161B1002198
:107A4000D3F80805C3F80011D3F80031C0B282F3AF
:107A50001188BFF36F8F70476FF00A00F7E700BF20
:107A600000D00040F0B5034610469C7893F803C060
:107A7000EFF31182202585F31288BFF36F8F1F78F3
:107A800093F801E0E41B04EA0C04A04288BFA0B212
:107A90003E180CEA06063D461E7082F31188BFF3BD
:107AA0006F8F0A188A4216D177450CD1EFF31182F5
:107AB000202181F31288BFF36F8F1978597082F3F8
:107AC0001188BFF36F8F1B79241AA34222BF064B84
:107AD00001221A60F0BD5E190135767901F8016B5B
:107AE00005EA0C05DEE700BF00D00040DB432DE9CE
:107AF000F04713F001050E46144604D02248FFF764
:107B0000B1FFBDE8F0879AB3EFF31188202383F328
:107B10001288BFF36F8F0D20F9F79EFC07460D20EA
:107B2000F9F786FC88F31188BFF36F8FDFF85CA04C
:107B3000DFF85C80CAF80051DAF800314FF40059E0
:107B40000123CAF800302546C8F88091DAF80031E0
:107B500083B1FFF769FF031EC8F88091F6DB013D92
:107B6000ADB27355002DF1D117B10D20F9F752FCCC
:107B70002046C6E7EFF31180202383F31288BFF37A
:107B80006F8F05F0E5FBE1E79C17002000D0004077
:107B900000E100E02DE9F041124F0D46144607F1D7
:107BA000450814B92046BDE8F0814FF0FF334FF08F
:107BB000FF32384603F056FD224629464046FFF77D
:107BC00051FF0646384603F013FD3EB94FF0FF3231
:107BD0004FF0FF33044803F045FDE6E7A41BA4B2D1
:107BE0003544DEE76C1700208417002038B5194CA7
:107BF00001221146204607F028F90122002104F154
:107C0000180007F022F940F20743A4F848304FF07B
:107C1000706323630C2384F8343000250E4B84F802
:107C20004550A4F84650D3F8042542F00102C3F8A9
:107C300004250121C3F80051D3F80021C3F804132F
:107C40002A4619600D20F9F715FC0D20F9F7E2FB23
:107C5000284638BD6C17002000D0004010B5FFF753
:107C6000E3FE002820DB174B93F8322093F83140D5
:107C700093F83310141B31EA0404C0B20DD193F809
:107C8000472093F8464093F84810141B31EA040447
:107C90000BD10D4B01225A600EE09C1801321140AD
:107CA00084F8350083F8321010BD9C180132114061
:107CB00084F84A0083F847100448BDE8104003F0F8
:107CC00097BC00BF6C17002000D000408417002034
:107CD000430970B507D10B4B596821B101250C68D8
:107CE000094E854001B970BD8A682A4002D04B68B0
:107CF000304698471CB1236821461C46F2E72346CC
:107D0000FAE700BFC01700204CF600002DE9F04351
:107D1000476840F20636D0063B7B87B002EA06068B
:107D200054BFC2F34010032001F01F05B6F5837F56
:107D3000144645EA43158DF8030043D00FD8062EAC
:107D400018D007D8B6B1022E3ED06FF0150007B09C
:107D5000BDE8F083B6F5807FF7D101260AE040F256
:107D60000222964232D0B6F5407F31D0B6F5007F80
:107D7000EBD102260123220303FA01F12AD57B6805
:107D8000C3F808153B695BBB05F01F026D0974D190
:107D9000920002F1A04284F48031D2F80037C1F39E
:107DA0000041C4F3404423F4E16344EA410423F076
:107DB00007031C4344EA800444EA0624C2F800474F
:107DC0000020C4E70726D5E70426D3E70526D1E738
:107DD0000326CFE7630344BF7B68C3F80C15D1E7E4
:107DE00010370DF102022946384601F0E3FE14F483
:107DF000403F80460CD12946384606F02AFE214BEA
:107E00009845DDD19DF80210384601F013FFD7E701
:107E100001AB4FF0000903AA29463846CDE90439E1
:107E2000CDE90199CDF80C9001F094FD154B9842E5
:107E30008BD114F4003315D09DF803308DF80E303B
:107E400084F48034C4F300444B4603AA29463846E0
:107E50008DF80C608DF80D4001F030FE094B984212
:107E6000CDD072E7CDE9043303AA0DF1030329460F
:107E70003846039301F06EFDF0E702F5E07253F827
:107E80002230FFDE0000AD0B38B545682B69B3B179
:107E90001035284601F0C4FE044680B90146284644
:107EA00001F09AFE084B98420BD108492246284619
:107EB00001F07AFE224605210620F9F7DBFA0020C0
:107EC00038BD6FF00400FBE70000AD0BD17C000073
:107ED000F0B516464268107B01F01F0444EA4014D6
:107EE000106987B000286ED0B6F5001F02F11005AA
:107EF00006D12146284606F0AEFD002007B0F0BDB1
:107F000001A80027B6F5800F0197476038D1B3F17B
:107F1000007F14BF052304238DF804300023CDE92E
:107F200004030393936823FA01F111F001010DF1A9
:107F300003073AD1B6F1A07F37D104F01F036209DD
:107F400003F5E07345D14FF0A04252F82330DB0730
:107F50002BD43A462146284601F02CFE1E4B98426F
:107F600019D0029703AA2146284601F0F3FC1B4BC7
:107F700098422BD101222146284601F06BFEBCE736
:107F8000B3F1C06F05D0B3F1007F14BF012302230A
:107F9000C2E70323C0E73946284601F053FE0F4BE2
:107FA0009842DED06FF00B00A8E73A4621462846FB
:107FB00001F000FE094B9842D4D19DF803102846E9
:107FC00001F038FECEE76FF0850097E76FF01500FF
:107FD00094E751F82330FFDE0400AD0B0000AD0B39
:107FE00002780B69012A08D0022A08D04AB9064A49
:107FF0001A6303F1180003F0FBBA044AF8E7044AD5
:10800000F6E7044AF4E700BF0000AD0B0100AE0B39
:108010000200AE0B0100AD0B2DE9F04F87B0D0F898
:1080200010B004934368D3F828809B8B03931746C2
:108030004FF0FF334FF0FF3205460C4605F05FFE70
:108040000BF118030293002300220BF11800002605
:1080500003F008FB3346BE4201D300234DE0207AF3
:10806000010776D40136BE4221680BD2820709D4BB
:10807000227D80EA020C0CF0010C02F004025CEAA2
:10808000020C08D023B901F06042B2F1005F1AD0AF
:108090004FF0000901E04FF001096268DDF80CE0E3
:1080A00003EB020CF44557D8C00705D408EB0300D6
:1080B000059307F0A9F9059B62681A4493B2B9F1D8
:1080C000000F2FD113BBD4F800A0A3884FF00009F4
:1080D000049A217A00922846524600F063F8031E63
:1080E0000BDB4FF480420298002303F0BBFA80B10F
:1080F000284600F037F86FF004032846029305F095
:1081000001FE029B184607B0BDE8F08F9946C246B3
:10811000DEE7DBF83030124A9342ECD1237ADB07FA
:1081200002D400230C3496E7C245FAD1A24609E0F6
:10813000A9EB02011FFA81F9DAF80C0018FA81F1B3
:1081400007F062F9DAF804209145AAF10C0AEFD29F
:10815000E7E76FF08503D0E76FF01B03CDE700BFC3
:108160000000AD0B70B544682368D3F80855D3F808
:108170000C65204602F004FD3146284602F03EFF21
:1081800000210546606A05F0C0FD204602F0E8FCCB
:10819000034B9D4214BF6FF00F00002070BD00BF65
:1081A0000000AD0BF0B587B047680C4616460021BD
:1081B00012220DF106001D4607F04EF904F00103EE
:1081C0008DF80430BDF830308DF80530BB8D029548
:1081D000AB42049614D384F00202C2F3400252016F
:1081E00001A9384602F036FD084B98420BD00B33FC
:1081F000984214BF6FF004006FF00F0007B0F0BD9D
:108200006FF01B00FAE70020F8E700BF0000AD0B9D
:1082100038B545682B6A04469847686A012105F01D
:1082200074FD2346AA6905F10801284602F05CFCAA
:10823000054B984204D1204605F08DFD002038BD45
:108240006FF00400FBE700BF0000AD0B2DE9F04725
:10825000DFF808C1424F002540F2FF16EBB2994209
:1082600002D80020BDE8F08750F8254014F4804F74
:10827000C4F3C32EC4F3080360D1240E17F80E9084
:10828000B34208BF4FF0FF330C2C5AD8DFE804F09C
:10829000070D1417595959595959591A4800C2F814
:1082A0000C355C1C3FD10135D8E7C2F814355C1C95
:1082B000F9D04FF0000810E0C2F80835F1E7C2F835
:1082C0001035F4E7C2F80835B9F1000FEFD15C1CA6
:1082D000E9D04FF000084FF0060950F825A00AF445
:1082E0000044002C16BF4FF00008C6464FF0010EA8
:1082F00003F01F045B092BD1A40004F1A044CAF3CE
:10830000412AD4F8003703EA0C0343EA8A0343EA1C
:10831000092343EA080343EA4E03C4F80037C2E7DF
:10832000C2F80C35D0E75C090ED14FF001084FF0D0
:10833000A04408FA03FEC4F808E5CEE76FF0150084
:1083400090E76FF085008DE70023C3F80835FFDE66
:1083500004F5E074002353F82430F8E7F0F8FCFF4C
:10836000A305010038B570B1074C084A4FF4004529
:108370000021E0FB054100232046F7F701FFBDE89F
:10838000384006F0E2BE38BD3F420F0040420F00C9
:108390001C39036907291DD8DFE801F0041C0A1CF9
:1083A0001C0C1C1819880023C2E900130020704718
:1083B0005988F8E79B88094840F24C61C3F30903E8
:1083C0004B43B3FBF0F100FB1133EDE79B88002139
:1083D0009B0AE9E76FF08500704700BF40420F003D
:1083E000F0B54468066985B00546206806F0F8FBDC
:1083F00020B96FF01204204605B0F0BDA06988B125
:1084000004F1180706F0ECFB0028F2D04FF4B0118D
:10841000384605F060FE6868012105F0E2FE0120A3
:1084200005F073FE206968B104F1100706F0D8FB6F
:108430000028DED038464FF4D01105F04CFE012064
:1084400005F063FEA06898B9142005F05EFE23696C
:108450009BB9A38843492068052205F066FE0028E1
:1084600018DA6FF004046868002105F0BAFEC2E76C
:1084700006F0B6FB0028E7D1BBE704F110070121A5
:10848000384605F014FE0F2006F08EFB002138461A
:1084900005F00DFE022005F038FE6F68384605F045
:1084A00073FE0028DDDBC10602D46FF01504DAE7A5
:1084B000020640D520232068A1888DF80E300123C4
:1084C00000930DF10E020DF10B0305F041FE0028A3
:1084D000C7DB9DF80B30812BE7D10227A1880097DD
:1084E00024238DF80A3020680DF10E030DF10A02E5
:1084F00005F02EFE0028B4DBBDF80E305BBAADF8F7
:108500000E30C3F30723737241F20103ADF80C3050
:108510002068A3883A4603A905F007FE0028A0DBDF
:1085200010233372686805F02FFE041E99DB14F0E7
:10853000010498D0B9E7F4238DF80E30BB88386871
:1085400001220DF10E0105F0F0FD002889DB01206C
:1085500005F0DBFD686805F017FE002881DB0306E7
:10856000A8D4A2E7C505010037B505230093002371
:1085700045688DF804300446002A3CD0D2E9000357
:1085800003F574331E4A903393FBF2F303EB40037D
:10859000C82BA8BFC82323EAE373DBB28DF80130F0
:1085A00059B30B685A004B681549002BB5BF03F54A
:1085B0007433A3F574339033903B93FBF1F313447E
:1085C0006FF031029342B8BF13463233DBB2284614
:1085D00001218DF8033005F004FEAB8828680522E0
:1085E000694605F0A2FD00210546606805F0F9FD29
:1085F000284603B030BD6423D0E76423E7E700BF1B
:1086000020A10700014B01221A60704700C0004002
:108610000C2903690BD1DB6A064907484B4393FBDE
:10862000F0F100FB113311605360002070476FF0D0
:108630008500704790D0030040420F00044B006952
:108640000022C3F80021D3F8003102F0D1BF00BFEF
:1086500000C000407FB505692B6B63B3422901D090
:108660000C292BD105F118064FF0FF324FF0FF33E4
:10867000304602F0C3FE134B0193286B0323002402
:1086800069460394029304F0FCFC4FF0FF324FF074
:10869000FF33284602F0E6FF286B04F049FD0A4B41
:1086A000D3F80825EA6201225A60304602F01EFF24
:1086B000204604B070BD6FF00A00FAE76FF0850045
:1086C000F7E700BF0586000000C0004010B5046950
:1086D0000020FFF7CBF820634FF0FF320021204647
:1086E00006F0B3FB04F1180006F0C7FA00220121DE
:1086F0000C20F8F7BFFE0C20F8F78CFE024B01228D
:10870000C3F80423002010BD00C0004030B50D297F
:10871000006920D1C488B0F90E500389B0F9021065
:108720001B1B491B4B43B0F91010491B93FBF1F382
:108730002344002B1946B8BFD91D584200F007004A
:1087400003F0070358BF43421248C9104343C2E92C
:108750000013002030BD102919D10479B0F90A5056
:108760004379B0F900101B1B491B4B43B0F90C10A7
:108770000948491B93FBF1F3234403EBD371002B0E
:1087800003F001034FEA6101B8BF5B42DEE76FF01F
:108790008500DFE748E8010020A1070030B4034668
:1087A0000029DA8B8069197F0CBF4FF400144FF059
:1087B000B86402F040022243836805699C697CB179
:1087C000130206D52D6801238B402B4218BF82F07F
:1087D000C062044BA446134030BC02F0B072604744
:1087E00030BC704740000006F8B544680546A069F3
:1087F00000283ED02E6906F0F3F900283BD07561C1
:10880000E38BA069217F43F48032D0F810C0D0F808
:1088100008E0DCF8007013F0010F4FF0010303FAD9
:1088200001F314BF3B4327EA0303CCF80030DEF822
:108830000030984700281DDB237F124A012707FAE2
:1088400003F3C6E90723A0698368DB6906F1180111
:10885000A3B13A46984700280CDB3946204604F07D
:1088600036FD002806DB084B336368683946FFF79E
:1088700095FF0020F8BD6FF01200FBE76FF0570086
:10888000F8E700BF11E400002DE4000070B50329F3
:1088900004691CD80F4B58560F4B5E560F49B04217
:1088A00002F1080201DD002070BD031D04EB43034B
:1088B0002569B3F901301B116B4393FBF1F501FB03
:1088C000153342F8085C42F8043C0130E7E76FF0EA
:1088D0008500E9E7F0050100EC05010040420F00CA
:1088E000F0B504460569466885B00021A42006F06D
:1088F0002CFC6B680DF107029B680F2120469847FE
:10890000002825DB9DF80730332B40D1327BD70779
:108910000BD5204B44F6161142F28B40C3E90001FF
:108920001D4949F22D26C3E90261930712D400269E
:10893000CDF809608DF80D6007238DF808306B685D
:1089400002AA5F68202106232046B84700280BDAD8
:1089500005B0F0BD6B681E6980231A461E212046B3
:10896000B0470028E3DAF3E70A4B1B682B616B681A
:108970003246DB682321204698470028E8DB6B68F5
:1089800047222A75DB68202120469847E0E76FF0F0
:108990001500DDE7D007002094B6010010B543684C
:1089A0000469586806F01CF918B1034B6360002095
:1089B00010BD6FF01200FBE7ACFE000030B50E29D1
:1089C000036911D11968114C0B130A25C1F30B016E
:1089D00093FBF5F005FB10336143634303EB113365
:1089E000C2E90003002030BD0D290CD1B3F90430D9
:1089F000642493FBF4F104FB113308B242F21071CA
:108A000013FB01F3ECE76FF08500ECE7A0860100B3
:108A1000F7B5212946680369154654D1B27A1B8CF3
:108A200012F02001727918BF1BB2002A4BD0F279E4
:108A3000377C042A09BF3268F2899268128909B129
:108A4000013FFFB2B07983FB02326946CDE90032C3
:108A5000FEF7DEFA044698BB019A009BC7F120009E
:108A6000B7F1200102FA00F023FA07F343EA00030A
:108A70005CBF42FA01F10B433A41CDE9003213F1F8
:108A8000004342F1000212B1104804F070FA776915
:108A900000984FB14FEAE07CA0FB0701B2690023C8
:108AA00007FB0C11F7F71CFB4FF47A7390FBF3F202
:108AB0002A60074A434393FBF2F102FB11336B60D8
:108AC000204603B0F0BD6FF08504F9E71106010000
:108AD00040420F00F7B500234568046907460022AD
:108AE000684606F0BAFBDDE90023C4E906232868DE
:108AF00006F076F820B96FF01206304603B0F0BDEC
:108B0000E869002845D1284605F07BFE0646002886
:108B1000F3D16B79002B64D02A79012393406360F1
:108B20002B7C23746B7C637404F12003A360022309
:108B3000E36095F8283083F00103A3747B68D8695B
:108B400000282BD17C68E0690028D6D094F820302A
:108B50003D690121994003691B681942836814BF6C
:108B60001B69DB689847676A1F4C204A4FF4004036
:108B70000021E7FB004100232046F7F701FB0246F6
:108B80000B46684606F069FBDDE90023C5E90623CC
:108B9000B3E706F025F80028B5D1ACE793F820102C
:108BA0005B8CD0F810C0D0F808E0DCF80040DA07A1
:108BB00054BF43F4B01383F4D013012523F480127F
:108BC0008D40DB074CBF2C43AC43CCF80040DEF8B3
:108BD000003098470028B5DA10F1860FB2D006466B
:108BE0008BE76FF0850688E73F420F0040420F0099
:108BF0002DE9F041044647680D4606F0F0F988B1CA
:108C00004FF02008EFF31186314688F31288BFF346
:108C10006F8F606805F03AFE50BB86F31188BFF392
:108C20006F8FEFE71F4B1B78002BE9D04FF0200828
:108C30006426606805F02AFE70B9012005F084FE04
:108C4000013EF6D10021212006F07FFAF0E786F3FD
:108C50001188BFF36F8FF5E7EFF31186314688F384
:108C60001288BFF36F8F606805F010FE0028EED009
:108C7000BB691D706368BA691B680020C3F844258E
:108C80000122C3F84825C3F82001D3F82041C3F8D6
:108C90005801D3F858019A6081F31188BFF36F8FA0
:108CA000BDE8F081871A0020F8B5002205460121B1
:108CB0000220F8F7DFFB0220F8F7ACFB6C6801211B
:108CC000E06805F014FE6B681A682369C2F8243561
:108CD000637D217D0B43C2F86C356E68D6E9004395
:108CE00013F001033CD02F6907F1080005F03DFEA9
:108CF0002A4B98424ED1387A04F10C0204F5907157
:108D000005F029FE387A012707FA00F000F014FC7C
:108D10000823C4F80035B369C4F844350023C4F807
:108D20004835A760D4F85831002BFBD00021C4F897
:108D300000156D682C68E86805F0D9FD0823C4F8B3
:108D400000352A7A52B9EB69C4F834350123C4F8E6
:108D50003835C4F81021D4F8102123600020F8BD64
:108D60000822C4F80025B269C4F84425C4F848357F
:108D70000123A360D4F82031002BFBD00023C4F8DA
:108D80002031D4F820310123E3604FF48073C4F81C
:108D90000433C7E76FF00400E1E700BF0000AD0B4C
:108DA00070B5012383400E4ABFF35B8FDC4352E86A
:108DB000001F01EA040542E80056002EF7D1BFF378
:108DC0005B8F4FF4803282400648C0F80823BFF31F
:108DD0005F8FBFF36F8F0B4214BF0120002070BD67
:108DE000081900200010014070B40E49D1E9003488
:108DF000D01AC31844F10004C2F30E06C1E90034CE
:108E0000A6F58053B3F5C04F09D2074B1B685A0C27
:108E1000DB039C19054B42F10005C3E9004570BC1A
:108E200003F020BBC00A00200C190020C80A002053
:108E300011B3BFF35B8F0123104A834052E800CF88
:108E40004CEA030C42E800C10029F7D1BFF35B8F65
:108E50000B4A4FF480338340C2F80433094BBFF30D
:108E60005B8F1B68BFF35B8FC340DB0742BF064BC2
:108E70004FF40032C3F80021704700BF08190020EA
:108E8000001001400019002000E100E030B5144B53
:108E90001868410CC003BFF35F8F124BD3F8043541
:108EA00047F6FF7293420AD10F4AD2E90045844245
:108EB00075EB010209D3C01841F1000130BD18184B
:108EC00041F10001B3F5006FF8D2074BD3E900235D
:108ED000904271EB0303F1D210F50040ECE700BFC4
:108EE0000C19002000100140C80A00202DE9F04FA5
:108EF00085B016461F469DF840A00446FFF750FF78
:108F00000190FFF7C3FFB04271EB07035CD2301A48
:108F100044F2010367EB0101984271F1000156D25E
:108F20003D4B03EB0413D3E902239F4208BF964253
:108F300065D03A494FF4803804F1500508FA04F836
:108F4000AD002046C1F84883ADB205F0E2FCC6F39F
:108F50000E0B05F1804504F5A87305F588355846D4
:108F60004FF003090293C0F30E03002B029A08BFCF
:108F70000120C0F30E0341F82230C1F84483D1F838
:108F800004356FF0020CACEB030C6044C0F30E0030
:108F900043F6FD72904232D9286868B1D1F80435A1
:108FA0000393A3EB0B00C0F30E00B0F5804F26D95E
:108FB000204605F0AEFC039BBAF1000F07D109EB88
:108FC000030009F10109CEE7BAF1000F09D06FF0F3
:108FD000150520460199FFF72BFF284605B0BDE88F
:108FE000F08F01230E4ABFF35B8FA34052E8000FBE
:108FF000184342E800010029F8D1BFF35B8F06490E
:109000000E98230101EB0412C8500F9B5360C2E974
:1090100002670025DDE700BFA00A00200010014024
:109020000019002070B52D4C2D4BC4F80833C4F83E
:1090300048332C4B2C4A00254FF0FF304FF0FF31C6
:109040004FF48036C4F80855C3E90201C4F804633C
:10905000C3E906014FF4003386B00121C4F804339C
:109060001120C2F880312A46F8F704FA1120F8F7E7
:10907000D1F91E4B01200322A06020601A601C4B16
:10908000009343F6FF720023CDE90155FFF72EFF51
:109090000220FEF723FC174A136823F00103136034
:1090A00047F6FF73C4F844630DF11700C4F8403568
:1090B00000F0C4FE104B98420CD1104A10499DF8A4
:1090C000170000F0C1FE9DF8170000F0EBFE2846E7
:1090D00006B070BD6FF01200FAE700BF001001404B
:1090E00001000F00A00A002000E100E008190020A4
:1090F000E98D0000041900200000AD0B08100140AC
:10910000401101402DE9F743374CD4F80433D9031B
:1091100019D540230022990810290CD1D4F84031E8
:10912000002B41D00023C4F84031D4F840314FF433
:1091300080324423EFE70433502BECD11AB12B4A91
:10914000136801331360D4F804339A0329D5BFF3AD
:109150005B8F274B53E8002F22F0020143E80010F9
:109160000028F7D1BFF35B8F930702D4D4F84431C2
:10917000BBB10025C4F84451D4F84431FFF786FE52
:10918000EFF31182202383F31288BFF36F8F194B03
:10919000D3E90667B042B94108D282F31188BFF320
:1091A0006F8F03B0BDE8F0834423B4E74FF0FF387E
:1091B0004FF0FF39C3E90689D3E904101D614FF46C
:1091C0000033C4F84833C4F84451D4F8443182F32E
:1091D0001188BFF36F8F0029E3D0009032463B46E1
:1091E00001208847DDE700BF001001400C19002076
:1091F00000190020A00A002030B5431C85B043F6BA
:10920000FF7223D09042A8BF104601280446B8BF81
:109210000124FFF73BFE0F4BD3E90013401AB0F5D2
:10922000804F43F6FF7513D22218AA4228BF2A4660
:1092300052184FF0000008490091CDE9010043F1B8
:1092400000030120FFF752FE05B030BD1446E0E7F1
:109250002A46EDE7C00A0020E98D000008B5FFF7B7
:1092600015FE024B1B68C01A08BD00BFC00A0020D3
:109270004FF0704393F8E02F062A09D1D3F8E83F66
:10928000C3F30313033B042B02D8024AD05C70479C
:10929000002070475806010008B505F046FB40B1B4
:1092A0004FF08053784AD3F82433C3F30423C2F831
:1092B0004035FFF7DDFF10B1744B754A5A6705F072
:1092C00034FB48B14FF080534FF08042D3F8443222
:1092D000C3F34233C2F83C35FFF7CAFF30B16D4AE1
:1092E000D2F8FC3023F08073C2F8FC3005F01DFB8F
:1092F00040B14FF080430022C3F80C21C3F8102185
:10930000C3F83825FFF7B4FF20B14FF080430322A4
:10931000C3F8A025FFF7ACFF60B15F4B0522C3F88F
:1093200010260122C3F888260022C3F818263F22FF
:10933000C3F814264FF08053D3F83021511C09BFD5
:109340004FF07043D3F8343193F8E02FD3F8E83F6F
:1093500008BFC3F30313062A4DD1033B042B03D8E4
:109360004E4AD35C002B46D04FF080524C4BD2F883
:109370000414C3F82015D2F80814C3F82415D2F841
:109380000C14C3F82815D2F81014C3F82C15D2F811
:109390001414C3F83015D2F81814C3F83415D2F8E1
:1093A0001C14C3F84015D2F82014C3F84415D2F8A1
:1093B0002414C3F84815D2F82814C3F84C15D2F871
:1093C0002C14C3F85015D2F83014C3F85415D2F841
:1093D0003414C3F86015D2F83814C3F86415D2F801
:1093E0003C14C3F86815D2F84014C3F86C15D2F8D1
:1093F0004424C3F8702505F098FA48B14FF0805323
:109400004FF08042D3F8583203F04F03C2F8E43EE5
:1094100005F08BFA48B14FF08043D3F80024D2070F
:1094200044BF6FF00102C3F800244FF08053D3F81B
:109430003021062A26D1D3F83431033B042B02D83D
:10944000184AD35C63B1184AD2F83C3743F48063BE
:10945000C2F83C374FF08053D3F83031062B11D18E
:109460004FF08053D3F83431033B042B02D80F4A1A
:10947000D35C3BB14FF01023D3F808224FF0804368
:10948000C3F8582508BD00BF0030014000C00740A8
:109490000DF0ADBA00ED00E00050004053060100B1
:1094A00000C000404E0601000010004049060100C7
:1094B00030B50468CCB1BFF35B8FB4FA84F3C3F169
:1094C0001F03DBB201229A4024EA020250E8005F47
:1094D000A54204D140E8002CBCF1000FF6D1BFF347
:1094E0005B8FE6D102480B7030BD0248FCE700BF3D
:1094F0000000AD0B0200AD0B10B50368CB40DB07DD
:1095000014D401238B400268BFF35B8F43EA02014E
:1095100050E8004F944204D140E8001CBCF1000F19
:10952000F6D1BFF35B8FEED1014810BD0148FCE7D7
:109530000000AD0B0400AD0B014BC3F804057047F0
:1095400000F00140F7B50546F8B101281BD104220F
:109550004FF4807301464FF0804003440244C0F84A
:1095600008130026012111601E608D421B688DF8D2
:10957000071008BF0DF1070642F210744FF0804744
:1095800045B1012D29D003B0F0BD0C224FF48273F8
:109590000221E0E7D7F8183403F4803366B9002BD2
:1095A000F1D0012005F0D0F9013CF3D1EBE705F053
:1095B000CBF9013CE4D1E6E7D7F8182402F0030226
:1095C0003260002BDFD09DF807000128EFD0012D7D
:1095D000D9D10C4B00225A71D5E7D7F80C3403F4DB
:1095E00080333EB9002BF4D0012005F0ADF9013CE9
:1095F000F3D1C8E7D7F80C2402F001023270002B37
:10960000E1D1E6E710190020044B1A7922B90122B2
:1096100018609A800248704702487047101900206D
:109620000000AD0B0C00AD0B08B5074B1B682BB150
:109630000020F7F711FF08B9F7F7ECFE4FF0804371
:109640000022C3F8182508BD1019002038B5B0B1A4
:10965000012855D14FF080420023C2F80031D2F8E2
:109660000021304A03F18043012119602E4B1B6811
:10967000002B50D04FF08043C3F8040340E04FF07C
:109680008043D3F81814D3F81824C8032AD502F05D
:109690000303012B04D013B10020FFF753FF002375
:1096A0004FF08042C2F818350023C2F80431D2F8D6
:1096B00004311E4AD2F8FC0040F08073C2F8FC303E
:1096C0001B4B1C6844F0010119605D685968491B17
:1096D000B1F50A5FFAD31C60C2F8FC000823154AF2
:1096E0000220BFE7D3F81424D107D8D5D3F81C241F
:1096F0009207D1D40C4A12681AB10222C3F804238B
:1097000038BDD3F80421002AFBD00022C3F804217D
:10971000D3F80431F4E71368002BFCD00023136066
:109720001368EDE7000100401019002000ED00E093
:10973000001000E004010040F8B54FF080431C4EDB
:10974000D3F804430125002704B9F8BDB4FA84F026
:10975000C0F11F00830003F580739BB203F18043C7
:1097600005FA00F21968D2B224EA02040029EBD00B
:109770001F601B684FF08043012AC3F8082305D0FF
:10978000022A08D03368C0B29847DDE77379002B0E
:10979000DAD17271F6E7D3F81814D3F818148907E0
:1097A000F0D1C3F81855C3F804239D60CCE700BF7F
:1097B0001019002070B5C3B20C4C0833054634F8BC
:1097C0001330DA050E4607D5C3F3432304EBC30277
:1097D00054F8333052689847A3682BB1E268314699
:1097E0002846BDE87040184770BD00BF181900201A
:1097F00010B4C0B2114A083032F81030D9051BD568
:10980000C3F3432123F4F85322F8103002F10E047D
:10981000002034F8023F13F4807F03D0C3F34323C6
:10982000994209D001302028F3D1002342F8313089
:10983000034810BCFFF760BE10BC70471819002029
:109840007019002001F18051F0B501F5C2510446B4
:10985000114A00208900012506468A420BD10F4B90
:10986000D3F87C2132B10022C3F87C21D3F87C31BB
:1098700040F00040F0BD02F14043A3F5C2439B0815
:1098800005FA03F31C4204D0176817B11660176875
:1098900018430432E1E700BF00610040006000406F
:1098A000CBB20246083308460C4931F8133099060A
:1098B00011D599070FD410685B0B01219940C0F8AE
:1098C0000813126802EB8303D3F8102522F0030279
:1098D000C3F810257047002105F09EB81819002024
:1098E000F7B5CDB2174E0835074636F81530DB0709
:1098F0000C4624D5FFF7D4FF36F815309A0606D566
:109900005B0B3A6803F5A273002142F8231020464E
:10991000FFF76EFF002301A826F81530019405F02B
:1099200028F8019B00EB8300074BD0F80027134079
:1099300043F00203C0F80037044803B0F0BD044808
:10994000FBE700BF18190020F0F8FCFF0000AD0B8A
:109950000400AD0B2DE9FF41136807460C4616467F
:10996000FBB1CDB2DFF84481083538F8152002F09C
:109970002202222A22D00022CDE900228DF80E20D8
:109980008DF80F200DF10E010DF10F02204604F0AD
:10999000FAFF38F8153023F0020343F0010328F8EA
:1099A000153073684BB393F800C058683F4AE3B270
:1099B000083332F813108D0702D5B0B13C481FE0D0
:1099C00021F02001C904C90C22F8131068B1BCF1C0
:1099D000030FF3D87068406805783868BCF1000F51
:1099E00011D105F5A27540F825C032F8131021F009
:1099F0001C0141EA8C0122F81310B36863BB2D48A7
:109A000004B0BDE8F08100EB850041EA4531D0F8B3
:109A100010E52EF0030EC0F810E53F6807EB850750
:109A200041F02001D7F8100522F8131020F4473038
:109A300020F44070C7F810052002D7F810E500F4B4
:109A4000F85040EA0C4040EA0E00C7F8100502EB5F
:109A50004500A0F85C40C8E7D3E900672046FFF75F
:109A6000C7FE002ECBD0114DD5E90023964203D17D
:109A70009F4201D1002209E00F480DF10F01FFF7CD
:109A800017FD0C4B9842BBD19DF80F2045F8326072
:109A9000E4B205EBC20308345F6035F8143043EAE2
:109AA000422343F4807325F81430A8E718190020E6
:109AB0000400AD0B0000AD0B701900202DE9FF4133
:109AC00007460C461E4612B3CDB2DFF8D0800835EB
:109AD00038F81530980701D4990621D413F01C0FDB
:109AE00002D05378012B1BD001238DF80F300023B7
:109AF000CDE900230DF10F01931C2046013204F043
:109B000042FF38F8153043F0030328F81530002ED3
:109B100042D0E1B2214D083135F81120930703D42A
:109B20001F4804B0BDE8F08196F800E0D7F800C007
:109B300022F020020EF5A270D2040023D20C4CF8C1
:109B4000203025F8112096F801C0BCF1000F23D079
:109B50003868B67800EB8E004FEA0C4CD0F8103520
:109B600023F4981323F4F853C0F81035230203F4B8
:109B7000F8530CF4403C3605D0F8107543EA0C035A
:109B800006F4801642EA4E32334342F020023B4351
:109B900025F81120C0F810350248C2E71819002036
:109BA0000400AD0B0000AD0B014BC3E9021270477E
:109BB00018190020C9B20831044B33F81130990646
:109BC00043BF5B0B0248137002487047181900200E
:109BD0000000AD0B0400AD0B70B50E4C94F86C504A
:109BE0000646A5B94022294604F1100005F034FCD0
:109BF0003068C0F87C51D0F87C3140F30730F7F77B
:109C000009FC0123044884F86C30A36570BD034847
:109C1000FCE700BF181900200000AD0B0C00AD0BD5
:109C2000034B93F86C00003818BF0120704700BF49
:109C3000181900200079024B03EB8000FFF75CBC91
:109C4000E00700200079024B03EB8000FFF730BCF7
:109C5000E007002073B5CBB20C460833214931F838
:109C6000133001689D0619D513F0020616D15B0B5F
:109C70009C0004F580754E51495901682144D1F882
:109C8000104544F00104C1F810452AB101680122D1
:109C900002FA03F3C1F8043302B070BDD1F8042313
:109CA000002AA8BF4FF00042C3F38203A8BFC1F847
:109CB0000423042B12D0052B12D001A8019404F028
:109CC00058FE019AD0F81035D34003F00103991CD7
:109CD000204602B0BDE8704004F09EBE0321F7E7C5
:109CE0000221F5E7181900202DE9F347514BD3F86D
:109CF0000403C0B2082140F00040FFF7A3FD051E99
:109D000016DA002301216846009304F094FEDFF880
:109D100028810127009999B94FF00040FFF792FD83
:109D20000121684604F087FE0028F3D125F00045A4
:109D3000404E414F0124002D66D102B0BDE8F087AE
:109D400091FAA1F4B4FA84F4E00804F1080304F0F1
:109D5000070238F813901DF80030019407FA02F258
:109D600023EA02030DF8003001A804F002FE019B73
:109D700003F5E0734FEA990150F82360C9F3820AB2
:109D80004B07D146C6F3014623D520465146FFF77F
:109D900011FD01A8019404F0ECFD019B03F5E073B3
:109DA000F6B250F82330C3F301439E4207D100219D
:109DB000204604F031FE3146204604F02DFE01A875
:109DC000019404F0D6FD019B07FA03F3C0F8203597
:109DD000A0E7022E0CD10321204604F01DFE0AF05C
:109DE0000503012BEBD149462046FFF7E3FCE6E7EC
:109DF0000221204604F010FEBAF1030FF3D0032E27
:109E0000DDD1BAF1020FEDE795FAA5F3B3FA83F3CA
:109E100004FA03F225EA020503F5A27207EB4303F5
:109E200056F82210B3F85C00C1F30141FFF7C2FC01
:109E300081E700BF0060004018190020014601487A
:109E4000FFF736BBE407002070B5044615460E4602
:109E5000B1B1AAB10D4B01228240134093B10C4B1A
:109E60000146186804F072FD70B1E00000F1804016
:109E700000F5F830C0F81065C0F81455054870BDFD
:109E80000548FCE70548FAE70548F8E73FC00F003A
:109E9000E40700200000AD0B0900AD0B0400AD0B82
:109EA0000500AD0B10B50C4B012484402340014646
:109EB0007BB90A4B234023B9094B0A48C3F8044530
:109EC00010BD094B186804F041FD0028F4D1074883
:109ED000F6E70748F4E700BFC03FF00E3FC00F00B1
:109EE00000F001400000AD0BE40700200500AD0BC1
:109EF0000400AD0B30B50A4B082493F83050012212
:109F00000023104203D0154208D00133DBB2013CDC
:109F10004FEA4202F5D103480B7030BD0248FCE71E
:109F2000881900200000AD0B0400AD0B054B93F821
:109F30002E00431E012B03D9043818BF012070479F
:109F4000002070478819002010B5164A16490020D5
:109F5000C2F8000591F82F40D2F8043381F82E4062
:109F60000C6823F033030CB143F02303C2F81C0147
:109F7000D2F81C41C2F81801D2F81841C2F8080101
:109F8000D2F8082191F83320D00791F8342048BF47
:109F900043F08003D207034A48BF43F04003C2F8AE
:109FA000003310BD007000408819002070B50D4AC4
:109FB000002392F8301001251E4618B90BB182F823
:109FC000301070BD90FAA0F3B3FA83F305FA03F4EE
:109FD0000C3302EB430320EA0400DE8021EA040193
:109FE0000123EAE78819002073B50023044601AA7B
:109FF0000E464FF48071019304F02FFD4FF48A71E7
:10A00000204604F02AFD4FF482710546204604F0F4
:10A0100024FD20B11EB115B1144BD3F8343601AA7A
:10A020004FF48471204604F018FD4FF486712046E9
:10A0300004F013FD4FF48871204604F00EFD0C4B24
:10A04000234083B14FF48E75294601AA204604F0BF
:10A0500004FD291F083589B22046ADB204F0FDFC8D
:10A06000B5F5AE7FF0D1019802B070BD0070004030
:10A07000C0FF3F002DE9F04F93B09A460DF1080C58
:10A080000AAF1C9D3F4B3E46E046002403EB041EF6
:10A090000134DEF8189548F8049B082CDEF81CE51E
:10A0A00046F804EBF2D1D3F8F065D3F840460194BA
:10A0B0004FF0010E0024D3F84496D3F84886C3F835
:10A0C000FC4FC3F8FCEF2F4B5CF804BB03EB041E02
:10A0D0000134CEF818B557F804BBCEF81CB5082CDF
:10A0E000F2D1019CC3F84046F6B2274CC3F844961F
:10A0F000C3F84886C3F8F065002684F8336084F816
:10A100003460A6602661256084F83100A683C3F818
:10A11000F015C3F8F4252DB32322C3F800231A4DFC
:10A12000184E0021012707FA01F303404FEA0112FC
:10A130001BD102F1804404F5E044C4F81035C4F8A2
:10A14000143532440131D2F8184524F0807444EAC1
:10A1500003630829C2F8183505F10205E3D113B0ED
:10A16000BDE8F08FC3F80053D9E702F1804303F54F
:10A17000E043EC7F95F81EC0C3F810C5C3F8144542
:10A180005346DEE7007000408819002010B5C37800
:10A190008278417A1B03120202F4E06203F48053D6
:10A1A0001343027802F0030213430279120402F40B
:10A1B000E02213434278120102F030021343827905
:10A1C000120602F0807213434279120502F48012E3
:10A1D00013430A0102F1804202F5E042C2F8183549
:10A1E000084AC47901F10C0302EB43039C71007A25
:10A1F000D871012303FA01F192F830300B4382F851
:10A20000303010BD8819002070B51F4D95F82E40D4
:10A21000002C37D10126FF2085F82E60FFF7C6FEFF
:10A220001A4B1B49C3F80041D3F80021C3F804417D
:10A23000D3F80421C3F81041D3F81021C3F8144116
:10A24000D3F814311C239A0806FA02F212F0330FE5
:10A250001FBF03F1804202F5E242146012681A1F28
:10A26000920806FA02F212F0330F1CBF5C505A58E3
:10A2700008335C2BE7D10720F7F7CCF8002305481B
:10A280002B6070BD0448FCE7881900200070004076
:10A29000FC7000400000AD0B0C00AD0B08B5024691
:10A2A000FFF744FE20B91046FFF770FF014808BDD4
:10A2B0000148FCE70000AD0B0B00AD0B014B93F820
:10A2C00030007047881900202DE9F04385B005461D
:10A2D0009946FFF72BFE88461646074608BB0DF148
:10A2E0000F012846FFF706FE0F4B9842044614D193
:10A2F0000E4BC3F8F875331E18BF01233246CDF854
:10A30000009041462846FFF7B5FE094B9DF80F2007
:10A3100083F83220022283F82E20204605B0BDE8C3
:10A32000F083044CF9E700BF0000AD0B0070004063
:10A33000881900200B00AD0B2DE9FF470746994611
:10A34000FFF7F4FD8A461446064600283FD10DF17A
:10A350000F013846FFF7CEFD1F4B9842054627D127
:10A3600063889DF80F803BB3B8F1010F31D8B9F184
:10A37000000F2ED02278637812B1B3FA83F67609F3
:10A38000CDF8009051463846FFF774FE6388134AB3
:10A390000BB143F48053C2F8F835114B83F8328087
:10A3A000227983F83520042283F8366083F82E2042
:10A3B000284604B0BDE8F08722786378002ADFD011
:10A3C000002BDDD1B8F1010F03D80126D8E7054DE8
:10A3D000EEE7054DECE700BF0000AD0B007000405C
:10A3E000881900200B00AD0B0300AD0B10B51B4B03
:10A3F0001A696ABB00F06042B2F1005F2AD193F89B
:10A400003220B1FBF2F402FB14142CBB0CB2002C72
:10A4100022DD93F82E40052C05D8032C0AD8022CF7
:10A420000DD00F4810BD062CFBD10E4AC2F82C06E9
:10A43000C2F830169A6842B1C3E9040103E08A42C7
:10A440000AD1C3E902020848ECE7C3E90201FAE7CE
:10A450000648E7E70648E5E70648E3E788190020ED
:10A460000500AD0B007000400000AD0B0C00AD0B03
:10A470000A00AD0B0600AD0B2DE9F3414F4CA3686C
:10A48000002B00F0998094F82E20022A05D0042A8F
:10A4900030D04B4802B0BDE8F0814A4D0126C5F8E6
:10A4A00000652168E26849B1032184F82E10C5F8DF
:10A4B0002C36C5F830262E604348EBE7C5F82C361D
:10A4C000C5F830262E6004F0DFFA08346E602146AD
:10A4D0000220FFF789FD0028F9D03A4B0022C3F88B
:10A4E0000821D3F80811C3F80C21D3F80C11C3F8D4
:10A4F0000025E1E7334D4FF00108C5F800852768D6
:10A5000057B1052284F82E20E268C5F82C36C5F82C
:10A510003026C5F80080CFE7A18B94F83220019255
:10A5200003EB41030093C5F82C36C5F83026C5F877
:10A53000008004F0A9FA94F836305BBB214D01236A
:10A540006B6069460220FFF74FFD0028F9D000221A
:10A55000C5F80821D5F80831C5F80C21D5F80C311B
:10A56000A18B94F832300B44E1689BB28B42A383F9
:10A5700021BF164BA283D3E90201C3E90001114BAD
:10A5800028BF22614FF000022CBF0F481048C3F8CB
:10A5900000257FE7D5F8F465F6B208FA06F6013E25
:10A5A000BE42CBD9C5F8048000210420FFF71CFD72
:10A5B0000028F9D00137F3E706486BE78819002037
:10A5C0000500AD0B007000400000AD0B901900209D
:10A5D0000B00AD0B0200AD0BF8B50246FFF7A6FC71
:10A5E000002851D1294E2A4C96F82E3086F82F306B
:10A5F000072386F82E3001237260C4F80035D4F8A2
:10A600000453C4F80003E3603AB125F0C00545F0F7
:10A610003305C4F800531F48F8BD00211020FFF790
:10A62000E3FC0028F9D00023C4F80431D4F8043145
:10A63000194BC4F82C3601270223C4F830362760A2
:10A6400004F022FAA76000212020FFF7CDFC0028AB
:10A65000F9D00F4B0022C3F80421D3F80411C3F83A
:10A660000821D3F80811C3F8002596F82F1086F8B2
:10A670002E10C3F81C21D3F81C11C3F81821D3F8ED
:10A680001821C3F80053C6E70448C5E7881900201D
:10A69000007000400000AD0BA01900200B00AD0BB6
:10A6A0007FB56249614E3320FFF79EFC10F0100F1A
:10A6B00005460BD05E4B1022C3F80823B218C3F82E
:10A6C0002C260222C3F8302601221A60594CAA0611
:10A6D00094F82E300ED5072B554A05D0D2F83436D3
:10A6E0009BB2E36000232361D2F80433DB0601D57B
:10A6F000FFF72AFCA80718D594F82E30A16802911C
:10A700000022E1688DF80420062BADF80C1018D05B
:10A71000072B35D0032B08D1454BC3F80025022366
:10A7200084F82E30236801A89847E9074FD594F89C
:10A730002E30033B042B4AD8DFE803F05A49294165
:10A740005E0094F8353023B1236913B1384B0122F0
:10A750001A60236801A89847374B93E8030086E8FE
:10A76000030000232361A368002BDED1304AC2F826
:10A770000035042384F82E3005238DF80430D1E70A
:10A78000FFF7E2FB02238DF804306368CBE7042374
:10A790008DF8043001A823689847254BD3F8F82595
:10A7A000D20444BF01225A602269062384F82E3065
:10A7B0002AB11F4B6169C3F82C26C3F830162369F0
:10A7C0002BB903238DF8043001A82368984794F827
:10A7D0002E30072B0AD0164B1848D3F8043300212B
:10A7E0001840FFF701FC012685094DB904B070BD82
:10A7F0000F4B01225A60EAE70D4B01229A60E6E70F
:10A8000095FAA5F3B3FA83F306FA03F225EA0205F3
:10A810005A08DB4303F001038DF809308DF804601A
:10A8200023688DF8082001A89847DEE790190020DA
:10A83000007000408819002098190020C0FF3F00D8
:10A8400010B4CC7B8A6803682CB9D1E90041C3F805
:10A850000845C3F80C15C3F8242503792C2253436B
:10A86000054AD3582BB1006810BC40F30730F6F707
:10A87000D1BD10BC704700BFC019002000F01F03FD
:10A8800040090BD19B0003F1A043074AD3F80017FE
:10A890000A4042F00202C3F800277047002203F585
:10A8A000E07352F82330FFDEF0F8FCFF30B5847B14
:10A8B000F4B9016801F01F0349091BD19B0003F1A2
:10A8C000A043114DD3F8002740F20C642A402243E4
:10A8D000C3F80027426802F01F0352090FD19B0002
:10A8E00003F1A043D3F800272A402243C3F80027EE
:10A8F000012030BD03F5E07354F82330FFDE03F58B
:10A90000E07351F82330F9E7F0F8FCFF70B50D461D
:10A9100086B04FF48011044604F000F908B34FF4F8
:10A920008013C4F80833D4F82435D3B9C4F80035FB
:10A930000623C4F80035AB6AC4F82435EB6913F07C
:10A94000010318BF0123C4F85035EB69012213F04D
:10A95000020314BFC4F84025C4F84035A26006B015
:10A9600070BD0221204604F0D9F84FF4007106466C
:10A97000204604F0D3F8C8B1D6B9AB68C4F80833A0
:10A980000223AB60AB68C4F804334FF080712046FB
:10A9900004F0C4F818B1D4F800329B0502D40123A6
:10A9A00023626361012385F82330D8E7002E67D046
:10A9B000EB695E060AD495F823303BB92946204658
:10A9C00004F06AF880F0010085F82300EB6913F0C9
:10A9D000040324D1C4F86031D4F86021C4F85C3198
:10A9E000D4F85C3195F825301BB195F82330002B55
:10A9F00052D00023C4F80032AB60394BC4F808339E
:10AA000044F30733002B47DB5A09012103F01F03EE
:10AA1000994002F16003334A42F823103CE095F874
:10AA20002030012B0AD00023C4F85035C4F840353B
:10AA3000C4F824354FF48013C4F80433D4F8C43474
:10AA4000C4F8C434980745D4590745D4DA0745D427
:10AA500095F823309B00DBB28DF8003095F8253057
:10AA60000BB985F82430EB695B0704D595F82330E2
:10AA7000002B3FF474AFD5E90031684698476EE784
:10AA80004FF48021204604F049F895F820307BB936
:10AA900095F82530002BADD02B8CADF80430EB6849
:10AAA00004932B6902936B690593AB690393C5E724
:10AAB0004FF40073C4F8003240F20223AB6003F19C
:10AAC000CE73C4F80833AB68C4F804330123A36021
:10AAD000236244E70123BFE70223BDE70323BBE76B
:10AAE00002029C0100E100E02DE9F04190F80480B1
:10AAF000174E07462C2000FB08F035180C4695F839
:10AB0000221001BBA96032506B6085F8251085F8D2
:10AB100024107CB1A37B85F827302046FFF7C6FEC2
:10AB200098B1637B85F82630A368AB62214638462E
:10AB3000FFF786FE2C2303FB08660648012386F8F0
:10AB40002230BDE8F0810448FBE70448F9E700BF84
:10AB5000C01900200000AD0B0C00AD0B0400AD0BC4
:10AB6000036802790621C3F80015044B2C2101FB70
:10AB70000233022283F82220704700BFC019002050
:10AB800010B51D4A04792C2303FB0423002199608E
:10AB900001681A4BC1F80833D1F8003223F4BC53D2
:10ABA000C1F800324FF08053D3F83001B0F1FF3FCD
:10ABB00009BF4FF07043D3F8343193F8E00FD3F866
:10ABC000E83F08BFC3F30313062808D1033B042B57
:10ABD00002D80B48C35C13B10923C1F800352C23FC
:10ABE00003FB042300200122C1F8000583F8222082
:10ABF00083F8240010BD00BFC019002002029C0190
:10AC00005D06010070B5044606790068104D40F3FA
:10AC10000730F6F70DFC2046FFF7B2FF2C2303FBAD
:10AC2000065393F8272062B993F826304BB923686E
:10AC3000D3F80805D3F80C45FFF720FE2046FFF7B0
:10AC40001DFE2C2303FB0655002385F8223070BD22
:10AC5000C01900202DE9F74FB94D90F80490046811
:10AC60002C2303FB09539046002283F823204B68D2
:10AC70000E4633B1CB6803F06043B3F1005F40F0A0
:10AC8000A2813378023B012B06D8336903F060437D
:10AC9000B3F1005F40F09781AA4BC4F808332C232E
:10ACA00003FB095393F8241001F0FF0241B19B68A4
:10ACB000DFF894B2C4F80433584603B0BDE8F08F0F
:10ACC00018F0140F0CBF0121002183F824103178F3
:10ACD00083F82010717883F82110F168D9607168C9
:10ACE000196131695961B1689961C8F3001183F83C
:10ACF0002510C3F81C807378C4F88835C4F8602127
:10AD0000D4F86031C4F84821D4F84831C4F824217B
:10AD1000D4F82431C4F80421D4F8043118F0010324
:10AD200018BF0123C4F8503518F0020318BF0123DF
:10AD3000C4F8403533782C2709FB0757032B00F262
:10AD4000BC80DFE803F092B17B024FF48073C4F85B
:10AD50000032D7E90323C4F84425C4F84835012359
:10AD6000A3604FF48011204603F0D8FE0028F8D1EC
:10AD7000D7E90523C4F84425C4F848352C2303FB40
:10AD800009534FF480229A60DFF8C0B12C2202FBF5
:10AD900009F218F00803A858019305EB020114D139
:10ADA0003278032A11D0012A40F09D8022600028C9
:10ADB00000F086802C2202FB09F27168AA5821B9A2
:10ADC000002A00F0D680012262612C2202FB09F2E7
:10ADD000A918AA58002A00F0CC8018F0040F1CBF54
:10ADE00000228A6018F0400F06D12C2202FB095283
:10ADF000916841F0020191602C2202FB0952019BF3
:10AE0000916841F4007191609268C4F80423002BAA
:10AE100000F0A8803278012A00F0A4800022C4F853
:10AE20005025C4F84025C4F82425C4F85021D4F88E
:10AE300050214FF48012C4F804233DE7D7E90323DF
:10AE4000C4F84425C4F84835D7E90523C4F83425A7
:10AE5000C4F838354FF48453C4F800320123236218
:10AE60002C2303FB095302228DE7D7E9032318F0B3
:10AE7000200FC4F84425C4F848354FF02C0315BF03
:10AE80004FF480724FF4007203FB095303FB095324
:10AE900015BFC4F80022C4F800224FF48022022219
:10AEA0009A60012323626FE7D7E90323C4F83425AE
:10AEB000C4F838354FF48053CEE7DFF894B065E737
:10AEC000096901B962612349DFF88CA0204603F0CB
:10AED00025FE012310F4007F18BF636110EA0A0FFA
:10AEE0001C49F3D066E70122A26000287FF462AF1C
:10AEF0000969A9B34FF0000A174B1AEA030F7FF450
:10AF000059AF1449204603F009FE10F4007F824631
:10AF1000F2D04FF08071204603F000FED4F800120A
:10AF2000E0B111F4007003D1012222628246626115
:10AF3000CB05E1D54FF48021204603F0EFFDD9E7A2
:10AF4000C019002002029C010B00AD0B0000AD0BEC
:10AF50000400AD0B02020400020004000122226280
:10AF60006261C7E72C2202FB0952926AC4F82425C9
:10AF7000A2E62C21D4F8C424C4F8C42401FB09554A
:10AF8000002185F824108AB11049114B12F0010FED
:10AF900014BF8B469B46013112F0020F18BF8B463F
:10AFA00012F0040F0B4A18BF934685E618F0400FC5
:10AFB0007FF482AE3946204603F06EFD044A002835
:10AFC00008BF934678E6DFF810B075E60000AE0BD8
:10AFD0000100AD0B0200AE0B0A00AD0B01490248A7
:10AFE000FFF794BCC01900200030004002494FF028
:10AFF0004020FFF78BBC00BFEC190020F7B50646D8
:10B0000003F0C0FD084603F0BDFD01A8019603F062
:10B01000AFFD019B2E4D00EB83000C46D0F80037AE
:10B02000019440F20D612B400B43C0F8003701A89A
:10B0300003F09EFD019B00EB83000127D0F8003751
:10B040002B400B43C0F80037042003F07DFC09259A
:10B0500001A8019403F08CFD019AD0F81035D3407B
:10B06000DB0715D401A8019603F082FD019B07FAC6
:10B0700003F3C0F80C35042003F066FC304603F0FF
:10B0800081FD013D042003F05FFC15F0FF05DFD1D9
:10B0900001A8019403F06CFD019A01239340C0F8CC
:10B0A0000C35042003F050FC204603F06BFD042017
:10B0B00003F04AFC01A8019403F05AFD019AD0F86C
:10B0C00010350448D34003F00103C01A03B0F0BDAB
:10B0D000F0F8FCFF0100AD0B08B5144BA8220021CD
:10B0E000184604F0B9F90322026111494261114A7C
:10B0F0008161C2614FF48062026200228262426218
:10B10000C26201660C4941661021816603460267EE
:10B11000C2664267BFF35F8F084911F8010D98546A
:10B120000132102AF9D1BFF35F8F08BD100400204F
:10B130006206010010000020000000207B060100D4
:10B1400010B4BFF35F8F0B4A0B490023C85C12F8A1
:10B15000014D844209D10133102BF7D10023BFF3F5
:10B160005F8F23B110BCFFF7B7BF0123F7E710BC17
:10B17000704700BF7B0601001004002038B5EFF3D4
:10B180001185202383F31288BFF36F8F064B9C68D1
:10B1900003F039FD85F31188BFF36F8F2046BDE8BA
:10B1A0003840F6F7DFB800BF181A002038B50A4B50
:10B1B00053F82040013053F82050A54200D838BD44
:10B1C000606830B1037FDB0701D403F0F1FC083481
:10B1D000F3E723689847FAE740FF000070B52A4B71
:10B1E0002A4C2B4D012286B003201A70FFF7DEFF98
:10B1F00001F0C0FA0420FFF7D9FF2646AE4204F161
:10B20000300410D300F03EFE204C224EAC4226D338
:10B2100000F04CFE01F011FD1F4A137B23F00103E7
:10B22000137306B070BD54F80C3C059354F8103CF1
:10B23000049354F8143C039354F8183C029354F8C4
:10B240001C3C019354F8203C009354E90A2354E930
:10B250000C0100F0FFFB54F8303C5E65CDE7D4E90B
:10B260000A23B3F1FF3F08BFB2F1FF3F05D052EA16
:10B270000301206803D100F0D5FE3034C6E7314623
:10B28000183001F05FF8F8E7871A002084F9000011
:10B2900084F90000DFF00000500B002070B500239F
:10B2A00086B00122CDE90423134E144D01930F22E1
:10B2B000CDE902321249142303FB005506EBC016F8
:10B2C00004464FF4C07000FB04110E4B00954FF480
:10B2D000A072304600F0BEFB737B0B4AEE6023F099
:10B2E000040373734FF4046304FB033313442C749B
:10B2F0006B6006B070BD00BFD00A0020181A002095
:10B30000C02D002055EC000080250020BFB5002096
:10B31000FFF74CFF284B83F30888284C284F6369BC
:10B3200043F4007363610025E02384F82230E5775D
:10B3300025766576A57684F82050636A43F4E02389
:10B34000636284F82350F5F7DBFFF6F725F94FF039
:10B35000FF33A362E362F6F7E5F9F6F741F919481E
:10B36000194C00F0EFFB0120FFF720FF0220FFF750
:10B370001DFF00F0CFFD154B15495C61154B059382
:10B380000123CDE903534FF480623B46CDE90155DB
:10B390000095204600F05EFB627B064622F0040228
:10B3A0002046627303F05EFE2846FFF777FF3A46B9
:10B3B00031462046F6F7D2F8C02D002000ED00E01F
:10B3C000DDB10000700C0020500B0020181A002086
:10B3D000402F00207C06010038B5064C064DAC42DB
:10B3E00001D3002038BDD4E90112204603F00EFC41
:10B3F0001434F4E728080020280800202DE9F34140
:10B40000044617461E46EFF31188202383F3128863
:10B41000BFF36F8FC368334A7BB1806891688842FD
:10B4200019D057EA060318D188F31188BFF36F8F3C
:10B430006FF00F0002B0BDE8F081916891F90E1035
:10B4400021610133E3609368A36088F31188BFF33F
:10B450006F8F0020EEE72169F2E791F90E1090F965
:10B460000E309942A8BF19466FF07E029142B8BFD4
:10B4700011468B422DDD03F0F8FB0546CDE9007641
:10B4800019482246414600F043FC0028E1D0EFF382
:10B490001186202383F31288BFF36F8FA068D0B189
:10B4A000236821699C420AD04BB193F90E3099422E
:10B4B000A8BF19466FF07E039942B8BF194603F042
:10B4C000D4FB40B10848314600F0B6FC6FF00A00EA
:10B4D000B0E70025D2E7002DF4D186F31188BFF341
:10B4E0006F8FF3E7181A0020881A0020F8B58368D8
:10B4F0000546002B3FD0234A926893423ED1C36851
:10B50000012B03D9013BC3600020F8BDEFF3118785
:10B51000202383F31288BFF36F8F0169806803F0E3
:10B52000A4FB2C68A54207D10023C5E9023387F3A9
:10B530001188BFF36F8FE7E7002CF5D0D4E9003214
:10B5400013605A60637B002623F002036373C4E92F
:10B550000066A66004F1180003F051FEAC6094F997
:10B560000E302B612046E66703F07CFD0648394625
:10B5700000F062FCC8E76FF01500C6E74FF0FF303F
:10B58000C3E700BF181A0020881A002037B51146FB
:10B59000EFF31185202282F31288BFF36F8F0468C6
:10B5A0009CB12368426823F003039442036008BF00
:10B5B00043600121204603F0E5FB044685F3118832
:10B5C000BFF36F8F204603B030BD51EA0302F5D0C0
:10B5D00000F10802CDE900131046294600F098FB5F
:10B5E0000028EFD1014B9B681C69EBE7181A00207B
:10B5F00070B5EFF31186202383F31288BFF36F8FAA
:10B600000468A0421AD0CCB1D4E9003213605A6069
:10B61000637B002523F00203C4E900556373A56032
:10B6200004F1180003F0EBFDE567204603F01AFD76
:10B6300031460B48BDE8704000F0FEBBD0E9023255
:10B640009A4218BF013383600221103003F0B6FE26
:10B650000028EDD186F31188BFF36F8F70BD00BF56
:10B66000881A002013B5EFF31181202484F3128887
:10B67000BFF36F8F846844B1013C846081F311880B
:10B68000BFF36F8F002002B010BD52EA030406D151
:10B6900081F31188BFF36F8F6FF00F00F3E7CDE9EF
:10B6A00000230246014800F033FBECE7881A002033
:10B6B0002DE9F8430546EFF31188202383F3128820
:10B6C000BFF36F8F002637466FF00A092C68A5423A
:10B6D00016D0ACB1D4E9003213605A60637BA76026
:10B6E00023F002036373C4E9007704F1180003F048
:10B6F00086FDC4F87C90204603F0B4FC0126E5E703
:10B700000023AB60022105F1100003F057FE30B9B1
:10B710002EB988F31188BFF36F8FBDE8F8834146D7
:10B720000248BDE8F84300F087BB00BF881A00203C
:10B7300007B5074B0093074907484FF0FF334FF415
:10B74000806200F013F9002003B05DF804FB00BF35
:10B7500058FF000080330020D00B00202DE9FF416E
:10B760004F4E04462027EFF3118887F31288BFF36A
:10B770006F8FD4F88450F5B9022104F19C0003F0D6
:10B7800074FB002868D004F19405002201212846AA
:10B7900003F0FCFC0028F8D1002302934FF0FF32A5
:10B7A0004FF0FF33CDE90023414604F18C023D48C0
:10B7B00000F002FDD7E7D4F888202B68C4F8843065
:10B7C000954208BFC4F88830D4F89C3043F0020397
:10B7D000C4F89C30EB6823F0040343F00103EB60F2
:10B7E0006B6888F31188BFF36F8F28469847EFF393
:10B7F000118887F31288BFF36F8FEB68D80623F0A8
:10B80000010236D4EA60EB689A0716D5306823F057
:10B810000203EB6088B10368002170B14268954271
:10B8200035D1036869BB72683360824200D17360AE
:10B83000002340F8083BFFF7DBFED4F89C3023F0F0
:10B840000203C4F89C3088F31188BFF36F8FDB05C7
:10B8500089D400F067FB86E7D4F89C30D9069BD5E5
:10B86000C4F89C0088F31188BFF36F8F04B0BDE863
:10B87000F08123F01103EB6005F11000FFF7B8FE33
:10B88000C1E70B607368834208BF7160D0E723B1E2
:10B890001A68014618461346BFE71A46F9E700BF83
:10B8A000381A0020881A0020F8B5C3689A070446A1
:10B8B0000F46C3F340062ED45B071CD40B680BB9AC
:10B8C00083680B60E368DD0744BFA3683B603D68A5
:10B8D0004CBF02260126002D3CD0204B9A68D5F89B
:10B8E00080309A420AD0D5F89C30D807C3F3800242
:10B8F00014D46FF0120600233B6025E003F06FFBC9
:10B90000D5F89C300028F0D1D907C3F3C002F0D598
:10B9100052B15B0708D46FF00F06ECE7002AFAD1AA
:10B92000C3F3C003002BF6D100232360D5F8883081
:10B9300063B9C5E92144284603F0B1FAE36843F04E
:10B940000403E3603B68A3603046F8BD1C60C5F8A3
:10B950008840F0E76FF01506CDE700BF181A002009
:10B960000146014803F006BBD00B0020F0B589B0BA
:10B9700004460020C4E921000E9D04F18C00C4E9B6
:10B98000230004F19400C4E9250055B32879002868
:10B9900040F2011008BF0120C4F89C0000204FF0C5
:10B9A000FF364FF0FF37CDE90330CDE90100CDE997
:10B9B00006670D4B0094204600F098F855B12968B1
:10B9C00011B1204603F011FB6B791BB1237B43F0CF
:10B9D00001032373204600F025FBC4F8804009B022
:10B9E000F0BD0120D8E700BF5DB70000F7B50C46F9
:10B9F000019016461D46EFF31187202383F312882A
:10BA0000BFF36F8F084603F03BFA55EA060309D1EE
:10BA100001A92046FFF748FF87F31188BFF36F8F16
:10BA200003B0F0BDE368074943F00803E360019BFE
:10BA3000A36232462B4604F1100000F083FC012083
:10BA4000EAE700BF13EF000001460148FFF7CEBF51
:10BA5000D00B00202DE9F043073285B022F0070219
:10BA60000E461F461099017300F158037F32C0E95A
:10BA700016330446002322F03F0204218360417301
:10BA80003F2A0F98A073C4E90633E37306F1400917
:10BA9000A2F1400805D883F31188BFF36F8F0846E1
:10BAA00002DFB51829462046F5F70AFA07300E9B43
:10BAB00020F00700E066C4E9199802930D9B0193FA
:10BAC0002D1A0C9B00932A463B4631462046F5F73B
:10BAD00013FD00236365044B9B6803B11B6F236751
:10BAE000284605B0BDE8F083181A0020F0B587B0ED
:10BAF00000250595109D04950F9D03950E9D0295BB
:10BB0000DDE912760D9D01950C9D00950446FFF729
:10BB1000A1FFB6F1FF3F08BFB7F1FF3F05D056EADE
:10BB2000070305D1204600F07DFA204607B0F0BD9E
:10BB30003A46334604F11800014900F003FCF4E7EB
:10BB4000DFF0000040F2011383810023C0E91933C4
:10BB50000367014B98607047181A0020094A9368E0
:10BB60006FF00A01D967084998674B6843F0805322
:10BB70004B60002383F31188BFF36F8F9368D86FF6
:10BB8000704700BF181A002000ED00E070B590F972
:10BB90000D20437B002A36DBD90634D11B4C63F0E1
:10BBA0007F032246437352F8183FE169934207D15D
:10BBB000C0E900210860E06111E09942F8D01B68FB
:10BBC000002BF5D090F90E5093F90E60B542F4D0E9
:10BBD000AE42F2DD5968C0E9003108605860A569DD
:10BBE000954200D005B9E568A3685A7BD20604D116
:10BBF000DA897F2A01D9AA6932B1AB4202D028463C
:10BC000000F01AFB656170BD6361FCE7181A002043
:10BC100038B590F90D20437B002A014604DA03F081
:10BC20007F03437303F0E4F90D4D2A46AB6852F8E5
:10BC3000184F944200D004B9EC688B4207D05A7B6D
:10BC4000D20604D1DA897F2A01D9A2692AB1A34296
:10BC500002D0204600F0F0FA23466B6138BD00BFE9
:10BC6000181A0020B3F1FF3F08BFB2F1FF3F03D025
:10BC70000249183000F066BB704700BFDFF00000DB
:10BC800070B590F90D20437B002A014604DA03F0D9
:10BC90007F03437303F0ACF94B7B1C4C63F07F03D1
:10BCA00022464B7352F8183FE069934207D1C1E92D
:10BCB00000200160E16111E09842F8D01B68002B80
:10BCC000F5D091F90E5093F90E60B542F4D0AE4222
:10BCD000F2DD5868C1E9003001605960A569A368C8
:10BCE000954200D005B9E5688B4207D05A7BD20651
:10BCF00004D1DA897F2A01D9AA692AB1AB4202D0DC
:10BD0000284600F099FA2B46636170BD181A00208E
:10BD1000F8B50E4B0C4611460D4A98681060DDE9E7
:10BD20000667EFF31182202282F31288BFF36F8F30
:10BD30009D68284603F06EF9284632463B46FFF7D9
:10BD400091FF2046BDE8F840FFF708BF181A002011
:10BD5000401A0020F8B50446EFF31187202383F33F
:10BD60001288BFF36F8F437B03F01F02002A0CBFC2
:10BD70000126002649B239D103F07F03437303F053
:10BD800037F92C4D437B817363F07F032A4643735D
:10BD900052F8183F934227D1E869C4E900200460B3
:10BDA000EC610FE09842F8D01B68002BF5D093F9B6
:10BDB0000EC06145F6D08C45F4DD5968C4E9003108
:10BDC0000C605C60AC69944200D004B9EC68AB686C
:10BDD0009C4202D0204600F02FFA6C6187F3118854
:10BDE000BFF36F8F3046F8BDE869DEE79B071ED5CD
:10BDF000856803F0FDF881732B689D4209D16B685B
:10BE0000C4E900531C606C60E8E76A689342F6D0AE
:10BE10001B68002BF3D093F90E209142F5D08A4293
:10BE2000F3DD5A68C4E9003214605C60D6E78173C0
:10BE3000D4E700BF181A002049B9EFF3058030B9E4
:10BE4000054B5A699B689A4201D0FFF787BE81F380
:10BE50001188BFF36F8F7047181A0020034648B946
:10BE6000EFF3058232B9064A51699268914201D0D6
:10BE7000FFF774BE83F31188BFF36F8F704700BF65
:10BE8000181A0020EFF31181202383F31288BFF3E7
:10BE90006F8F054B9A68D37B013BD37381F3118875
:10BEA000BFF36F8F704700BF181A002070B5EFF313
:10BEB0001186202383F31288BFF36F8F144DAB6874
:10BEC000DA7B0132DA732A4652F8184F944200D0D6
:10BED00004B9EC685A7BD20604D1DA897F2A01D9E9
:10BEE000A2692AB1A34202D0204600F0A5F9234658
:10BEF0006B6186F31188BFF36F8FEFF311802023FE
:10BF000083F31288BFF36F8FBDE87040FFF7A6BFC1
:10BF1000181A0020024B03F11802C3E906227047E9
:10BF2000181A002070B5EFF31186202383F31288CE
:10BF3000BFF36F8F1B4CA168E0690B68814214BF8F
:10BF40001A46002249680B605960A368E1692AB962
:10BF5000154AC3E900210B60E3610CE093F90E0080
:10BF600092F90E50A84218D0854216DD5168C3E9F7
:10BF700000210B605360A5690B4B9D4200D005B9B1
:10BF8000E568A3689D4202D0284600F055F9656136
:10BF90003046BDE87040FFF7E1BD8A42D8D0126854
:10BFA000D5E700BF181A0020301A0020F8B550EA73
:10BFB000010306460C4603D1FFF7B4FF0020F8BD8D
:10BFC000EFF31187202383F31288BFF36F8F124D95
:10BFD000124BA8681860FFF71BFEA868104923469B
:10BFE0003246183000F0AEF9AA68537B43F00403E0
:10BFF000537304463846FFF7B1FDAB68D3E90A2313
:10C00000B3F1004F08BF002AD8D103F020F9201A5D
:10C0100020EAE070D3E700BF181A0020401A002081
:10C02000DFF0000038B50446EFF31185202383F3D9
:10C030001288BFF36F8F437B5B070FD5183003F077
:10C04000DEF8637B23F0040320466373FFF79EFD55
:10C0500029460548BDE83840FFF7EEBE85F3118854
:10C06000BFF36F8F38BD00BF881A0020014B98685E
:10C07000704700BF181A00202DE9F8430446077BDB
:10C08000EFF31185202383F31288BFF36F8F437B77
:10C09000190705D585F31188BFF36F8FBDE8F883C5
:10C0A000D90943F008025DD14273A36813B1204659
:10C0B00002F0A6FF04F1180003F0A1F8A66D04F148
:10C0C0005808B04511D04FF0000976B1304602F063
:10C0D00097FF06F1180003F092F8C6F87C903046FE
:10C0E000FFF754FDA66DB045EFD1DFF8C080D8F85A
:10C0F00008309C423ED1EFF30589B9F1000918BF21
:10C100004FF00109D8F81860294A964200D00EB9BC
:10C11000D8F80C60B34202D0304600F08DF82046CB
:10C12000C8F8146001F0FDF8B9F1000F02D0214801
:10C13000FFF708FDD8F808309C4231D1EFF30583B2
:10C1400073BB227BD20718D42846FFF707FDFB07F5
:10C15000A4D5002383F31188BFF36F8F04231846FF
:10C1600002DF9BE703F07F0343F00803437302F011
:10C170003FFF9AE74FF00009C4E785F31188BFF34A
:10C180006F8F83F31188BFF36F8F0423184602DF8C
:10C19000EFF31180202383F31288BFF36F8FD4E76E
:10C1A00085F31188BFF36F8FD1E700BF181A002005
:10C1B000301A0020700C0020D3B5DDE90667089C1A
:10C1C000CDE90067FFF7A4FD1CB1034B9B681B6919
:10C1D000236002B0D0BD00BF181A0020044BC01A63
:10C1E000044BC0105843044B01221A54704700BF3F
:10C1F000F00C0020ABAAAAAA881A0020C3897F2BC2
:10C2000012D80A4B1B6863B1094B90F90E201B68CA
:10C210009A4209DB437BDB0606D1064BC31A18BFE3
:10C22000012303F0010070470023FAE7E80700202C
:10C23000441A0020D00A002070B50E4B0E4C1E7C14
:10C2400006EB460304EBC3040546204602F0D7FF85
:10C250000A4B002228469A55FFF7D0FF48B1084BF9
:10C2600008491A68013A2046D317BDE8704000F02B
:10C2700069B870BD181A0020F00C0020881A002040
:10C28000E8070020DDC1000038B5EFF31185202359
:10C2900083F31288BFF36F8F104B114A9C681068AC
:10C2A000A04206D1FFF7C8FF85F31188BFF36F8F57
:10C2B00038BD00211B7C11600A4AD35C002BF3D0EF
:10C2C0002046FFF79BFF0028EED0637BDB0602D100
:10C2D0002046FFF7D5FC2046E4E700BF181A0020EF
:10C2E000401A0020881A0020024B1868984208BFA4
:10C2F00000207047EC070020034B1B680BB9FCF7CC
:10C30000ADBF0020704700BF481A002030B570B1A3
:10C310000B4B5B6898420AD0036843B1D3E9042110
:10C32000D0E90445121941EB0501C3E90421D0E924
:10C33000003213605A600023C0E9003330BD00BFF3
:10C34000EC070020B3F1FF3F08BFB2F1FF3F2DE93A
:10C35000F84F0446994615461F467AD08160EFF3A0
:10C360001188202383F31288BFF36F8FB9F1000F78
:10C37000DFF8E4A020DBFFF7BFFFDAE90027013593
:10C3800049F100092D1849EBE073C4E90453AD18D5
:10C39000064643EB07074FF00109FFF7A5FFDFF85B
:10C3A000BCE0DEF804A00346EBB9C4E900EACAF831
:10C3B0000040CEF8044028E0DAE900126FF00103F3
:10C3C0005B1A4FF0FF3161EB02025B1B62EB09026B
:10C3D000012B72F10001BCBF01230022C0E904322D
:10C3E0004FF00009D9E7D3E9041CD4E904208A42BC
:10C3F00070EB0C0B24DA891A5A686CEB0000C3E965
:10C400000410C4E9003214605C60FFF76DFF8442E1
:10C410000ED1134B1B685BB9B9F1000F02D1FFF7C6
:10C420006BFF0646304602F0D3FE0021FCF7E4FE27
:10C4300088F31188BFF36F8F28463946BDE8F88F1F
:10C44000521A60EB0C009A45C4E90420ADD01B6879
:10C45000AAE700252F46EFE7080D0020EC07002093
:10C46000481A00202DE9F047EFF31185202383F3CC
:10C470001288BFF36F8FDFF8A490DFF8A480C9F8AB
:10C480000000FFF731FF00260027D9F80030D8E977
:10C4900000ECD91750B1D0E90442A34271EB020A73
:10C4A0001CDAE41A62EB0102C0E9044213EB0E034A
:10C4B0004FF000044CEB01012046C8E90031C9F8F7
:10C4C000004002F085FE2146FCF796FE85F31188B8
:10C4D000BFF36F8FBDE8F047FFF7D6BE14EB0E0237
:10C4E0004CEBE473C0E90467C8E90023FFF70EFFD3
:10C4F00085F31188BFF36F8F83689847EFF3118539
:10C50000202383F31288BFF36F8FD9F800301B1BF1
:10C51000C9F80030FFF7E8FEB7E700BF481A00206F
:10C52000080D002010B5EFF31184202383F3128847
:10C53000BFF36F8FFFF7E0FE054A0346D2E9000123
:10C54000181841EBE37184F31188BFF36F8F10BDAE
:10C55000080D0020F8B50646EFF31187202383F37A
:10C560001288BFF36F8F026822B187F31188BFF37F
:10C570006F8FF8BDD0E90A54691C44F10003022909
:10C5800073F1000334D3013D44F1FF34002CBCBFF0
:10C5900015462C4602F05FFE013041F100014019C2
:10C5A00044EB0101012871F1000149DB02F053FE67
:10C5B000013041F100016FF00203401944EB010129
:10C5C00083426FF000438B413FDB02F044FE0130B9
:10C5D00041F100016FF00102401944EB01044FF0FA
:10C5E000FF33121A63EB04031A493046FFF7AAFE21
:10C5F000336B01333363336A6BB187F31188BFF355
:10C600006F8F336A30469847EFF31187202383F307
:10C610001288BFF36F8F334653F8184F9C42A4D053
:10C62000002CA2D0204602F02CFD0023E36787F304
:10C630001188BFF36F8F2046BDE8F84002F012BDAD
:10C640006FF001024FF0FF33CEE700224FF00043BE
:10C65000CAE700BF55C500002DE9F04105461C465C
:10C6600090461F46EFF31186202383F31288BFF311
:10C670006F8FB4F1FF3F08BFB2F1FF3F05D186F3E2
:10C680001188BFF36F8FBDE8F081002C09DB012A10
:10C6900074F10003BCBF0122002412F1FF3844F101
:10C6A000FF37284602F0ABFDDDE906010023C5E9AE
:10C6B0000A012B6342463B4628460249FFF742FEE9
:10C6C000DDE700BF55C5000038B50346EFF311851F
:10C6D000202282F31288BFF36F8FC1600121816035
:10C6E0000068834206D185F31188BFF36F8F002461
:10C6F000204638BDD0E9003213605A600023C0E9FB
:10C70000003302F018FE294604460248FFF794FB66
:10C71000EEE700BF891A0020F8B507460C4616461A
:10C7200002F05DFC08B10020F8BD0D4B9B681D6F49
:10C73000002DF8D0221DF6D2EFF31184202383F3CD
:10C740001288BFF36F8F47F004012846B04784F387
:10C750001188BFF36F8F0028E5D040F8045BE3E752
:10C76000181A00200146024A0020FFF7D5BF00BF7B
:10C77000D1CE0000014800F0EDBB00BF8A060100E9
:10C780002DE9F04F8DB043680293837815469A07E0
:10C79000804640F10D8100240E78002E00F00A81C1
:10C7A000252E0BD04B1C03930134029B414630468F
:10C7B00098470028C0F2F6800399EDE74E788B1C6D
:10C7C000252E0393F0D00027B946BB46BBF11F0FBF
:10C7D00038D8A6F12003102B0AD8DFE803F02A0985
:10C7E00009300909092109090928092D09091F002A
:10C7F000A6F13003092B33D92A2E37D11BF0400F75
:10C8000055F8043B40F08280002BA7BF4BF0200B73
:10C810009946C3F100094BF0280B01E04BF0010BE6
:10C82000039B13F8016B0393002ECFD130E04BF044
:10C83000020B4BF0040BF3E74BF0080BF0E74BF067
:10C84000100BEDE7BBF17F0F19D8A6F13003092BD0
:10C85000D2D81BF0400F03D00A2101FB0737DFE7D6
:10C860000A2101FB09394BF0200BD9E72E2E06D106
:10C870001BF0400F40F09E804BF0400BD0E76C2E39
:10C8800031D02BD8682E36D06A2E3CD04C2E3AD0E0
:10C89000002F46F02003B8BF2BF04002A3F1650142
:10C8A000BCBF1FFA82FB0027022901D9612B2FD1BF
:10C8B000073525F00705DFF8ACA2083507271BF080
:10C8C000080F66D00AEB070B56465E4563D1A4EB12
:10C8D0000A0A06EB0A02A9EB07096FE1742E9FD042
:10C8E0007A2E9DD0D4E71BF0800F18BF4BF4007B4D
:10C8F0004BF0800B94E71BF4807F18BF4BF4007B58
:10C900004BF4807B8CE74BF4207B89E71F4687E75D
:10C91000A6F16301122900F2F080DFE811F01300A4
:10C920004F00EE00EE00EE00EE004F00EE00EE00D5
:10C93000EE00EE00EE00FE00E900EE00EE001B004F
:10C94000EE00AF0055F8043B8DF8183001270DF1CB
:10C95000180AB4E755F804AB834BBAF1000F08BFCF
:10C960009A461BF0400F14BF39464FF0FF31504636
:10C9700002F08AFD0746A2E7029B41462020984725
:10C9800000280FDB013EB742F6D34C44A41BB1464E
:10C9900098E74E46F7E716F8010B029B4146984789
:10C9A000002892DA98F8023043F0040388F8023045
:10C9B0004FF0FF3420460DB0BDE8F08F1BF0800F24
:10C9C00034D01BF4007F2CD0073525F00705AA468C
:10C9D00069685AF8080B2BF010050029ADB237DA58
:10C9E000404261EB410145F480650DF1180B0A23CB
:10C9F0005A4602F055FDA0EB0B0301936B0662D57E
:10CA0000019B25F001019F4289B240F3A180002ED5
:10CA100000F0998015F0100240F09C80BB460D4656
:10CA200023E0AA465AF8040BC117D4E7AA461BF420
:10CA3000807F5AF8041B01D10846F5E71BF4007FFC
:10CA400015BF48B208B241F3C01141F3C031C2E78B
:10CA500050EA0103C9D11BF0400FC6D0002FC4D14A
:10CA60002BF0110295B2BB46019740F2064115EA40
:10CA700001021CBF0BF1010B00222CE02BF0100275
:10CA80001FFA82FB0A231BF0800C49D01BF40071B3
:10CA90001DBF073525F00705AA46AA461ABF5AF852
:10CAA000080B69685AF8040B50EA010545D12BF0D0
:10CAB00016051BF0400FADB242D0002F40D12BF035
:10CAC000170295B2019715F0100248D0019B002E75
:10CAD00042D103F1010B29075AD4EB0706D5D945FA
:10CAE0006FDD0199A9EB0B035F18CB465B4649E06C
:10CAF0004BF0100B10237826C5E7782B04D1C6F134
:10CB0000780343F01003BEE7029B41462520984777
:10CB10000028FFF647AF023447E608230026B2E7B5
:10CB2000AA461BF480715AF8040BBDD01BF40071A7
:10CB30001ABFC0B2614680B2B6E72BF0060295B2CA
:10CB40000DF1180B54E725F01105ADB2BB468CE78B
:10CB50000D46B8E73B460D4603F1020BBBE7DDF897
:10CB600004B082E7B9060100B2060100CDE9043243
:10CB70004146029B202098470028FFF613AF049BF4
:10CB8000059A01339945F1DCA4EB0B01CC189B46C7
:10CB90000AB3029B4146302098470028FFF602AFB7
:10CBA0008EB901342744019B391B994224DC1D4670
:10CBB0005DBB019AA9EB0B092244554614469144EA
:10CBC00035E0019F92E7023441463046029B984788
:10CBD0000028E7DAE6E640F206410D42E2D015F021
:10CBE000020F14BF2B20202015F4806F04F10104E4
:10CBF000414618BF2D20E9E7029B41463020984767
:10CC0000002804F10104CEDACCE606AB013D414632
:10CC1000585D029B98470028CADAC3E6029B41464A
:10CC200020209847002804F10104FFF6BBAEA9EBD1
:10CC30000403002BF2DCBFE5704708B500F004F8F0
:10CC4000F3F718FF002008BD08B500F00FF860B931
:10CC5000F3F7D6FE48B9F3F7AFFE30B9F3F77EFE2F
:10CC600018B9BDE80840F3F747BE08BD08B5002075
:10CC7000F5F7F2FB003818BF012008BD00EBC1003A
:10CC8000408840087047F8B50346FFF7F7FFB0FA51
:10CC900080F0C0F11F0003EB800CCA00DCF81060CC
:10CCA000171D0C4606328DB256B9012101FA00F06B
:10CCB000D9680143D960CCF81040DD539D52F8BDCE
:10CCC000F1000431585AD85303EBC0009E52C5807E
:10CCD0005D52F4E710B500EBC104E388994202F11C
:10CCE00004010AD1012303FA02F2C36823EA020312
:10CCF000C360002340F8213010BDA28840F82130E5
:10CD000000EBC20100EBC300CB808280F4E708B5E2
:10CD10000346FFF7B3FFB0FA80F2C2F11F021846D4
:10CD2000BDE80840FFF7D6BF2DE9F843B1FA81F519
:10CD3000C5F11F0900EB89080346D8F810200E46FC
:10CD4000C2B10327D8F8104018462146FFF796FFD6
:10CD5000B04206D34A461846FFF7BCFF2046BDE85E
:10CD6000F88303EBC404013FE088C8F8100001D049
:10CD70008242E7D1C5F120024FF0FF349440DA68D7
:10CD80001440EBD094FAA4F2B2FA82F2111D53F8D7
:10CD900021402146DFE738B50346FFF76FFF0D4618
:10CDA000044611461846FFF769FF03EBC505044426
:10CDB000600068801846FFF761FF014423F83140A6
:10CDC00038BD38B50346FFF759FF0C46A51A511A6E
:10CDD00003EBC40405444800608003EBC2006C0010
:10CDE000448023F8321018461146FFF747FF0144EC
:10CDF00023F8315038BD38B50546FFF73FFF0C46E4
:10CE0000014405EBC1035B88DA070AD42846FFF723
:10CE10007EFF21462846FFF731FF22182846FFF7FC
:10CE2000BAFF35F83410611A05EBC1035B88DB07E4
:10CE30000CD42846FFF76BFF35F834102246611AF0
:10CE40002846FFF7A8FF35F83430E41A2146284673
:10CE5000BDE83840FFF717BF61B100680439091A0F
:10CE600021F007030344C9085A8822F001025A80BE
:10CE7000FFF7C1BF704770B5056809B9002070BDE4
:10CE800001F007030B33CC0804EBD304AB689C42DE
:10CE900028BF1C4621462846FFF746FF06460028C5
:10CEA000ECD001462846FFF7E9FEA04207D9321927
:10CEB0002846FFF786FF11462846FFF7E4FE05EBFC
:10CEC000C6021046538843F0010353800430D6E76E
:10CED0001146FFF7D0BF043A2DE9F041CC1D1144B3
:10CEE00024F0070421F007010E1BF708B7FA87F2B8
:10CEF000C2F12405AD004FF000080735C2F1200251
:10CF0000ED0804604146A760C4F80C80920004F16B
:10CF1000100002F0A1FA6B0043F00103638004EB00
:10CF2000C5027B1B5900A4F800805180A21924F887
:10CF30003550A2F80280A35304EBC70329465A8850
:10CF400042F001025A802046BDE8F041FFF79BBE47
:10CF5000002070470FB407B504A951F8040B0191E4
:10CF6000F3F70CFE03B05DF804EB04B070470FB4A8
:10CF700007B504A951F8040B0191F3F7FFFD03B0C5
:10CF80005DF804EB04B07047036800220BB9184643
:10CF900070478B4210D10B6842B9426803609142DE
:10CFA00000D1436000230B60012070471360436889
:10CFB000994208BF4260F5E71A461B68E6E7038B13
:10CFC00013F0070305D10368002B0CBF00200320DA
:10CFD0007047022B05D1408BB0FA80F040098000E9
:10CFE0007047012B05D10368002B0CBF00200520E2
:10CFF00070470020704710B50C4600B111B96FF0B2
:10D00000150010BD081D00F0D2F80028F9D1A36862
:10D01000032BF6D9F3E72DE9F0410D4607461946F3
:10D02000281D90461E4600F0D6F8044638B1334617
:10D03000424629463846A446BDE8F0416047BDE86F
:10D04000F08110B4EFF31182202484F31288BFF32F
:10D050006F8F416110BC0121F3F7C2BD38B50C469A
:10D06000054658B151B10B6843B14B6833B11C222E
:10D07000002102F0F1F92C61002038BD6FF015009D
:10D08000FBE770B505460E46FFF7B5FF041E14DB3F
:10D09000EFF31182202383F31288BFF36F8F6B8B22
:10D0A0002C8B4FF6FF718B4204F0070407D182F3FB
:10D0B0001188BFF36F8F6FF00A04204670BD022CF9
:10D0C0000CD101336B8382F31188BFF36F8F002380
:10D0D000224631462846FFF79EFFEEE7062C14D87D
:10D0E000DFE804F004131313041A04000023336070
:10D0F0006B683BB9C5E90066ACB902212846F3F775
:10D100006FFDDAE71E606E60F6E782F31188BFF309
:10D110006F8F6FF00404D0E782F31188BFF36F8F35
:10D120006FF08504C9E782F31188BFF36F8FC4E7FE
:10D1300010B5EFF31182202383F31288BFF36F8FB2
:10D14000048B04F00704022C0AD0012C0CBF6FF0F2
:10D1500004006FF0850082F31188BFF36F8F08E041
:10D16000438B013B9BB2438323B92146F3F738FD40
:10D17000204610BD2046EEE738B5A8B1A1B1EFF3C7
:10D180001185202282F31288BFF36F8F048BFFF783
:10D19000FBFE30B104F0070085F31188BFF36F8FF9
:10D1A00038BD6FF07700F7E76FF01500F8E703463A
:10D1B00040B1426802F00302022A06D0032A04D0DA
:10D1C000012A05D06FF0150070471A68002AF9D0BF
:10D1D00000209860704710B54268816002F0030239
:10D1E000022A03464FF0000407D0032A02D05C60F5
:10D1F000002001E018685C6010BD18685C600028C1
:10D20000F6D0FFF761FAF3E7704710B420B1446835
:10D21000C068A44610BC60474FF0FF3010BC704798
:10D2200010B420B10468C068A44610BC60474FF039
:10D23000FF3010BC704737B501230D4601AA2021ED
:10D240000446FFF7E2FF58B99DF8043065F3010387
:10D250008DF8043001AA012320212046FFF7E0FFCA
:10D2600003B030BD37B501230D4601AA2021044685
:10D27000FFF7CBFF58B99DF8043065F382038DF8B2
:10D28000043001AA012320212046FFF7C9FF03B083
:10D2900030BD08B50A4601230F21FFF7B6FF08BDD0
:10D2A00037B501230D4601AA20210446FFF7ADFF43
:10D2B00058B99DF8043065F3C7138DF8043001AAFE
:10D2C000012320212046FFF7ABFF03B030BD37B567
:10D2D00001230D4601AA22210446FFF796FF58B903
:10D2E0009DF8043065F382038DF8043001AA012310
:10D2F00022212046FFF794FF03B030BD02F0ACB806
:10D3000002F082B801460068F3F7A6BD08B5F3F74E
:10D31000D3FDBDE80840F3F7F3BD00210120F3F78A
:10D320009BBD6FF08500704761B662B680F31188CF
:10D33000BFF36F8F704772B6002383F31188BFF37A
:10D340006F8FBFF34F8F30BF62B6BFF36F8F7047E1
:10D3500072B6002383F31188BFF36F8FBFF34F8F33
:10D3600020BF80F31188BFF36F8F62B6704720280B
:10D3700009D9B0F1004F08D80138B0FA80F0C0F1F7
:10D380001F0040007047082070473E20704708B5D6
:10D39000F4F77CFA002008BD70470023038243693C
:10D3A000C3607047416A8968F4F7DCBAEFF3118211
:10D3B000202383F31288BFF36F8F00230B60436831
:10D3C00033B9C0E9001182F31188BFF36F8F704742
:10D3D00019604160F7E710B50346EFF31181202291
:10D3E00082F31288BFF36F8F006828B15C6802680F
:10D3F0001A60A04208BF5A6081F31188BFF36F8F93
:10D4000010BD027A01320272704710B508B14B6844
:10D4100043604C68002308464B60F4F721FB20462C
:10D4200010BD83680B440360704783880268194409
:10D430008180D018704730B484880568A318838031
:10D44000281930BC01F0E0BF10B5838802685C1C6D
:10D450008480D154D01810BD034600689A88401AC1
:10D4600011441860998070470268531E03608388D6
:10D470000133838002F8011C70478288521A0346E8
:10D4800082800068084418607047034600689A88E4
:10D49000521A01449A801960704710B503681C78CD
:10D4A0000121FFF7EAFF204610BD02688068101ACC
:10D4B0007047012310B50621044600F8013BF8F738
:10D4C0002BFA18B9A37963F03F03A37110BD38B5E7
:10D4D0000446807AF4F71CFA6169054649B1637A1B
:10D4E000DB0704D4436A1B6820469B6898470023E7
:10D4F000636121462846BDE8384001F098BC10B56C
:10D500000346BFF35B8F53E8000F40EA010243E894
:10D510000024002CF7D1BFF35B8F10BD01210C302C
:10D52000FFF7B3BF30B402EBC303044608469A4288
:10D5300001D130BC7047114611F8085BA54206D1F5
:10D54000018A53789942F4D330BC536818470A468D
:10D55000EDE7BFF35B8F50E8003F0B4040E800323F
:10D56000002AF8D1BFF35B8F704708B50020002177
:10D57000F4F73AFD18B1BDE80840F4F7EBBC08BD7C
:10D58000033138B5C9B205460E20F5F707F8032177
:10D5900004460C30FFF749FF01230370A0F8015047
:10D5A000204638BD70B505460E460F200421F4F71D
:10D5B000F5FF042104460C30FFF737FF0122067007
:10D5C00042704580204670BD08B5072201F04CFF2F
:10D5D000B0FA80F0400908BD18B111B10846F5F75E
:10D5E0001DB86FF01500704713B5044680B10621D1
:10D5F0006846F8F791F948B99DF80530694603F097
:10D600003F0320468DF80530FFF7E6FF02B010BD5E
:10D610006FF01500FAE7003818BF01207047034685
:10D6200010F4004F0CBF07200620DA0348BF00F0BB
:10D6300005009B0348BF00F0FB0070472DE9F74F42
:10D640008A4601904FF0FF314FF0FF30F4F74AFC6B
:10D650000446002849D020210C30FFF7E6FE2022A6
:10D66000002180464FF0000901F0F6FEDAF8007064
:10D6700008F1010B4D46DAF80420914509D30198D1
:10D6800088F800500022214603B0BDE8F04FF4F7BF
:10D6900003BD7A7897F800C0A81C81181F2908D903
:10D6A000BCF1090FC0F11F0217D1002A15DD4FF0A0
:10D6B000080CD6B2711C0BF80510691CC9B20236F1
:10D6C0000BF801C079685BFA80F02E4401F09CFEF3
:10D6D000F5B209F101090837CDE72046F4F7C0F9A2
:10D6E0006FF0150003B0BDE8F08F6FF06800F9E748
:10D6F000012303FA01F15AB1BFF35B8F50E8003FF9
:10D700000B4340E80032002AF8D1BFF35B8F70472B
:10D71000C943BFF35B8F50E8003F0B4040E8003245
:10D72000002AF2D0F7E770B5064686B00D464FF0F6
:10D73000FF304FF0FF31F4F7D5FB0446B0B10C30A9
:10D7400095B10121FFF780FE06F1100203A92046E2
:10D7500000950823F4F7B4FB0022214642F20A00A8
:10D76000F4F79AFC06B070BD2946EBE76FF068004D
:10D77000F8E7183001F020BCF5F792BAFDF738BF92
:10D780000369C9B20C2201FB0233186C00F00700D8
:10D79000704770B5C9B20369EFF31185202484F393
:10D7A0001288BFF36F8F0C2606FB0134246C14F033
:10D7B000C00408D0A24206D085F31188BFF36F8F52
:10D7C0004FF0FF3070BD06FB013301221A6485F370
:10D7D0001188BFF36F8F436803EBC1035B68984701
:10D7E0000020EFE78022FFF7D4BFF8B5069F046959
:10D7F000C9B2EFF31186202585F31288BFF36F8F2E
:10D800000C2505FB0144256C05F0070CBCF1010F4C
:10D810000CD1276486F31188BFF36F8FC4E90E2300
:10D82000436853F8313098470020F8BD05F0C00533
:10D83000AF4286F31188BFF36F8F0CBF6FF0770094
:10D840004FF0FF30F1E713B580240094FFF7CDFFD0
:10D8500002B010BD10B40069CBB21C2403FB04005D
:10D86000002110BC1047002001F081B81046FDF7E0
:10D87000BFBE43685B68D3F810350B60002070476B
:10D8800043685B6802EA010021EA0201C3F8080567
:10D89000C3F80C150020704743685B680020C3F88C
:10D8A0000815704743685B680020C3F80C15704783
:10D8B00043685A68D2F8043521EA03000B40C2F8E5
:10D8C0000805C2F80C350020704710B50369586888
:10D8D000F8B1884219D19C6808685860A14200D10B
:10D8E0009860002008602AB15A680A609A685960F6
:10D8F00002B99960002010E0814206D108682060DA
:10D9000098688142EDD19C60EBE7044600680028EE
:10D91000F2D1002AE8D16FF0150010BDFDF7A2BECC
:10D920001FB5CDE9011202228DF80C209DF80C20C4
:10D93000816842F002028DF80C208C68012201A956
:10D94000A04704B010BD83880068FFF7E9BF07B5A2
:10D95000130A8DF804108DF8062001A903228DF812
:10D960000530FFF7F0FF03B05DF804FB2DE9F84345
:10D97000064689461446984601F031FB00BB75689F
:10D98000366906F11C074FF0FF324FF0FF3338467F
:10D99000FFF7C4FFB28A544004EA090482EA08028D
:10D9A0005440A4B2281D22461021FFF7D0FF05469F
:10D9B00000B9B4823846FDF71BFE2846BDE8F8835F
:10D9C0006FF00A05F9E700220B461146FFF7CEBFBC
:10D9D00000231A46FFF7CABF0A460023FFF7C6BF57
:10D9E0000023FFF7C3BF10B586B000238DF80430C5
:10D9F0000B885BBAADF805304B885BBAADF80730E1
:10DA00008B885BBAADF80930CB885BBAADF80B30C8
:10DA10000B895BBAADF80D304B895BBAADF80F30AE
:10DA20008B895BBAADF81130CB895BBAADF8133096
:10DA30000B8A59BAADF81510041D62B11A461021AF
:10DA40002046FFF784FF20B9112201A92046FFF7E5
:10DA50007AFF06B010BD1322F7E7F7B546680569EF
:10DA6000706801F0BDF8002855D041F27D22706841
:10DA70003389ADF8042001A90222FFF751FF0446C3
:10DA8000002841D143F27D4270683389ADF804200B
:10DA900001A90222FFF744FF0446A8BB002163202E
:10DAA00001F053FB21461222281D01F0D5FC4EF255
:10DAB000E0032C83AC76AB8244F21E02706833899B
:10DAC000ADF8042001A90222FFF72AFF27460446E9
:10DAD000D0B90436AA8A10213046FFF738FF044631
:10DAE00090B96A8A0E213046FFF731FF044658B9D3
:10DAF00049F61F03022201A93046ADF804308DF823
:10DB00000670FFF720FF044605F11C00FDF770FDCD
:10DB1000204603B0F0BD6FF01204F5E72DE9F74F92
:10DB20000D46D0F804900469174601F058FA824671
:10DB3000002840F0848004F11C084FF0FF324FF0C1
:10DB4000FF334046FFF7EAFE0126E28AAE40B6B256
:10DB500022FA05F56FEA060BE9071FFA8BFB4CD496
:10DB6000E38903EA0B02E281BA0758D46389F80615
:10DB70004CBF334303EA0B036381A389B9064CBF4F
:10DB8000334303EA0B03A381A388FA034CBF03EAE0
:10DB90000B033343BD03A380638A4AD503EA0B0317
:10DBA0007803638240D5A38A0BEA0303A3824FF074
:10DBB000010AB4F81930FA054CBF334303EA0B03EA
:10DBC000A4F819305246211D4846FFF70CFF0546C0
:10DBD000F0B922238DF80430237E8DF80530B4F897
:10DBE000193004225BBA0DEB020109EB0200ADF81B
:10DBF0000630FFF7A8FE05460AE002EA0B02E282C1
:10DC0000202109F10400FFF7A2FE05460028A7D055
:10DC10004046FDF7EDFC284603B0BDE8F08F7D07D8
:10DC20000AD53343E381A1E73903C2D5A38A33433D
:10DC3000BCE733436382BCE76FF08505E8E76FF02C
:10DC40000A05E8E7F0B589B0476805690E4601F0B6
:10DC5000C6F9044688BB1C3528464FF0FF324FF00A
:10DC6000FF33FFF75BFE0DF1050202920122786897
:10DC7000039210230DF106028DF8053007213B8930
:10DC8000059202228DF8104006928DF81C109DF826
:10DC90001C10846811438DF81C10A46802A9A047C9
:10DCA000044620B9BDF806305BBA9BB23360284603
:10DCB000FDF79EFC204609B0F0BD6FF00A04F9E7BD
:10DCC00000F05FB8002201210320F3F7D3BB00224C
:10DCD00001210420F3F7CEBB38B5044605690122C3
:10DCE0001146284601F0B1F8012205F11800002183
:10DCF00001F0ABF82046BDE83840FAF789BA006970
:10DD0000FDF7B0BC0069FDF773BC13B501AA04466A
:10DD100000F040F8002805DB019B2268197918689B
:10DD2000FAF794FA02B010BDCA07436805D4C1F3EC
:10DD30004201012904D0022909D06FF01500704773
:10DD40001B684FF0CC72C3F82425002070471B6875
:10DD50004FF0C862F7E710B544680021606AFFF72A
:10DD6000D4FF2046BDE81040FCF7FABE10B5446869
:10DD70002046FCF705FF606A0121BDE81040FFF76F
:10DD8000C4BF10B54468FFF7F1FF2046FCF73AFF27
:10DD9000002010BD30B543681360057A446804EB79
:10DDA000C504A34202D36FF0010030BD5C798C4200
:10DDB00001D00833F0E70020F7E710B504692046EA
:10DDC00000F05BFF0023636110BDF8B587687C68D5
:10DDD00006469CB1436893F82630DB071DD40569DD
:10DDE0004FF0FF334FF0FF322846FDF707FB6B691A
:10DDF000002B05DC00242846FDF778FB2046F8BD03
:10DE0000013B6B61002BF5D17B6830469847041EBF
:10DE1000BEBF6B6901336B61EDE70024EEE7F0B440
:10DE2000D0E901631B693BB177688F4208DB356835
:10DE3000954205DCF0BC18476FF05700F0BC704706
:10DE40006FF01500FAE7F0B4D0E901631B6A3BB14B
:10DE500037698F4208DBF568954205DCF0BC18474E
:10DE60006FF05700F0BC70476FF01500FAE770B420
:10DE7000D0E90162956A03460C46A5B196F82420C4
:10DE800012B92B4670BC1847306A024410F8011BC7
:10DE9000A14202D121461846F3E79042F6D16FF035
:10DEA000850070BC70476FF05700FAE72DE9F34129
:10DEB000D0E901470E4694F825100569FF298046F0
:10DEC0000FD194F82610C1F38101022914D0D8F89B
:10DED00008301B6B003918BF01214BB96FF0570098
:10DEE00003E0FFF7C4FF0028EBDA02B0BDE8F081E1
:10DEF000404698470028F8DBA268B2F1004F05D0F1
:10DF000011464046FFF78BFF0028EEDB6269B2F155
:10DF1000004F05D011464046FFF795FF0028E4DB8F
:10DF20002368B3F1004F14D0D8F808305B69002B98
:10DF3000D4D001A9404698470028D6DB2268019B2F
:10DF40009A421CDD11464046FFF769FF002805DABA
:10DF5000CBE762686FF000439A42E5D19EB994F82E
:10DF600026309B0716D03B68404698470028BCDB0C
:10DF7000A069FAF7F7F96B6901336B610AE062682F
:10DF80009342EBDDDEE76B6901336B6194F8263079
:10DF9000DA0601D40020A8E74046FFF716FFA4E701
:10DFA000012303FA01F103691B68194218BF82F0CB
:10DFB000010212B18368DB68184783681B69FBE7BD
:10DFC00008B54368986A38B193F82C100122FFF71E
:10DFD000E7FF00EAE07008BD6FF08500FBE74368EB
:10DFE0001868B0F1004018BF01207047034608468A
:10DFF00031B95B681B68B3F1004F01D01360704703
:10E000006FF015007047F7B544680546FFF7D5FE79
:10E01000A06A00283AD000F0E3FD002838D0E38D54
:10E02000A06A94F82C1043F400320769D0F808C0B5
:10E0300013F0010F4FF001063B6806FA01F614BF1A
:10E040003343B3433B60DCF800309847002821DBC2
:10E05000A06A94F82C400669836801A95B68984718
:10E06000002809D016DB011E18BF0121284603B085
:10E07000BDE8F040FFF71ABF019B32685A40012308
:10E08000A3401A4214BF01200020ECE70146EDE74F
:10E090006FF0120003B0F0BD4368986A20B193F8A6
:10E0A0002C100022FFF77CBF6FF0850070470346FD
:10E0B0000A4600681979012303FA01F103691B6814
:10E0C000194218BF82F0010212B18368DB68184759
:10E0D00083681B69FBE7F0B403460A461979DB88BD
:10E0E00000681343066987683468DA0748BF83F419
:10E0F000402301258D4023F48012DB074CBF2C43C5
:10E10000AC4334603B68F0BC1847014640F2E7304E
:10E1100008B54FF47A72002300EBC1304914F2F7CE
:10E120002FF8BDE8084001F010B81FB5CDE9011285
:10E1300002228DF80C209DF80C20816842F002022A
:10E140008DF80C208C68012201A9A04704B010BDF5
:10E1500010B586B0009203930122089B01920493AC
:10E16000002207238DF808208DF814309DF8143014
:10E17000826843F002038DF8143094680B46022243
:10E180006946A04706B010BD7FB501260096002362
:10E1900081888DF80F3004460DF10D0300680DF1F4
:10E1A0000F02FFF7D5FF002811DB9DF80D50EB079C
:10E1B0000FD50096E0238DF80F30A18820680DF16F
:10E1C0000E030DF10F02FFF7C3FF002804DA6FF012
:10E1D0000405284604B070BD9DF80E3045EA0325BD
:10E1E000F7E710B518300C46FFF761FF24B1322075
:10E1F000BDE8104000F0D8BC1420F9E7F0B546683F
:10E20000046987B0022300270546012130468DF8B6
:10E210000F30CDE90477FFF7E4FF0823B1880093BE
:10E22000306804AB0DF10F02FFF792FF3946064646
:10E230006868FFF7D6FFBE421CDBBDF810104BBA72
:10E240002380BDF812305BBA6380BDF81430E380E0
:10E25000BDF8162052BAA280627A112A02D809B1FA
:10E2600043F0080313F0080F0CBF6FF00A00002002
:10E2700007B0F0BD6FF00400FAE710B586B0009269
:10E2800003930122089B01920493002207238DF837
:10E2900008208DF814309DF81430826843F0020392
:10E2A0008DF8143094680B4602226946A04706B0E8
:10E2B00010BD1FB500938DF80F10134681880068BC
:10E2C0000DF10F02FFF7D9FF05B05DF804FB30B583
:10E2D00089B0054608468DF8100011460DF1110071
:10E2E0001A461C4601F090F804AA01920134022259
:10E2F0002868AB8802948DF80C209DF80C2081686A
:10E3000042F002028DF80C208C68012201A9A0477E
:10E3100009B030BD38B5002120EAE0744FF4004563
:10E3200040F2E7304FF47A720023C4FB0501F1F7A5
:10E3300027FFBDE8384000F008BF13B50423046987
:10E3400040680DEB0302A821FEF75FFF002806DB03
:10E35000BDF804302380BDF806306380002002B091
:10E3600010BD30B5446887B005460DF10701204661
:10E37000FEF78FFF002846DB9DF80730BC2B44D109
:10E3800001212046FEF757FF00283CDB01212046F3
:10E39000FEF768FF002836DB01212046FEF780FFEC
:10E3A000002830DB0021632000F0CFFE68682C6974
:10E3B000102302AAB021FEF728FF002823DBBDF8B6
:10E3C0000830A3809DF80D309DF80A20190201F451
:10E3D00040710A43E2809B019DF80B2003F44073D7
:10E3E00013432381BDF80E306381BDF81230A38141
:10E3F000BDF81430E381BDF8163023822846FAF7C1
:10E40000F3F900EAE07007B030BD6FF01500FAE7ED
:10E4100010B551F8043C1C6958680021FAF7BEF9A0
:10E4200004F12C00BDE81040FDF79ABA38B550F859
:10E43000184C2569AB6A53B1696A20469847AB6AA4
:10E440002BB160680121BDE83840FAF7A7B938BDA3
:10E450002DE9F3414668D0F81080154604460F4672
:10E4600030460021FAF79AF9C8F828500DB3C8F8D9
:10E47000247060680121FAF791F9B069357F066967
:10E48000836801A95B68984740B9019B32685A408C
:10E490000123AB401A4214BF01200020002808DDF0
:10E4A000256960680021FAF779F905F12C00FDF77C
:10E4B00057FA002002B0BDE8F08138B504696368FE
:10E4C00004F108021D6827210723A847002804DB60
:10E4D000237A13F00F0F18BF002038BD422901D155
:10E4E000FFF7EBBF0329FBD00C290CBF6FF08500B1
:10E4F0006FF03C00704737B543681B680446984787
:10E50000002819DB2046FAF7EBF9002802DA10F1AF
:10E51000860F11D125696B680DF107029B682621D2
:10E5200020469847002805DB6B682A7DDB682021A0
:10E530002046984700EAE07003B030BDF0B40C27E5
:10E5400007FB0214866814F8045C45F0020504F821
:10E55000045CB468A446F0BC604730B589B061F093
:10E560007F0144688DF807100DF107010291012128
:10E57000606803911D46002123898DF81010CDE9B4
:10E58000052502A902228DF81C20FFF7D7FF09B04C
:10E5900030BD30B589B061F07F0144688DF8071057
:10E5A0000DF107011D460291012160682389039145
:10E5B000CDE90525002107228DF810108DF81C20CB
:10E5C00002A90222FFF7BAFF09B030BD1FB54368A8
:10E5D0008DF80120022258688DF800101B890292E4
:10E5E0008DF80C2001A90122CDF804D0FFF7A6FF79
:10E5F00005B05DF804FB10B588B043688DF80710CE
:10E600000DF107010291012158681B890391CDE9A1
:10E61000052107228DF81C200024022202A98DF872
:10E620001040FFF78BFF08B010BD2DE9F04798466A
:10E63000436888B0D3F8049093F808A08DF80410CC
:10E64000002301278DF810300DF10303CDE90537C4
:10E6500007230E46144601AD8DF81C3002225346A6
:10E6600002A9484602950397FFF768FFB8B99DF8DD
:10E67000032022EA040304EA08041C43A2420ED049
:10E68000022303938DF810303A46534602A94846B8
:10E690008DF804608DF805400295FFF74FFF08B034
:10E6A000BDE8F08710B586B0009203930122089B65
:10E6B00001920493002207238DF808208DF814306E
:10E6C0009DF81430826843F002038DF8143094688A
:10E6D0000B4602226946A04706B010BD10B543683C
:10E6E00004699988186886B028238DF80F300523AF
:10E6F00000930DF10F0204ABFFF7D4FF002810DBED
:10E700009DF812309DF811201B0443EA02239DF866
:10E71000102013432360BDF81330A380002006B0FF
:10E7200010BD6FF00400FAE72DE9F04389B001272E
:10E73000144699464FF0100800970DF10F0305AAF3
:10E7400005460E468DF81480FFF7ACFF00BB9DF820
:10E750000F2022EA040304EA09041C43A24217D052
:10E760000DEB0803059302238DF810808DF81140FE
:10E7700006938DF81C309DF81C30AA6843F0020304
:10E780008DF81C30946833463A4605A92846A047C0
:10E7900009B0BDE8F08330B5436885B00446186819
:10E7A00000F01EFA50B365680F238DF80F30012377
:10E7B0002868A98800930DF10F020DF10E03FFF7F1
:10E7C00071FF002803DB9DF80E30B12B03D06FF0F2
:10E7D000040005B030BD6068302301790068702204
:10E7E000FFF7A2FF0028F2DB0223297928681A46E6
:10E7F000FFF79AFF0028EADB0020EAE76FF012003B
:10E80000E7E74379014623B151F8060B83681B689B
:10E8100018476FF08500704737B5212945680469AE
:10E8200001D0422914D16846D4E9062300F03AFD0C
:10E83000DDE9000100F089FC2846FFF7E2FF48B956
:10E84000286883685B68214603B0BDE830401847FC
:10E850006FF0850003B030BD43681B68D3F88004B7
:10E86000C3F88004704742681368D3F8100150B1B0
:10E87000D269002012780A70C3F81001D3F8102171
:10E8800001221A6070474FF0FF307047026803465C
:10E89000D2F8580140B95B68DB0706D4D2F82001F2
:10E8A000003818BF012070470120704743681B687B
:10E8B000D3F80423D20517D5D3F82021A2B1EFF362
:10E8C0001182202181F31288BFF36F8FD3F82011BA
:10E8D00031B10021C3F82011D3F820110121D960F2
:10E8E00082F31188BFF36F8FD3F85831704713B597
:10E8F00001AA0446FFF74EFA002805DB019B2268B7
:10E9000019791868F9F7A2FC02B010BD6FF0850004
:10E91000704700F150039B009BB203F1804303F565
:10E92000883300221A601B6870474FF08053D3F879
:10E930003001421C04BF4FF0704393F8E00F831F77
:10E94000584258417047004700F02EB9C840C043B4
:10E9500000F001007047C00000F1804000F5F83081
:10E96000C0F81015C0F814257047FBF767BAFAF71E
:10E97000E9BD036803F01F025B0902600CBF4FF0A2
:10E98000A04000207047F7B5019001A8DDE90847D5
:10E9900016461D46FFF7EDFF019BB6F1000C18BFB0
:10E9A0004FF0010C00EB83000B1E18BF0123002D5C
:10E9B00043EA4C0314BF4FF00C0C4FF0000C002C3A
:10E9C00043EA0C0314BF4FF4E06C4FF0000C002F2F
:10E9D00043EA0C03D0F8002714BF4FF4403C4FF03B
:10E9E000000C43EA0C0322EA030301B109780EB1DB
:10E9F0003678760019430DB12D78AD0031430CB156
:10EA00002478240229430FB13F783F040C433C4350
:10EA1000C0F8004703B0F0BD1FB50DF10F0301931F
:10EA200000238DF80F1000931A461946FFF7ABFF2D
:10EA300005B05DF804FB024611F0010007D04FF06D
:10EA4000A041D1F820351360C1F8203503B900206A
:10EA50007047FAF745BFFAF723BFA1F5807310B5E9
:10EA60009B08012404FA03F318400CD001F1804103
:10EA700001F5E041086830B10020086009681168BC
:10EA800019431160204610BD08B500210120FBF795
:10EA9000ABFA0028F9D008BD91F820200346032ADC
:10EAA00029D8DFE802F0212519028A68500304D52D
:10EAB000D3F84C250869904207D18A6852031AD4CA
:10EAC000D3F84C258969914215D000200622C3F85D
:10EAD0000005C3F800257047D3F84C25086990421B
:10EAE000F3D1D3F83C25EDE7D3F84C250969EAE7E3
:10EAF000D3F83C25FAE70120704730B5A2F58075C0
:10EB0000AD080124AC400C4207D0815829B1002146
:10EB1000815082581A6822431A6030BD13B5002311
:10EB20000C4601934FF4A47201ABFFF7E6FF2146B8
:10EB30004FF48272FFF7E1FF21464FF49272FFF724
:10EB4000DCFF21464FF4A872FFF7D7FF21464FF4B0
:10EB5000A672FFF7D2FF21464FF4B072FFF7CDFF48
:10EB60004FF4AE722146FFF7C8FF019802B010BD06
:10EB7000036803F01F025B0902600CBF4FF0A04066
:10EB80000020704707B5019001A8FFF7F1FF019A37
:10EB900001239340C0F8083503B05DF804FB08B5C5
:10EBA000FCF7CEFA002008BD08B1F2F77FBF70472E
:10EBB00010B5436904463BB90020E268537843F03E
:10EBC00001035370404210BD98470028F4D000283C
:10EBD000B8BF4042E368FF28A8BFFF201870ECE7E9
:10EBE00040B1C368587810F001001EBF1878B0FA21
:10EBF00080F040097047EFF31183202383F31288DC
:10EC0000BFF36F8FFEE708B5FFF7F5FF10B400F113
:10EC10000C04C0E9034410BCFEF75DB938B50446E6
:10EC2000EFF31185202383F31288BFF36F8FFEF774
:10EC300013F904F10C0000F074FA30B1294604F124
:10EC40001400BDE83840FDF7F7B885F31188BFF32D
:10EC50006F8F38BD08B52024EFF3118384F3128839
:10EC6000BFF36F8FFEF767FBF6E790F90E308B422C
:10EC700001D0FDF76FB80020704703460020C3E9BC
:10EC80000200C3E900337047D0E9003213605A60D4
:10EC9000427B002322F00202C0E90033427383600A
:10ECA00070472DE9F843914604469DF820200D4613
:10ECB00000F10807EFF31186202181F31288BFF3DA
:10ECC0006F8F02B14568D4F80880474518D0B8F175
:10ECD000000F15D04046FFF7D7FF08F1180000F0ED
:10ECE0008EFA0023C8F87C30C8F81090404600F037
:10ECF000B9F938463146FDF79FF80020BDE8F883A2
:10ED0000A3B10820FDF72EFD002838D00122C0F85D
:10ED100004900260016801F003015DB922680A43B2
:10ED20000260626820606AB960600BE0C9F8003078
:10ED30004846EFE72A68032A16D80160616869B976
:10ED4000C4E90000042104F1100000F037FB0028A2
:10ED5000CFD186F31188BFF36F8FCFE70A6802F037
:10ED6000030202430A60DFE722F003020A43026063
:10ED70002A6802F0030240EA02032B60E2E76FF028
:10ED80000B00E6E710B5044630B10268930703D0E4
:10ED9000446809B100F031FB204610BD0023C0E9F2
:10EDA000003300F10803C0E9023300F11003C0E9A9
:10EDB00004337047F8B500F10806EFF311872023FC
:10EDC00083F31288BFF36F8F8568AE4200F11004A1
:10EDD00017D0B5B12846FFF757FF05F1180000F02E
:10EDE0000EFA00232846EB672B6100F03BF908215F
:10EDF000204600F0E3FA39463046BDE8F840FDF71A
:10EE00001BB80821204600F0D9FA0028F3D187F377
:10EE10001188BFF36F8FF8BD07B50123009300235E
:10EE20000A461946FFF73DFF03B05DF804FB07B53E
:10EE300000230A4600931946FFF733FF03B05DF83D
:10EE400004FB00680021FFF79DBF5AB18A4209D335
:10EE500000F11003C0E90212C0E90000C0E9043368
:10EE6000002070476FF015007047026801238B4047
:10EE700022EA0303036022FA01F000F00100704768
:10EE800010B5032104460C30FFF7EFFF30B104F159
:10EE9000100000F0B4F9B0FA80F0400910BD20B1C4
:10EEA000002211468C3000F071B9704770B5C3680C
:10EEB000C3F340069B07044616D4856802210C3034
:10EEC000FFF7D3FF80B1D5F884206AB194421DD1F9
:10EED00022689EB9D5F88830C5F884209C4201D1BB
:10EEE000C5F8882000232360E36813F01F001EBFCD
:10EEF00043F00203E36040F0020070BD3260D5F8D9
:10EF00008820944208BFC5F88860EBE7164612686F
:10EF1000DBE773B50446EFF31185202383F31288F2
:10EF2000BFF36F8F0023A0F1100603210438019373
:10EF3000FFF79BFF28B1A369019301A93046FCF7B5
:10EF4000B3FC85F31188BFF36F8F02B070BD13B5AA
:10EF500001900846EFF31184202383F31288BFF356
:10EF60006F8F01A9FCF7A0FC84F31188BFF36F8FAA
:10EF700002B010BD10B5FFF7EAFF041E08DDEFF385
:10EF80001180202383F31288BFF36F8FFCF766FF95
:10EF9000204610BD08B5A022002100F05DFA08BD92
:10EFA00038B5302204460D46002100F055FA4FF4E2
:10EFB00080736560E36038BD38B50446EFF31185B2
:10EFC000202383F31288BFF36F8FFFF759FF20468A
:10EFD000FFF76CFF85F31188BFF36F8F38BDEFF338
:10EFE0000580003818BF012070476FF05700704748
:10EFF000D0E9003213605A600023C0E90033704743
:10F0000008B5FFF7F5FF437B23F0020343730023AA
:10F01000836008BD38B504460D46FCF7F9FD637BF7
:10F0200043F002036373E5B1A5602B689D4209D1EB
:10F030006B68C4E900531C606C6012E06A689A4215
:10F04000F6D01B68002BF3D094F90E2093F90E1024
:10F050008A42F3D09142F1DD5A68C4E9003214606B
:10F060005C6038BD10B5EFF31184202383F3128860
:10F07000BFF36F8FFCF78AFD84F31188BFF36F8FA6
:10F0800010BD08B5EFF31181202282F31288BFF37F
:10F090006F8F83680BB1FFF7B3FF81F31188BFF364
:10F0A0006F8F08BD10B50146EFF31184202383F361
:10F0B0001288BFF36F8F437B13F0280F0AD1836848
:10F0C0000BB1FFF79DFF4B7B23F004034B73084606
:10F0D000FCF75CFD84F31188BFF36F8F10BD012135
:10F0E0001838FFF7DFBF08B50346EFF31181202280
:10F0F00082F31288BFF36F8F0068834207D008B194
:10F10000FFF77EFF81F31188BFF36F8F08BD0020EA
:10F11000F8E710B5FFF7B5FFBDE81040183000F074
:10F120006EB838B504680546AC424FF0000000D117
:10F1300038BD002CFCD02046FFF7EBFF2046FFF740
:10F1400091FF2C680120A542F1E770B505460E46F7
:10F15000FCF72CFFB6F1FF3F08BFB5F1FF3F0446B7
:10F16000284612D04FF47A7147F6FF730022C4FB91
:10F170000132D80B40EA4240B0F1004F4FEAD232A0
:10F1800072F1000228BF6FF0004070BD38B5EFF398
:10F190001185202383F31288BFF36F8F0468A04288
:10F1A00012D09CB1E16722612046FFF729FF04F1EC
:10F1B000180000F024F82046FCF7E8FC012085F355
:10F1C0001188BFF36F8F38BD0020F8E72046F6E7BF
:10F1D00008B50246FDF788F870B1D0E904319B1AF2
:10F1E00061EBE272B3F1004F72F1000104DA002A20
:10F1F000ACBF1846002008BD6FF00040FBE738B5F3
:10F200000246EFF31185202383F31288BFF36F8F3B
:10F210000368CBB1FDF768F804461046FDF776F8B1
:10F2200000224FF000438442C0E9042306D1FDF7D9
:10F2300063F8FFF7CDFF0021F9F7DEFF002085F32B
:10F240001188BFF36F8F38BD6FF01500F7E708B571
:10F25000FDF768F908BDFDF765B9B3F1FF3F08BFD9
:10F26000B2F1FF3F70B506461D46144614D01A434E
:10F2700016D0002B08DBFDF755F9041941EB050109
:10F28000C6E90041304670BD6FF001031C1B4FF012
:10F29000FF3363EB0501F3E74FF0FF342146EFE75F
:10F2A0000024FBE7B3F1FF3F08BFB2F1FF3FF8B521
:10F2B000074616461C4610D054EA020311D0FDF74B
:10F2C00031F9B0420A46A14103460AD2F31A64EB6F
:10F2D0000204C7E900343846F8BD4FF0FF331C463E
:10F2E000F7E70023FBE70023C0E9081200F118024A
:10F2F000C0E90622C0E9003303634363704710B5D9
:10F300000446FFF77CFFA8B9636A0BB12046984713
:10F3100004F11800FFF7E7FE60B1FFF7A3FEEFF37B
:10F320001180202383F31288BFF36F8FBDE8104054
:10F33000FCF794BD10BD2DE9F041846805460E46EA
:10F34000D4B16378012B22D114F8533C9A0711D51C
:10F35000A4F160073846FFF7DCFE082E0CBF6FF003
:10F3600003030023E36114F8533CDB0602D1384663
:10F37000FFF778FE00232370EB68C3F38632164351
:10F38000002066F39433A860EB60BDE8F081022BA7
:10F39000F0D12378002BEDD054F8048CB8F1000F95
:10F3A000E8D004F11400FFF72AFFA4F114070023AA
:10F3B000E36239464046FFF7CAFDDBE738B5EFF3B5
:10F3C0001185202383F31288BFF36F8F0468A04256
:10F3D00011D0D4E9003213605A600023C4E900332D
:10F3E0002046FFF7A8FF85F31188BFF36F8F201E1B
:10F3F00018BF012038BD0024F5E720B1011F50F8E7
:10F40000040CFFF70BBC70470A44914200F1FF3334
:10F4100000D1704710B511F8014B03F8014F91422C
:10F42000F9D110BD884210B501EB020402D9844223
:10F43000234607D8431EA14208D011F8012B03F838
:10F44000012FF8E7024401468A4200D110BD13F8AB
:10F45000014D02F8014DF7E702440346934200D103
:10F46000704703F8011BF9E710B5013902449042D7
:10F4700001D1002005E0037811F8014FA34201D02B
:10F48000181B10BD0130F2E710B5024601448A4254
:10F49000134603D01C780132002CF8D1181A10BD85
:10F4A000F0B5C3F137070446FFB203F01F0310465F
:10F4B000082BE6B233D0102B3ED06508A40844EAEE
:10F4C000817445EAC1752D194FEA910242EB510250
:10F4D000290941EA02716D1842EB1212290A41EA28
:10F4E00002616D1842EB1222290C41EA02416D18AB
:10F4F00042EB1242AD1842F10002EC0844EA4274B9
:10F50000D10804EB8402A6EB4205EDB2092D0CD91B
:10F510000134A5F10A0541F10001EDB212E0E40861
:10F5200044EA417406F00705C908303554EA01027F
:10F5300000F8015BBCD1F0BD240944EA017406F077
:10F540000F050909092D84BFED19EDB2EDE70000A3
:0CF550000148006870470000100D00200A
:08F55C00580CFF7F01000000C4
:10F564009D1A000000000000000000002CF60000BE
:10F574009FEB000000000000D9B300000000000071
:10F58400000000004CF60000000000006CF60000D3
:10F59400000000008CF60000D97900000000000093
:10F5A4002590000000000000B518000000000000D5
:10F5B40031B700000000000000000000CCF600009D
:10F5C40000000000ACF60000000000004CF7000052
:10F5D400000000000CF70000000000002CF7000001
:10F5E40000000000ECF60000000000006CF70000D2
:10F5F400C11A000000000000000000002CF8000008
:10F6040000000000ACF70000000000008CF70000D0
:10F6140000000000CCF70000000000000CF800001F
:08F6240000000000ECF70000FB
:10F62C005105010008FD0000ACFA0000080800209C
:10F63C0018170020D5760000000000000000000024
:10F64C007005010018FD0000BCF900000C0800203A
:10F65C00C0170020897E00000000000000000000A0
:10F66C00600501000000000090F900000A0800206D
:10F67C006C170020ED7B0000000000000000000073
:10F68C003B060100F4FE000004FB000024080020EF
:10F69C00F4180020A98C00000DE900000000000007
:10F6AC00AB050100F4FD0000C8FA000014080020AE
:10F6BC003418002007E000000000000000000000EB
:10F6CC00B805010024FE0000C8FA0000160800204E
:10F6DC004C18002007E000000000000000000000B3
:10F6EC0018FC000000000000A0FA00000408002034
:10F6FC004815002000000000000000000000000081
:10F70C00440501000000000084F9000006080020F8
:10F71C0000000000E1730000000000000000000089
:10F72C00890501003CFD0000E0F9000010080020F4
:10F73C00CC170020D9DC0000C1DC00000000000068
:10F74C009605010098FD0000E0F900001208002069
:10F75C0000180020D9DC0000C1DC00000000000013
:10F76C007E05010030FD000098F900000E08002015
:10F77C009C0700205BDA0000000000000000000085
:10F78C00CA05010054FE0000F8F90000180800201A
:10F79C004E1A0020E1830000000000000000000071
:10F7AC00D40501000000000068FA00001A080020CF
:10F7BC0064180020CD86000000000000000000004E
:10F7CC00E205010074FE000014FA00001C08002081
:10F7DC009818002063E30000000000000000000007
:10F7EC00F40501009CFE000030FA00001E08002009
:10F7FC00D4180020F7E40000000000000000000016
:10F80C0000060100C0FE00004CFA00002008002099
:10F81C00EC18002097E7000000000000000000003A
:10F82C0035060100C8FE000084FA00002208002002
:10F83C00780A0020D58A00000000000000000000BB
:10F84C003997000047E90000000000001BD30000BE
:10F85C008CF60000ADE80000DDAF000047E90000C9
:10F86C00EDAF000047E90000000000001BD30000D2
:10F87C00E99C000047E90000A1A6000047E9000050
:10F88C00000000001BD30000000000001BD3000090
:10F89C00000000001BD300000000000039590000DC
:10F8AC00ACF700003D8600006C1700205D7C00006A
:10F8BC0000000000816F0000000000001BD300005E
:10F8CC00000000001BD300000000000005910000A8
:10F8DC00000000001BD30000000000001BD3000040
:10F8EC00000000001BD30000000000001BD3000030
:10F8FC00000000001BD30000000000001BD3000020
:10F90C000000000069590000000000001BD300003B
:10F91C00000000001BD30000000000001BD30000FF
:10F92C00000000001BD30000000000001BD30000EF
:10F93C00000000001BD30000000000001BD30000DF
:10F94C00000000001BD30000000000001BD30000CF
:10F95C00000000001BD30000000000001BD30000BF
:10F96C00000000001BD30000000000001BD30000AF
:08F97C00000000001BD3000095
:0CF984004D7000002974000058020000C3
:08F99000957B0000ED7A0000F8
:10F998001DDB000045DC0000E1D90000D9D90000DA
:10F9A800D1D90000C7D90000000000000000000005
:10F9B800000000000D7D000073D8000081D8000011
:10F9C80099D80000A5D80000B1D80000D17E000069
:08F9D800CBD800000000000084
:10F9E00029DD000000000000198000000000000078
:08F9F000000000006581000029
:10F9F800000000000000000000000000FDE1000021
:10FA080091830000000000000000000000000000DA
:10FA18000000000051E400003BE300000D870000F7
:10FA28000000000000000000F107000000000000D6
:10FA380000000000DDE400008D88000000000000E8
:10FA480000000000000000000000000000000000AE
:10FA5800DDE60000BD890000000000000000000095
:10FA680000000000000000000000000055860000B3
:10FA780011860000000000000000000000000000E7
:10FA8800000000000000000019E80000118A0000D2
:08FA9800000000000000000066
:0CFAA0005D4D0000214C0000A94B00004F
:10FAAC002D770000E5D7000047D8000000000000CB
:0CFABC0081D700000000000000000000E6
:10FAC800C1DF000099E00000DFDF0000EDDF00008B
:10FAD800000000000000000000000000000000001E
:10FAE800000000000000000000000000000000000E
:0CFAF80000000000000000000000000002
:0CFB040067E80000F18B000059E80000E9
:10FB10000000000000000000A0000000F000000055
:10FB200000000000000106020100000000000000CB
:10FB30000338FDD87047000090010000FF0E000060
:10FB4000F4070020C00400200000000000000B06A5
:10FB50000200000058FB00000000000087030100C5
:10FB600024000206000000208F0301001E000B117C
:10FB7000411900000000000099D3000070FB000054
:10FB80008CFB00004700000000000000C037002090
:10FB900070FB0000A0FB00002E0000000000000031
:10FBA000A03B002070FB0000B4FB0000020100003D
:10FBB00000000000743C00200E030000312500000E
:10FBC0000F0400006D2500003E010000C91B00006D
:10FBD000FF010000891B00003E010000A91B00007E
:10FBE000100100001DD5000070FB0000F8FB0000B4
:10FBF0004700000000000000903D002042542043D8
:10FC0000544C5220525820707269000042542043D4
:10FC1000544C52205258000062745F6863695F63FD
:10FC20006F6E74726F6C6C65720000005A6570685C
:10FC30007972204F532076342E332E30000000008E
:10FC4000574553545F544F504449522F7A6570685A
:10FC500079722F7375627379732F626C7565746F27
:10FC60006F74682F636F6E74726F6C6C65722F6C3B
:10FC70006C5F73772F6E6F726469632F6C6C6C2F7F
:10FC80006C6C6C5F6164762E6300000030000000D5
:10FC9000415353455254494F4E204641494C205BF5
:10FCA00025735D20402025733A25640A000000007A
:10FCB0000925733A2041637475616C204556454EA1
:10FCC000545F4F564552484541445F535441525446
:10FCD0005F5553203D2025750A0000007072657045
:10FCE0006172655F636200000000010000000000B7
:10FCF0000001010000000000010304055D76000022
:10FD00002D76000000000000D9770000A1760000E9
:10FD10006977000067D80000FFFFFFFF0000005078
:10FD20000000000000000000006000400000000033
:10FD3000FFFF00004CF700003E00000000400040C4
:10FD4000010000000000000000000000000040066C
:10FD500000000101E17F000010000000CFDC000086
:10FD60006CFD0000651A0020FF000000004000400C
:10FD700078FD00000200000090FD0000020000007D
:10FD800088FD0000020100000E80000C0F80000BB7
:10FD90000E00000C0F00000B0030004000000000BF
:10FDA000000000000000000000004006000001010B
:10FDB000E17F000010000000C5DC0000C8FD00006D
:10FDC000751A0020FF00000000300040D4FD000044
:10FDD00002000000ECFD000002000000E4FD000055
:10FDE000020100000780000C0880000B0700000CD7
:10FDF0000800000B00000080FFFFFF7F0000008074
:10FE000000000080FFFFFF7F000000800000000076
:10FE100000000000C505010000FF08004CF60000CE
:10FE20001D00000000000080FFFFFF7F0000008039
:10FE300000000080FFFFFF7F00000080E80300005B
:10FE400000000000C505010000FF0A004CF600009C
:10FE50001E0000004CF700005A00000000000000E7
:10FE6000000000006CF700000B0001006CF70000C0
:10FE70000C000100CFE20000B3E2000015E3000037
:10FE800084FE00004CF700005F0000004CF600000C
:10FE90001800000000000000000000009D89000024
:10FEA0002CF70000190000000800000093E5000096
:10FEB0005BE50000F7E50000CDE500002BE6000063
:10FEC0004CF700005C0000000CF70000040000008C
:10FED00000000000000000000000000080A21900E7
:10FEE00020BF02006CF70000040000006400000066
:10FEF00000000000002000400100000000000000A1
:10FF000014FF00000000D60100000000861A002047
:10FF1000851A00200020004020FF000002000000A1
:10FF200038FF00000200000030FF00000201000066
:10FF300003800000028000010300000002000001B5
:10FF400064F5000064F50000A4F50000ACF50000C5
:10FF50002CF600002CF600008106010000010000D4
:10FF600000000000000001000A00190032006400D7
:10FF7000C800900154064005001572302F61313AD7
:10FF80002020307825303878202072312F61323AA5
:10FF90002020307825303878202072322F61333A93
:10FFA00020203078253038780A0072332F61343AB7
:10FFB0002020307825303878207231322F69703A1D
:10FFC0002020307825303878207231342F6C723A06
:10FFD00020203078253038780A0020787073723A03
:10FFE00020203078253038780A004661756C7469B5
:10FFF0006E6720696E737472756374696F6E2061C9
:020000021000EC
:1000000064647265737320287231352F7063293AE6
:10001000203078253038780A00556E68616E646C3F
:100020006564204952516E3A2025640A002A2A2A22
:100030002A2A204D5055204641554C54202A2A2A20
:100040002A2A0A002020537461636B696E67206559
:1000500072726F722028636F6E746578742061729B
:100060006561206D69676874206265206E6F742019
:1000700076616C6964290A002020556E737461638F
:100080006B696E67206572726F720A00202044618E
:100090007461204163636573732056696F6C61748A
:1000A000696F6E0A0020204D4D4641522041646424
:1000B000726573733A20307825780A002020496EE3
:1000C000737472756374696F6E20416363657373D3
:1000D0002056696F6C6174696F6E0A002020466C4F
:1000E0006F6174696E672D706F696E74206C617AD0
:1000F00079207374617465207072657365727661BE
:1001000074696F6E206572726F720A002A2A2A2A39
:100110002A205553414745204641554C54202A2A10
:100120002A2A2A0A0020204469766973696F6E20A2
:100130006279207A65726F0A002020556E616C69C1
:10014000676E6564206D656D6F72792061636365AC
:1001500073730A0020204E6F20636F70726F6365A7
:1001600073736F7220696E737472756374696F6EE6
:10017000730A002020496C6C6567616C206C6F61AC
:1001800064206F66204558435F52455455524E20B7
:10019000696E746F2050430A002020496C6C6567BB
:1001A000616C20757365206F66207468652045500A
:1001B00053520A002020417474656D707420746F6E
:1001C000206578656375746520756E646566696E13
:1001D000656420696E737472756374696F6E0A006A
:1001E0002A2A2A2A2A20425553204641554C542077
:1001F0002A2A2A2A2A0A002020537461636B696E16
:1002000067206572726F720A002020507265636900
:100210007365206461746120627573206572726F0A
:10022000720A002020424641522041646472657384
:10023000733A20307825780A002020496D70726565
:1002400063697365206461746120627573206572EF
:10025000726F720A002020496E737472756374693C
:100260006F6E20627573206572726F720A0052653C
:1002700073657276656420457863657074696F6E26
:1002800020280053707572696F757320696E7465EC
:100290007272757074202849525120005350534592
:1002A0004C20696E20746872656164206D6F6465AE
:1002B00020646F6573206E6F7420696E646963617A
:1002C0007465205053500A002A2A2A2A2A204841BD
:1002D0005244204641554C54202A2A2A2A2A0A00F0
:1002E0002020427573206661756C74206F6E2076D5
:1002F0006563746F72207461626C652072656164FD
:100300000A0020204465627567206576656E740A70
:100310000020204661756C7420657363616C6174A4
:10032000696F6E20287365652062656C6F77290A96
:1003300000415243485F4558434550542077697403
:100340006820726561736F6E2025780A0A002A2A78
:100350002A2A2A204465627567206D6F6E69746F62
:100360007220657863657074696F6E202A2A2A2A64
:100370002A0A002A2A2A2A2A2025732025642920CD
:100380002A2A2A2A2A0A00464C4153485F30005341
:1003900052414D5F300000000000000000FFFFFFF1
:1003A000FFFFFF0000000000000104000200000049
:1003B0000200000000000000050000000000000036
:1003C000000000000000000005574553545F544FE3
:1003D000504449522F7A65706879722F7375627331
:1003E00079732F626C7565746F6F74682F686F73A3
:1003F000742F6863695F636F72652E63006576743E
:100400005F666C6167732026202831554C203C3C88
:10041000202830292900415353455254494F4E203A
:100420004641494C205B25735D20402025733A25C9
:10043000640A0062745F6863695F6576745F67650C
:10044000745F666C616773286864722D3E657674AC
:10045000292026202831554C203C3C2028312929B0
:100460000062756600737563636573730009636F7B
:100470006D6D616E64206F70636F646520307825E8
:100480003034782074696D656F75740A0065727216
:10049000203D3D20300009436F6E74726F6C6C65B7
:1004A0007220756E726573706F6E736976652C203D
:1004B000636F6D6D616E64206F70636F6465203073
:1004C00078253034782074696D656F75742077698C
:1004D0007468206572722025640A004254205258C4
:1004E00020575100574553545F544F504449522FA1
:1004F0007A65706879722F7375627379732F626C85
:100500007565746F6F74682F686F73742F68636993
:100510005F636F6D6D6F6E2E630006010501040150
:1005200007020301050202010302050401010102A1
:100530000103010401060108010C0110011801204A
:1005400001400180616463403430303037303030F6
:1005500000636C6F636B40343030303030303000CB
:1005600072616E646F6D4034303030643030300012
:100570006770696F4035303030303030300073781C
:100580003135303962403365006932634034303090
:100590003034303030006932634034303030333002
:1005A000303000000102030405060773706B2D70E4
:1005B00077722D6374726C007664642D7077722D7F
:1005C0006374726C00FF11E5728A636373383131B2
:1005D0004035610074656D704034303030633030C8
:1005E0003000687473323231403566000001020217
:1005F000000102006C6973326468313240313900A5
:100600006C7073323268625F707265737340356309
:100610000009636F6E76657273696F6E2072657321
:10062000756C74206973206F7574206F6620726119
:100630006E67650A00766261747400756172744059
:100640003430303032303030000000000001000023
:100650000001010000010101010000000000010192
:1006600001015465726D696E616C0000000000004C
:100670000054545220524547474553006D61696EFE
:1006800000737973776F726B71002A2A2A20426F88
:100690006F74696E67205A6570687972204F5320B5
:1006A0006275696C642076342E332E30202A2A2A13
:1006B0000A00286E756C6C29002A666C6F61742ABA
:0406C0000000000036
:1006CC00000000000000000000000000000000001E
:1006DC00000000000000000000000000000000000E
:1006EC0000000000000000000000000000000000FE
:1006FC0000000000000000000000000000000000EE
:10070C0000000000000000000000000000000000DD
:10071C0000000000000000000000000000000000CD
:10072C0000000000000000000000000000000000BD
:10073C0000000000000000000000000000000000AD
:10074C00000000000000000000000000000000009D
:10075C00000000000000000000000000000000008D
:10076C00000000000000000000000000000000007D
:10077C00000000000000000000000000000000006D
:10078C0000000000000000000D250000000000002B
:10079C00000000000000000000000000000000004D
:1007AC00000000000000000000000000000000003D
:1007BC00000000000000000000000000000000002D
:1007CC00000000000000000000000000000000001D
:1007DC00000000000000000000000000000000000D
:1007EC0000000000000000000000000000000000FD
:1007FC0000000000ECF6000000000000FC050020EA
:10080C00FC05002000000000010000000C06002088
:10081C000C06002014060020140600200000000026
:10082C000100000024060020240600200000000027
:10083C0000000000000000000000000000000000AC
:10084C00000000000000000000000000000000009C
:10085C00000000000000000000000000000000008C
:10086C00000000000000000000000000000000007C
:10087C00000000000000000000000000000000006C
:10088C00000000000000000000000000000000005C
:10089C00000000000000000000000000000000004C
:1008AC00000000000000000051CF0000000000001C
:1008BC008FD30000000000000000000000000000CA
:1008CC006BD50000000000000000000000000000DC
:1008DC002D1E0000000000000000000000000000C1
:1008EC00C40E002000000000814B0000000000003E
:1008FC00CC0E002000000000594400000000000055
:10090C00D40E002000000000E55D00000000000097
:10091C00DC0E002000000000194400000000000064
:10092C007C15002000000000FD65000000000000A8
:10093C00D4150020000000002D5B0000000000001A
:10094C00FC1600200000000095370000000000009D
:10095C00F416002000000000953700000000000095
:10096C00EC16002000000000053400000000000020
:10097C00E416002000000000953700000000000085
:10098C00DC16002000000000053400000000000010
:10099C00D416002000000000953700000000000075
:1009AC00000000000000000000000000000000003B
:1009BC000000000000000000B8070020B80700206D
:1009CC000100000001000000C8070020C80700203B
:1009DC0068250000D14A0000A3950000E9C0010081
:1009EC00FF0000003FC00F0090020000EC07002049
:1009FC00EC070020FFFF01000200030000040000D0
:020A0C000000E8
:100A0E0000000000000000000000000000000000D8
:100A1E0000000000000000000000000000000000C8
:060A2E00000000000000C2
:100A34000000000000000000300800203008002002
:100A440038080020380800200300030000000000DC
:100A54000000000090FB00002C3C0020000000007F
:100A6400000000005C0800205C08002064080020EE
:100A740064080020010001000000000000000000E4
:100A8400E8FB0000D83D002000000000000000004A
:100A94008808002088080020900800209008002082
:100AA4000A000A0004000000011B00007CFB000097
:100AB400883A00200000000000000000B408002074
:100AC400B4080020BC080020BC080020010001007C
:100AD4000000000000000000A4FB0000783D00209E
:040AE40015E015E024
:040000030000132DB9
:00000001FF
